:020000040801F1
:1000000050C70020CD3B010831790508B93B0108F4
:10001000B93B0108B93B0108B93B0108B93B0108EC
:10002000000000000000000000000000253C010866
:10003000B93B010800000000713E01087DA50108E0
:100040002D3F01082D3F01082D3F01082D3F0108DC
:100050002D3F01082D3F01082D3F01082D3F0108CC
:100060002D3F01082D3F01082D3F01082D3F0108BC
:100070002D3F01082D3F01082D3F01082D3F0108AC
:100080002D3F01082D3F01082D3F01082D3F01089C
:100090002D3F01082D3F01082D3F01082D3F01088C
:1000A0002D3F01082D3F01082D3F01082D3F01087C
:1000B0002D3F01082D3F01082D3F01082D3F01086C
:1000C0002D3F01082D3F01082D3F01082D3F01085C
:1000D0002D3F01082D3F01082D3F01082D3F01084C
:1000E0002D3F01082D3F01082D3F01082D3F01083C
:1000F0002D3F01082D3F01082D3F01082D3F01082C
:100100002D3F01082D3F01082D3F01082D3F01081B
:100110002D3F01082D3F01082D3F01082D3F01080B
:100120002D3F01082D3F01082D3F01082D3F0108FB
:100130002D3F01082D3F01082D3F01082D3F0108EB
:100140002D3F01082D3F01082D3F01082D3F0108DB
:100150002D3F01082D3F01082D3F01082D3F0108CB
:100160002D3F01082D3F01082D3F01082D3F0108BB
:100170002D3F01082D3F01082D3F01082D3F0108AB
:100180002D3F01082D3F01082D3F01082D3F01089B
:100190002D3F01082D3F01082D3F01082D3F01088B
:1001A0002D3F01082D3F01082D3F01082D3F01087B
:1001B0002D3F01082D3F01082D3F01082D3F01086B
:1001C0002D3F01082D3F01082D3F01082D3F01085B
:1001D0002D3F01082D3F01082D3F01082D3F01084B
:1001E0002D3F01082D3F01082D3F01082D3F01083B
:1001F0002D3F01082D3F01082D3F01082D3F01082B
:080200002D3F01082D3F01080C
:1002080081F0004102E000BF83F0004330B54FEABF
:1002180041044FEA430594EA050F08BF90EA020F2C
:100228001FBF54EA000C55EA020C7FEA645C7FEABF
:10023800655C00F0E2804FEA5454D4EB5555B8BFE2
:100248006D420CDD2C4480EA020281EA030382EA53
:10025800000083EA010180EA020281EA0303362DE5
:1002680088BF30BD11F0004F4FEA01314FF4801CB8
:100278004CEA113102D0404261EB410113F0004FCA
:100288004FEA03334CEA133302D0524263EB430381
:1002980094EA050F00F0A780A4F10104D5F1200E1F
:1002A8000DDB02FA0EFC22FA05F2801841F100017A
:1002B80003FA0EF2801843FA05F359410EE0A5F14E
:1002C80020050EF1200E012A03FA0EFC28BF4CF07F
:1002D800020C43FA05F3C01851EBE37101F0004535
:1002E80007D54FF0000EDCF1000C7EEB00006EEB42
:1002F8000101B1F5801F1BD3B1F5001F0CD34908CC
:100308005FEA30004FEA3C0C04F101044FEA445222
:1003180012F5800F80F09A80BCF1004F08BF5FEAA9
:10032800500C50F1000041EB045141EA050130BD89
:100338005FEA4C0C404141EB0101013C28BFB1F59B
:10034800801FE9D291F0000F04BF01460020B1FAE6
:1003580081F308BF2033A3F10B03B3F120020CDAB9
:100368000C3208DD02F1140CC2F10C0201FA0CF097
:1003780021FA02F10CE002F11402D8BFC2F1200CFC
:1003880001FA02F120FA0CFCDCBF41EA0C019040B2
:10039800E41AA2BF01EB0451294330BD6FEA0404FB
:1003A8001F3C1CDA0C340EDC04F11404C4F12002E6
:1003B80020FA04F001FA02F340EA030021FA04F3F8
:1003C80045EA030130BDC4F10C04C4F1200220FA4F
:1003D80002F001FA04F340EA0300294630BD21FA8D
:1003E80004F0294630BD94F0000F83F4801306BF53
:1003F80081F480110134013D4EE77FEA645C18BF47
:100408007FEA655C29D094EA050F08BF90EA020FDD
:1004180005D054EA000C04BF1946104630BD91EAD5
:10042800030F1EBF0021002030BD5FEA545C05D1D8
:100438004000494128BF41F0004130BD14F5800417
:100448003CBF01F5801130BD01F0004545F0FE418B
:1004580041F470014FF0000030BD7FEA645C1ABFC0
:10046800194610467FEA655C1CBF0B46024650EAF7
:10047800013406BF52EA033591EA030F41F4002123
:1004880030BD00BF90F0000F04BF0021704730B5A9
:100498004FF4806404F132044FF000054FF000017E
:1004A80050E700BF90F0000F04BF0021704730B53F
:1004B8004FF4806404F1320410F0004548BF404214
:1004C8004FF000013EE700BF42004FEAE2014FEA69
:1004D80031014FEA02701FBF12F07F4393F07F4F44
:1004E80081F06051704732F07F4208BF704793F047
:1004F8007F4F04BF41F40021704730B54FF460745A
:1005080001F0004521F000411CE700BF50EA01025C
:1005180008BF704730B54FF000050AE050EA010205
:1005280008BF704730B511F0004502D5404261EB75
:1005380041014FF4806404F132045FEA915C3FF4B6
:10054800D8AE4FF003025FEADC0C18BF03325FEA53
:10055800DC0C18BF033202EBDC02C2F1200300FA04
:1005680003FC20FA02F001FA03FE40EA0E0021FA29
:1005780002F11444BDE600BF70B54FF0FF0C4CF417
:10058800E06C1CEA11541DBF1CEA135594EA0C0FC9
:1005980095EA0C0F00F0DEF82C4481EA030621EA04
:1005A8004C5123EA4C5350EA013518BF52EA03353F
:1005B80041F4801143F4801338D0A0FB02CE4FF0F1
:1005C8000005E1FB02E506F00042E0FB03E54FF021
:1005D8000006E1FB03569CF0000F18BF4EF0010E19
:1005E800A4F1FF04B6F5007F64F5407404D25FEA15
:1005F8004E0E6D4146EB060642EAC62141EA5551C8
:100608004FEAC52040EA5E504FEACE2EB4F1FD0C09
:1006180088BFBCF5E06F1ED8BEF1004F08BF5FEA87
:10062800500E50F1000041EB045170BD06F0004639
:1006380046EA010140EA020081EA0301B4EB5C04E6
:10064800C2BFD4EB0C0541EA045170BD41F48011DE
:100658004FF0000E013C00F3AB8014F1360FDEBF03
:10066800002001F0004170BDC4F10004203C35DADF
:100678000C341BDC04F11404C4F1200500FA05F362
:1006880020FA04F001FA05F240EA020001F0004203
:1006980021F0004110EBD37021FA04F642EB060179
:1006A8005EEA430E08BF20EAD37070BDC4F10C04A3
:1006B800C4F1200500FA04F320FA05F001FA04F267
:1006C80040EA020001F0004110EBD37041F1000153
:1006D8005EEA430E08BF20EAD37070BDC4F120055E
:1006E80000FA05F24EEA020E20FA04F301FA05F2C6
:1006F80043EA020321FA04F001F0004121FA04F26E
:1007080020EA020000EBD3705EEA430E08BF20EA3D
:10071800D37070BD94F0000F0FD101F00046400077
:1007280041EB010111F4801F08BF013CF7D041EAF9
:10073800060195F0000F18BF704703F000465200FD
:1007480043EB030313F4801F08BF013DF7D043EACE
:100758000603704794EA0C0F0CEA135518BF95EA84
:100768000C0F0CD050EA410618BF52EA4306D1D10B
:1007780081EA030101F000414FF0000070BD50EA2A
:10078800410606BF1046194652EA430619D094EAB4
:100798000C0F02D150EA013613D195EA0C0F05D19E
:1007A80052EA03361CBF104619460AD181EA0301F2
:1007B80001F0004141F0FE4141F470014FF00000AA
:1007C80070BD41F0FE4141F4780170BD70B54FF045
:1007D800FF0C4CF4E06C1CEA11541DBF1CEA1355C5
:1007E80094EA0C0F95EA0C0F00F0A7F8A4EB0504A7
:1007F80081EA030E52EA03354FEA013100F088809E
:100808004FEA03334FF0805545EA131343EA126366
:100818004FEA022245EA111545EA10654FEA00261B
:100828000EF000419D4208BF964244F1FD0404F5D4
:10083800407402D25B084FEA3202B61A65EB030530
:100848005B084FEA32024FF480104FF4002CB6EBED
:10085800020E75EB030E22BFB61A754640EA0C006D
:100868005B084FEA3202B6EB020E75EB030E22BFAD
:10087800B61A754640EA5C005B084FEA3202B6EBEE
:10088800020E75EB030E22BFB61A754640EA9C00AD
:100898005B084FEA3202B6EB020E75EB030E22BF7D
:1008A800B61A754640EADC0055EA060E18D04FEA3B
:1008B800051545EA16754FEA06164FEAC30343EADB
:1008C80052734FEAC2025FEA1C1CC0D111F4801FA8
:1008D8000BD141EA00014FF000004FF0004CB6E7A1
:1008E80011F4801F04BF01430020B4F1FD0C88BF40
:1008F800BCF5E06F3FF6AFAEB5EB030C04BFB6EB4B
:10090800020C5FEA500C50F1000041EB045170BD3D
:100918000EF0004E4EEA113114EB5C04C2BFD4EB6A
:100928000C0541EA045170BD41F480114FF0000EEE
:10093800013C90E645EA060E8DE60CEA135594EA6A
:100948000C0F08BF95EA0C0F3FF43BAF94EA0C0F6D
:100958000AD150EA01347FF434AF95EA0C0F7FF4E2
:1009680025AF104619462CE795EA0C0F06D152EA36
:1009780003353FF4FDAE1046194622E750EA41061A
:1009880018BF52EA43067FF4C5AE50EA41047FF42B
:100998000DAF52EA43057FF4EBAE12E74FF0FF3C90
:1009A80006E000BF4FF0010C02E000BF4FF0010C61
:1009B8004DF804CD4FEA410C7FEA6C5C4FEA430CDA
:1009C80018BF7FEA6C5C1BD001B050EA410C0CBF29
:1009D80052EA430C91EA030F02BF90EA020F00208B
:1009E800704710F1000F91EA030F58BF994208BFF2
:1009F80090422CBFD8176FEAE37040F001007047AF
:100A08004FEA410C7FEA6C5C02D150EA013C07D105
:100A18004FEA430C7FEA6C5CD6D152EA033CD3D050
:100A28005DF8040B704700BF8446104662468C464A
:100A38001946634600E000BF01B5FFF7B7FF00287D
:100A480048BF10F1000F01BD4DF808EDFFF7F4FFA6
:100A58000CBF012000205DF808FB00BF4DF808ED31
:100A6800FFF7EAFF34BF012000205DF808FB00BF54
:100A78004DF808EDFFF7E0FF94BF012000205DF876
:100A880008FB00BF4DF808EDFFF7CEFF94BF01202B
:100A980000205DF808FB00BF4DF808EDFFF7C4FF24
:100AA80034BF012000205DF808FB00BF4FEA410277
:100AB80012F5001215D211D56FF47873B3EB6252A8
:100AC80012D94FEAC12343F0004343EA505311F0CF
:100AD800004F23FA02F018BF404270474FF0000061
:100AE800704750EA013005D111F0004008BF6FF09F
:100AF800004070474FF00000704700BF4FEA4102C6
:100B0800B2F1E04324BFB3F5001CDCF1FE5C0DD963
:100B180001F0004C4FEAC0024CEA5070B2F1004FAD
:100B280040EB830008BF20F00100704711F0804FB0
:100B380021D113F13872BCBF01F00040704741F475
:100B480080114FEA5252C2F11802C2F1200C10FA79
:100B58000CF320FA02F018BF40F001004FEAC1235D
:100B68004FEAD32303FA0CFC40EA0C0023FA02F301
:100B78004FEA4303CCE77FEA625307D150EA0133D7
:100B88001EBF4FF0FE4040F44000704701F00040A7
:100B980040F0FE4040F40000704700BF80F0004085
:100BA80002E000BF81F0004142001FBF5FEA41033D
:100BB80092EA030F7FEA226C7FEA236C6AD04FEA3D
:100BC8001262D2EB1363C1BFD21841404840414082
:100BD800B8BF5B42192B88BF704710F0004F40F434
:100BE800000020F07F4018BF404211F0004F41F450
:100BF800000121F07F4118BF494292EA030F3FD01C
:100C0800A2F1010241FA03FC10EB0C00C3F120032E
:100C180001FA03F100F0004302D5494260EB4000BD
:100C2800B0F5000F13D3B0F1807F06D340084FEA28
:100C3800310102F10102FE2A51D2B1F1004F40EB1D
:100C4800C25008BF20F0010040EA03007047490085
:100C580040EB0000013A28BFB0F5000FEDD2B0FA22
:100C680080FCACF1080CB2EB0C0200FA0CF0AABF45
:100C780000EBC25052421843BCBFD04018437047E3
:100C880092F0000F81F4000106BF80F400000132E9
:100C9800013BB5E74FEA41037FEA226C18BF7FEAC0
:100CA800236C21D092EA030F04D092F0000F08BF02
:100CB8000846704790EA010F1CBF0020704712F0E9
:100CC8007F4F04D1400028BF40F00040704712F128
:100CD80000723CBF00F50000704700F0004343F08D
:100CE800FE4040F4000070477FEA226216BF0846C3
:100CF8007FEA23630146420206BF5FEA412390EA86
:100D0800010F40F4800070474FF0000304E000BF7B
:100D180010F0004348BF40425FEA000C08BF70472C
:100D280043F0964301464FF000001CE050EA0102F0
:100D380008BF70474FF000030AE000BF50EA010205
:100D480008BF704711F0004302D5404261EB4101F2
:100D58005FEA010C02BF84460146002043F0B64317
:100D680008BFA3F18053A3F50003BCFA8CF2083A3C
:100D7800A3EBC25310DB01FA02FC634400FA02FC45
:100D8800C2F12002BCF1004F20FA02F243EB02004C
:100D980008BF20F00100704702F1200201FA02FCAE
:100DA800C2F1200250EA4C0021FA02F243EB0200A1
:100DB80008BF20EADC7070477BB972B90029BEBF52
:100DC80000204FF0004106E008BF00281CBF6FF06C
:100DD80000414FF0FF3000F077B8ADF1080C6DE935
:100DE80004CE002909DB002B1ADB00F0A9F8DDF896
:100DF80004E0DDE9022304B07047404261EB4101A1
:100E0800002B1BDB00F09CF8DDF804E0DDE9022391
:100E180004B0404261EB4101524263EB4303704727
:100E2800524263EB430300F08BF8DDF804E0DDE9A0
:100E3800022304B0404261EB41017047524263EB28
:100E4800430300F07DF8DDF804E0DDE9022304B097
:100E5800524263EB4303704753B94AB9002908BFAC
:100E680000281CBF4FF0FF314FF0FF3000F02CB8C6
:100E7800ADF1080C6DE904CE00F062F8DDF804E08D
:100E8800DDE9022304B07047D0B5FFF71DFB00224F
:100E98000B4B06460F46FFF76FFB00F017F80446AA
:100EA800FFF7F0FA0022074BFFF766FB02460B46F6
:100EB80030463946FFF7A8F900F008F82146D0BDBA
:100EC8000000F03D0000F041704700BF4A0011D219
:100ED80012F5001211D20DD56FF47873B3EB62528C
:100EE8000ED44FEAC12343F0004343EA505323FA98
:100EF80002F070474FF00000704750EA013002D10D
:100F08004FF0FF3070474FF00000704710F8012B8A
:100F180011F8013B012A28BF9A42F7D0D01A70472E
:100F2800034611F8012B03F8012B002AF9D1704769
:100F3800034613F8012B002AFBD1181A0138704711
:100F48002DE9F0478C468E46089E154604461946FC
:100F5800002B40F0D080724547D9B2FA82F74FB1E2
:100F6800C7F120030EFA07FCBD40BC4020FA03F38A
:100F780043EA0C0C4FEA154EA8B2230CBCFBFEF852
:100F88000EFB18CC08FB00F943EA0C43994528D915
:100F9800EB1808F1FF3204D2994502D9A8F10202F0
:100FA8002B44A3EB0903A4B2B3FBFEFC0EFB1C33DA
:100FB8000CFB00F044EA0344A04214D92C190CF1AC
:100FC800FF3304D2A04202D9ACF102032C44241A04
:100FD80043EA02401EB1FC40002334607360BDE860
:100FE800F0874246DDE76346F1E7002A79D0B2FA96
:100FF80082F3002B3FD01946C1F1200302FA01F514
:1010080000FA01F42EFA03F20EFA01FE20FA03F3B5
:10101800AFB243EA0E034FEA154EB2FBFEFC0EFBDD
:101028001C201A0C0CFB07F842EA004290455AD9DA
:10103800AA180CF1FF3004D2904502D9ACF1020095
:101048002A44A2EB08029BB2B2FBFEFC0EFB1C2258
:101058000CFB07F743EA02439F4246D9EB180CF111
:10106800FF3204D29F4202D9ACF102022B44DB1BAF
:1010780042EA004202E0AEEB020301224FEA154EBB
:10108800AFB2200CB3FBFEFC0EFB1C330CFB07F8C5
:1010980040EA034398452AD9EB180CF1FF3004D2F3
:1010A800984502D9ACF102002B44A3EB0803A4B283
:1010B800B3FBFEFC0EFB1C330CFB07F744EA0344AE
:1010C800A74216D92C190CF1FF3304D2A74202D932
:1010D800ACF102032C44E41B43EA00400F461146DE
:1010E80078E71F2188E76046ABE76246BFE76046BE
:1010F800DBE76346EFE7734506D916B900210846D2
:101108006DE7C6E9000EF9E7B3FA83F787B97345C7
:1011180001D3824207D8841A6EEB030301209C4650
:101128001EB900215BE73846FAE7C6E9004CF8E744
:10113800C7F1200CBB4000FA07F422FA0CF520FA9C
:101148000CF1BA401D432EFA0CF30EFA07FE4FEAD3
:10115800154941EA0E011FFA85FEB3FBF9F809FBB0
:1011680018300B0C08FB0EFA43EA00439A4540D9A5
:10117800EB1808F1FF3004D29A4502D9A8F1020011
:101188002B44A3EB0A0389B2B3FBF9F809FB183324
:1011980008FB0EFE41EA03418E452CD9691808F177
:1011A800FF3304D28E4502D9A8F10203294443EA49
:1011B8000040A1EB0E01A0FB02984145CE464346F4
:1011C80002D306D14C4504D20138B9EB020E68EBC4
:1011D8000503002EA5D0B4EB0E0261EB030101FA62
:1011E8000CFC22FA07F3F9404CEA0303C6E9003184
:1011F80097E74046C5E74346D9E7000000000000EE
:101208002DE9F04F984685B000F15803C0E9163330
:10121800129B0026838104239FED257B073222F051
:10122800070A0374119B01EB0A090F4680ED087B3E
:101238004946C0E9066686608373C6730446DDF8CE
:1012480038B002F06BFA109BC51D25F00705C4F8ED
:101258008850C4E9207A02930F9BA9EB0505CDE9D4
:1012680000B32A4643463946204602F061FD0F9BEB
:10127800C4E91B8B6367109B6665A367EFF3118254
:10128800102383F31288BFF36F8F0B4B596A5C628C
:10129800E16782F31188BFF36F8F9B680BB1D3F8B6
:1012A8008C302846C4F88C3005B0BDE8F08F00BFFC
:1012B8000000000000000000D43B002000000000F7
:1012C8001FB513A3D3E90023FFF776FD01A926F084
:1012D80065FB9DF807309DF806201B0443EA42533E
:1012E8009DF80820BDF8040043EAC2239DF80920B0
:1012F800A0F2BC7043EA42139DF80A2043EA520365
:1013080043EA406005B05DF804FB00BFAFF300801E
:1013180000CA9A3B000000002DE9F0412DED028B38
:1013280090F8AD300446B0EE408A86B01BB9F7EEAF
:10133800007A37EEC08AD4F884202F4B9A4213D112
:1013480018EE100AFFF7C0F829A3D3E90023FFF726
:10135800A3FB011E18BF012104F184000EF092FEC8
:1013680084ED288A012005E0B4F8A430B3F5807F25
:1013780005D1002006B0BDEC028BBDE8F08104F178
:10138800500840462AF0D6FF0028F2D0DFED1B7A3D
:1013980068EE277AFCEEE77ACDED037A94F8806060
:1013A80094F8A4209DF80C30276E206D6EB18DF84E
:1013B800153002238DF8142000210122009305AB7B
:1013C800B847404656F0F6F9CAE7012531468DF888
:1013D80013208DF814302A460DF113030095B847F1
:1013E800009532462946276E206D05ABE8E700BF19
:1013F800AE47E17A14AEEF3FACC5070800007F4363
:101408002DE9F04F044685B00846616006219046F4
:101418001D469DF838709DF83CB01AF013F8A0608E
:10142800067C16F0010602D07F4820F081F89DF86E
:10143800403005FB08F084F82A309DF844307D30B0
:1014480084F828307E2390FBF3F0C0011630B0F505
:10145800D07F38BF4FF4D070C4E904852773606229
:101468004DF037FF0DF1080A0622C4E907066F4957
:101478002046A66162F084F8022251462046ADF863
:10148800088062F07DF8022251462046ADF80850E7
:1014980062F076F8F623032269462046ADF800305C
:1014A8008DF8026062F06CF87B1EDBB2082B05D861
:1014B80040F25515DD4015F0010501D15C48B4E74F
:1014C800052F09D0072F06D0032F73D1012384F8E5
:1014D8002930002502E02E4684F82960002646F3CC
:1014E8004F10C0EB0020FEF7DDFF0022514BFEF746
:1014F8008DFE0022504BFFF769F9FFF7D7FA5FFA24
:1015080080F8C6F38200C0EB0020FEF7CBFF002274
:101518004A4BFEF77BFE0022494BFFF757F9FFF7CE
:10152800C5FAC7B206F00300C0EB0020FEF7BAFF09
:101538000022404BFEF76AFE00223F4BFFF746F9B8
:10154800FFF7B4FAC0B2002D5ED08DF808008DF810
:1015580009808DF80A70032251462046013662F050
:101568000FF8802EBBD1BBF1000F1AD0354D01A961
:101578002A88AB782046ADF8042003228B7061F0EE
:10158800FFFF0B222046304961F0FAFFD5F803002F
:10159800EB7902900522514620468AF8043061F022
:1015A800EFFF204661F0DAFFA06961F0FBFF05B0AC
:1015B800BDE8F08F092F84F829608AD10FF2580905
:1015C800D9E90089354616A7D7E900672846FEF706
:1015D80069FF42464B46FEF719FE32463B46FFF787
:1015E800F5F8FFF763FAC0B28DF808008DF8090026
:1015F8008DF80A00032251462046FF3561F0C0FFEE
:10160800B5F5FF4FE2D1AEE78DF808808DF8097087
:101618008DF80A009FE700BF0000000000C04F409F
:101628000000000000C05F40948E0808914308083D
:10163800758608080000F83F0000084000000C40CC
:1016480000001C40FA5607089843080800000000EC
:1016580010EE103A33F0004210B52DED028B06D192
:101668000120BDEC028BBDE8104044F0B9BA002B54
:1016780005DABDEC028BBDE8104044F0BFBAB3F107
:10168800FF4F06DB30EE008AB0EE480ABDEC028B55
:1016980010BDB3F5000F6049BBBFDFED607A6FF096
:1016A8001802002260EE277AB8BF17EE903AF7EEDC
:1016B800007ADC15C3F316037F3C1944144401F483
:1016C800000282F07E5204EBD15403F10F011A4359
:1016D80007EE102A524A0A4037EE678AB2BBB5EEC7
:1016E800408AF1EE10FA0FD1002C00F08C8007EE42
:1016F800904A9FED4C0A9FED4C7AF8EEE77A27EE78
:10170800808A07EE878ABFE741A1D1E90001FFF788
:10171800F5F9B6EE007A07EE900A07EEC87A68EE99
:10172800087A27EE277A14B938EE478AACE707EE2D
:10173800904ADFED3C6AF8EEE77A07EEE67A37EE94
:10174800488A9FED397A17EE878A9DE7F0EE007A8E
:101758009FED365ADFED364A364A78EE277A1A4434
:10176800C3F5571388EE276A07EE904A03F52273EC
:101778001343F8EEE76ADFED307A002B66EE065A7F
:1017880025EEA57A07EE275ADFED2C7A45EE077A83
:101798009FED2B5A07EE875ADFED2A7A47EE274A44
:1017A800DFED297A44EE877A67EE877A45EE257A67
:1017B8001ADDB6EE007A28EE077A27EE087A77EE79
:1017C800877A67EE867A14B937EE677AACE79FEDC9
:1017D800156A46EE867A37EE677A37EE488ADFED85
:1017E800127A16EEA78A4FE778EE677A67EE867A5E
:1017F80014B938EE678A47E79FED0A7A46EEC77A4A
:1018080037EEC88AEBE79FED118A3DE7AFF300801A
:10181800555555555555D53F20FB4A000000004CFD
:10182800F0FF7F00D1F717378071313F25333A3EFB
:10183800298E633E305CCFFF9788173E2549923E3C
:10184800ABAA2A3F4FD01C3ECDCCCC3E00000000B6
:10185800F8B510EE904A10EE103A34F000472DED2E
:10186800048BB0EE609A0DD183F480035B0013F50E
:10187800000F40F2AA8230EE098AB0EE480ABDECA9
:10188800048BF8BD23F000411846B1F1FF4F02D890
:10189800B7F1FF4F08D9B3F17E5FECD184F480042F
:1018A800640014F5000FE4E7002B25DAB7F1974F31
:1018B80080F09482B7F17E5F39D3FA15C2F19602AF
:1018C80047FA02F505FA02F2BA4229D105F00105F4
:1018D800C5F10205B7F17E5F2AD1002C80F27B8228
:1018E800B5EE400AF1EE10FA1CD1D80FBDEC048B0E
:1018F800BDE8F84044F074B9B7F1FF4F10D1B1F129
:101908007E5F00F0628205D9002CDFEDD17A29FED6
:10191800278AB2E7002C80F25B82B1EE498AACE7F5
:101928000025D7E7B7EE007A87EE008AA5E70025FD
:10193800B4F1804F0A4640F05782B1F1BF4F0CD244
:10194800B1F1D05F02D920EE008A96E7B0EEC08AE6
:1019580059BB012D00FE088A8FE723F04046B0EE00
:10196800C08AB6F17E5F17D1002CBCBFB7EE007AF3
:1019780087EE088A002B80DAA1F17E51294305D130
:10198800BDEC048BBDE8F84044F038B9012D7FF474
:1019980074AFB1EE488A70E739B9002CD9DA002B58
:1019A800A4D06B1E58425841A0E7DE0F013E55EA0D
:1019B8000600E5D0B7F19A4F71D9A64B994208D8DD
:1019C800002C0BDA0020BDEC048BBDE8F84044F095
:1019D800F9B8A14B994208D9002CF3DC0020BDECE2
:1019E800048BBDE8F84044F0DFB8B7EE007ADFEDCD
:1019F8009B7ADFED9B9A38EE478A93A1D1E90001E3
:101A080068EE278AFFF77AF8B5EE007A07EE900AB3
:101A1800DFED946A68EE299A48EE477AB6EE007AC6
:101A280007EEC87A68EE087A27EE277AF0EE687A29
:101A380047EE667A39EEA77A17EE103A6FF30B0382
:101A480007EE103A77EE699A77EEE97A013DF7EEFC
:101A5800006ABFEE008A6FF30B04354367EE890A0C
:101A680008FE268A06EE904A39EE666A67EE267AFE
:101A780046EE070A30EEA77A17EE101A002921F071
:101A8800004340F31381B3F1864F40F2CC80B5EEAA
:101A9800C08AF1EE10FA4CBF0120002093E713F042
:101AA800FF4F05BF9FED707A6FF01701002168EEB8
:101AB800077A08BF17EE902AD315C2F316027F3BA8
:101AC80042F07E500B4469498A4206DD68498A42E1
:101AD80040F3A7800133A0F500000021654A06EE17
:101AE800100AF7EE006A02EB8102D2ED005A75EE99
:101AF800867A36EE657AC6EEA74A27EE245A15EEA0
:101B0800102A6FF30B0206EE902A5B4A02EA600283
:101B180042F0005202F5800202EB415207EE902A91
:101B280006EEE77A77EEE57ADFED545A36EE676A25
:101B380065EE057A06EE667A9FED516A47EE865A9B
:101B48009FED506A27EE247A66EEA64A05EEA76A4C
:101B5800DFED4D5A46EE275A9FED4C6A05EEA76A0F
:101B6800DFED4B5A46EE275A36EE856A67EEA77ABE
:101B780026EE076A05EEA76AF0EE085A74EEA57A13
:101B880077EE867A17EE902A6FF30B0207EE902A0B
:101B980077EEE55A27EE277A66EEA76A75EEE45ADD
:101BA80036EE656A06EE057A9FED3A6A76EE877A32
:101BB80017EE902A6FF30B0207EE902A364A77EE5B
:101BC800E66A02EB810227EE866A37EE667ADFED77
:101BD800336A67EEA67ADFED326A47EE267A92ED2F
:101BE800007A77EE877A07EE103A2E4BF8EEC76A3E
:101BF80003EB810336EE277AD3ED005A37EE257AC8
:101C080037EE267A17EE103A6FF30B0307EE103A09
:101C180077EE666A76EEE56A76EEC66A77EEE67A7B
:101C280014E701215AE755D1DFED1F6A37EE677ACD
:101C380070EEA66AF4EEC76AF1EE10FA3FF727AF26
:101C480086234BE0AFF30080E13D55555555D53F10
:101C580000000000F3FF7F3F0700803F70A5EC36CF
:101C680000AAB83F3BAAB83F0000804B71C41C00D3
:101C7800D6B35D0060FB070800F0FFDF55326C3E0D
:101C880042F1533E05A38B3EABAAAA3EB76DDB3E9D
:101C98009A99193F0040763F50FB0708C623F6B8CB
:101CA8004F38763F58FB07083CAA3833534A9342CB
:101CB80007D9B5EEC08AF1EE10FA4CBF012000201A
:101CC8008DE607D137EE677AB4EEE07AF1EE10FAD6
:101CD800B6DBEEE7B3F17C5F72D9DB157E3B4FF4E0
:101CE8000000474A002940FA03F00844C0F3C753EC
:101CF800A3F17F0342FA03F2C3F1170302EA0002D9
:101D0800C0F3160040F4000007EE102A40FA03F072
:101D180077EEC77AB8BF404237EEA07ADFED396A6E
:101D2800DFED395AB7EE000A9FED386A17EE103A20
:101D38006FF30B0307EE103A77EE677A67EE266AC1
:101D480070EEE70ADFED327A27EE277ADFED317A97
:101D580000EEA77A76EE877A77EEE66A37EE667A4D
:101D680067EEA76A07EE877A16EEA56ADFED2A5AAC
:101D780046EE265A9FED296A15EEA66ADFED285A27
:101D880046EE265AB0EE676A05EEE66AF0EE006A9D
:101D980067EE865A36EE666AC5EE866A36EEC77A0A
:101DA80077EE677A30EE670A10EE103A03EBC0530D
:101DB800B3F5000F06DA43F07BFD20EE088A5CE5F8
:101DC8000020A9E700EE103AF7E7B7EE008A54E5DD
:101DD8009FED148A51E5B0EE408A4EE5B7F1FF4F0A
:101DE8003FF48DAD0A460225B4F17C5F7FF4B5ADB2
:101DF800002BFFF6B2ADB1EEC08A3EE500001643F7
:101E0800000080FF0072313F4CBB31330EEADD35F4
:101E18008CBEBF351872313F55B38A38610B363BDB
:101E2800ABAA2A3E0000000010EE103AB3F1FF4FB3
:101E380010B52DED048BB0EE408A06DB30EE008A3B
:101E4800B0EE480ABDEC048B10BD774A934276DCAD
:101E580023F00042B2F17E5F13D3FFEE007AB4EEB6
:101E6800670AF1EE10FA06D10120BDEC048BBDE83B
:101E7800104043F0B5BEBDEC048BBDE8104043F004
:101E8800BDBEB2F1645F0FD2B2F14A5F24BF20EE4B
:101E9800007AF6EE007ABDEC048B28BF07EE670ADD
:101EA800BDE8104043F0BEBC604A134493424ED88C
:101EB800F7EE007A38EE277A17EE103ADC157F3CF9
:101EC800002CD5BF77EE677A37EE488A78EE677AC6
:101ED80077EEC87A87EE879AC3F31603544A93427B
:101EE800CCBF43F07C5243F07E52F7EE007AC8BF75
:101EF800C3F5000307EE102AC4BF01349B1037EE68
:101F0800678AF6EE008A68EE288A68EE888A002BCF
:101F180044D1B5EE408AF1EE10FA1DD1002C7AD0EA
:101F280007EE904AB0EE498A9FED427AF8EEE77ADA
:101F380007EE878A9FED407A07EE878A80E7B3F13C
:101F4800B44FB5DBDC159FED3D9A7F3CC4E7012318
:101F580000249FED3A9AD4E731A1D1E90001FEF7B8
:101F6800CDFDB7EE007A07EE900A07EEC87A27EEA5
:101F7800287A14B938EE478A62E707EE904ADFED0F
:101F88002D6AF8EEE77A07EEA69A37EE497A37EE29
:101F9800488A9FED297A17EE878A51E7F0EE007A92
:101FA8009FED276A9FED277A78EE277AC8EE276A91
:101FB80066EEA67A07EE867A9FED236A07EE276A11
:101FC8009FED227A06EE277A9FED216A07EE276AAF
:101FD8009FED207A06EE277A9FED1F6A07EE276AA3
:101FE800B0EE687A06EE277A27EE267A24B978EEDC
:101FF800C78A38EE688A23E707EE904ADFED0D6A54
:10200800F8EEE77A07EEA69A39EE079A78EEC98ACB
:1020180038EEC88ABDE79FED098A11E7AFF3008063
:10202800555555555555E53FD613D43EE0096A41F7
:10203800F6043500D1F717378071313F00000000F2
:102048009788173E4FD01C3E25333A3E298E633E73
:102058002549923ECDCCCC3EABAA2A3F2DE9F0478C
:102068000546884600AF44F00AFAA9680646B1F565
:10207800004F36BFA8F10403002303F00703B1F5AE
:10208800004F34BF0420082002F0070407341C4422
:102098000444E40804EBD2048C4228BF0C46012215
:1020A8003146284644F0A5F910EA020A16D1E94655
:1020B80088B06A46504BCDE90538032342F8103FF3
:1020C8004FF4C25153464D4800F09EFECD468AF368
:1020D8001188BFF36F8F0423184602DF3146284664
:1020E80044F09DF906EB000949460022284644F0D1
:1020F80080F9A9EB00094E4518D0E94688B0694631
:102108003F4BCDE90538032341F8103F3B481346C0
:102118000A464FF4C25100F077FE0023CD4683F300
:102128001188BFF36F8F0423184602DF3146284613
:1021380044F075F98442804623D028D2344431468D
:102148002246284644F02DFA01223146284644F01A
:102158006CF9214644F063F92618012231462846D5
:1021680044F047F9C30708D43146284644F0C9F972
:1021780032462146284644F03BFA2146284644F098
:1021880055FA4FF001094846BD46BDE8F08706EB11
:10219800000A01225146284644F02BF910EA0209A8
:1021A80027D15146284644F03AF940448442EAD8B7
:1021B8005146284644F0A5F95146284644F02FF9DF
:1021C800A4EB0808804509D23444514628462246E3
:1021D80044F0E7F92146284644F028FA52463146A9
:1021E800284644F005FA01223146284644F01DF9F4
:1021F800C7E74FF00009C6E794110808F455070827
:10220800B81108082DE9F843884600AF00297DD0A9
:1022180005680122284644F032F90146044628465A
:1022280044F0E7F810EA020616D1E94688B06A4693
:10223800384BCDE90538032342F8103F4FF4C2511B
:102248003346354800F0E0FDCD4686F31188BFF3EC
:102258006F8F0423184602DF2146284644F0DFF832
:10226800261831460022284644F0C3F8361AB442EC
:1022780018D06E4688B06946284BCDE90538032347
:1022880041F8103F244813460A464FF4C25100F063
:10229800BBFD0023B54683F31188BFF36F8F04237A
:1022A800184602DF00222146284644F0BEF821469F
:1022B80044F0B5F8261801223146284644F099F82A
:1022C800C20708D43146284644F01BF93246214655
:1022D800284644F08DF900222146284644F089F822
:1022E800261A01223146284644F083F8C30709D448
:1022F8003146284644F005F922463146284644F03E
:1023080077F934462146284644F090F9BD46BDE8A1
:10231800F88300BFE1110808F4550708B811080848
:1023280008B5024844F01DFD002008BD0E1208083B
:102338000E4A0346904202D30D4A904211D30D4AE9
:1023480022B1934202D30C4A93420AD30B4A52B1A8
:102358000B48834234BF01200020934238BF00203D
:102368007047012070471046704700BF0C5007089F
:102378000CA5080800000000000000000000000094
:10238800000000002DE9F04F9BB000AF04468B46DB
:10239800D7F890A0FA637B6349B9037846788078C8
:1023A80000EB830020445E4522D8A0EB040B0AF022
:1023B800010394F80280FB62E378B8F1000F0CBFC8
:1023C8004FF000090AF001093B6313B11AF0020F3C
:1023D80017D1B9F1000F14D1FB6B1BB15946204638
:1023E8007A6B98475D4628466C37BD46BDE8F08F46
:1023F800451C2846FEF79CFD013028440BF1010BD3
:10240800D1E7CAF3C003FB612378BB629B00BB61C1
:1024180063683B62BB6A04EB8301FB6B002B7DD1D5
:102428005D468844B9F1000F1DD08B469946A94EE8
:102438001BF8013B54F82300002808BF3046FEF77C
:1024480077FDD7F8943001304BB1D7F898304B4529
:1024580082BFD7F8943023F8190009F10109C34560
:102468000544E5D1D8461AF0050F0CBF4FF0020B12
:102478004FF0010B00260AF00203FB633B6B9E4200
:10248800B1D298F8013008F1020854F823A0504658
:10249800FFF74EFFFA69034602B3B86318F8021C47
:1024A800386A44F03FFCBB6BC0B1EA468AB06A4662
:1024B800894B05933B6ACDE906314FF40073ADF8BB
:1024C8002030864B42F8103F00234FF412518448C5
:1024D80000F09AFCD546023D0136CFE723B1FB6AEE
:1024E8002BB9A5EB0B05F7E7FB6B002BF4D079486C
:1024F800BAF1000F18BF5046FEF71AFDD7F894300E
:1025080053B1D7F8983099453FBFD7F89420431C6A
:1025180022F8193009F101090544DDE7B9F1000F86
:102528006DD04346102B28BF10230026BB6397F8B5
:10253800389007F14800BA6B796262F08AFA796AD2
:1025480000227A620AF0020201EB08033A610AF0FB
:1025580004027B61FA6002337A6A396B8A4267D374
:102568006378F96A1AF0020F7B624B4418BF0022A5
:10257800DBB208BF7208002940F0A9801AF0040FE6
:1025880014BF314600216370A170E27020467A6B57
:10259800B969FB6B9847051EFFF625AFBB6A314644
:1025A80023707B6A7A6B63703B6B84F80280E370FC
:1025B80007F15800FB6B9847061EC0F2C5803A6BBE
:1025C800BB69386B03EB4203ABEB0301D7E90D237F
:1025D800C91A7B6903EB4000FB6B98470028C0F2DF
:1025E800B5804FF000082E44351807F1480AC84551
:1025F80078D300217A6B0846FB6B9847F3E6B8F16D
:10260800000F0CD01AF0040F0ED04346102B28BF31
:102618001023BB6397F8386007F158008BE74646EC
:10262800C146C7F838808BE74E46C7F8388087E739
:1026380013F8015C13F8021C54F82500BB60FFF77F
:1026480077FE0246F869BB6838B1386AC7E90132D3
:1026580044F068FBD7E90132F0B912B3FA6A72B1F3
:10266800B9F10F0F18D809F1280107F1400009F155
:102678000102014401F8205C5FFA82F90CE0FA6873
:1026880052B10F2E08D806F1280107F14000721C3C
:102698000E1806F8105CD6B27A6A023301327A62F2
:1026A8005AE73A69002ADBD10F2EF5D806F128003F
:1026B80007F1400C6044721C00F8101C07F1680117
:1026C800023651FA82F2F6B202F8105CE4E7002111
:1026D80059E700BF3C12080843120808040000012B
:1026E8004455070818F80A3054F823B087F84730DB
:1026F800D7F8943033B3D7F89830984522D2D7F822
:10270800943033F8186001217A6BFB6B07F14700AE
:10271800984700281ADB0E4B0544BBF1000F08BF91
:102728009B4626B95846FEF703FC461CB6B231460E
:1027380058467A6BFB6B9847002807DB054408F17D
:10274800010854E70026DEE735464CE605464AE62A
:102758003C120808014B1860704700BF8001002038
:10276800044608B5EFF31183102383F31288BFF3EF
:102778006F8F47F091FF204601F03EFA024844F07F
:10278800F0FA45F0F2F8FCE7F7120808034A0020CF
:10279800536823F002035360704700BF004004E011
:1027A80008B5094A136943F00053136141680748A3
:1027B8000C3183681B681BB1984700EAE07008BDBC
:1027C8006FF05700F9E700BF000802461C510708E0
:1027D800082810B502D90024204610BD044B53F830
:1027E8002040204648F026FC0028F5D1F3E700BF3A
:1027F800B45A070810B5EFF31184102383F3128835
:10280800BFF36F8F084803683BB9084A916A41F0E3
:1028180001019162916AC907FCD50133036084F311
:102828001188BFF36F8F10BDB43600200008024630
:1028380010B5EFF31184102383F31288BFF36F8F61
:1028480011490B68A3B90122104BD3E8EF1F0029E7
:1028580003D1C3E8E02F0028F7D104D102210C4AA4
:102868000C4844F0CDFE84F31188BFF36F8F10BD80
:10287800012B08BF084803F1FF3302BF826A22F028
:10288800010282620B60EEE7B4360020B036002009
:10289800BC1308081C5607080008024607B505F0CF
:1028A800E9FC0E4B0E4A1A600E4BD3F8942042F006
:1028B8000402C3F89420D3F8943003F0040301937E
:1028C800019B094BDA6A42F00102DA629A6822F047
:1028D80002029A6003B05DF804FB00BFC80600203E
:1028E80000093D00000C0246000802462DE9F047A9
:1028F800044607464FF00109DFF84C8094FAA4F526
:10290800B5FA85F509FA05F32E0108EB05156FEA06
:10291800030A24EA03042B7B63B158F806301B69C9
:102928006BB94644736802222846196807EA0A0701
:1029380044F0F6FD002CE1D13846BDE8F087284682
:1029480098470028F6D1ECE7BC56070810B50022D6
:1029580088B00E490E4848F0C6FF00220023002424
:10296800CDE906230E234FF44072CDE90334CDE9B7
:102978000144084B08490094084809F0A9FD084992
:10298800064848F00EFE204608B010BDAD290108E3
:1029980068280020B92C010830500020802300202E
:1029A80004140808014809F0DDBA00BF3C110020F2
:1029B8002DE9F047804620480F4644F08DFD064635
:1029C800002832D000252846BDE8F087237B83B154
:1029D8002368DB680BB120469847636883F8069044
:1029E80023681B69CBB9636802222046196844F042
:1029F80097FD013610345445E8D3B8F1000FE2D002
:102A0800002DDFD02846FFF771FF0546002FF7D0CD
:102A18000021642048F0C7FEF2E7204698470028C6
:102A2800E1D009FA06F31D43E3E705464FF0010933
:102A3800024CDFF80CA0DEE7C8360020BC560708B9
:102A4800CC560708014B53F820007047EC5A07088A
:102A580008B5034608462BB1044A136000F044FC4D
:102A6800002008BD6FF01500FBE700BF84010020BF
:102A780010B5044C237813B9034809F073FA0123FD
:102A8800237010BD2E4900203C11002010B50446CB
:102A9800094844F021FD3CB1084BD3E8EF1F013948
:102AA800C3E8E21F002AF8D105480AF033FBBDE865
:102AB8001040044809F056BAC0360020C436002039
:102AC800682800203C1100200022044BD3E8EF0FB7
:102AD800C3E8E12F0029F9D1704700BFC0360020B4
:102AE80070B5FFF7F1FF0546074C084EB44200D316
:102AF80070BD63685B792BB123685B6813B12946A5
:102B0800204698471034F1E7BC560708CC5607080A
:102B180010B5044C0449204644F031FA034B1C60BC
:102B280010BD00BF54100020D85A0708B83600203E
:102B380000230D4A10B513700C4A4FF47A711360D4
:102B48000B4A0C481360FFF783FFFFF7E1FF0A4BBE
:102B58000A4918468B4200D310BD1A1A5C68121134
:102B6800013222711033F5E72F490020C0360020CA
:102B7800C4360020F3740508BC560708CC5607086D
:102B8800014642F210720023014844F019BA00BF0E
:102B980054100020014844F0AFBA00BF5410002080
:102BA800024B0146186844F002BB00BFB83600204B
:102BB800014844F037BB00BF5410002070B5254BC6
:102BC8001B78002B43D0FFF7E5FF044600283BD1D4
:102BD800214B224D1B68002B12DD48F03CFE0A22D7
:102BE8000023FEF739F9D5E90032C01A40F2E9337B
:102BF80061EB0201984271F1000101D3FFF770FF08
:102C0800D5E9003213F57A7342F10002C5E90032C2
:102C1800ECB1BDE87040FFF7CBBF6B685B7923B1BF
:102C28002B68214628461B6898471035B542F4D3CF
:102C38002046FFF7B5FF0A4BD3E8EF1F0139C3E879
:102C4800E21F002AC4D0F7E7064D074EEEE7002042
:102C580070BD00BF2E490020C0360020602800202B
:102C6800C4360020BC560708CC56070870B50D4D71
:102C7800297861B90120FFF79BFE0B4C0B4EB4423B
:102C880006D3FFF79BFF0028FBD101232B7070BDF3
:102C980063685B791BB1236820469B6898471034AA
:102CA800EDE700BF2F490020BC560708CC5607089F
:102CB80000212DE9F8430846FFF77AFE044648B399
:102CC8004FF4FA784FF0000901F03EF91A4B1B4A0D
:102CD8001B58136033B11A4B1B68092B02DD1948C6
:102CE80009F040F90025184F44B12046FFF7FEFDD2
:102CF800044618B94FF0FF384FF0FF39FFF75EFF71
:102D0800064628B9B5B90F4842464B4609F066F958
:102D18003546E9E74FF0FF384FF0FF39D4E72B6825
:102D28009B691BB100222846114698471035BD42C1
:102D3800F5D3E8E7054DFAE708000000BC360020A7
:102D4800C43600203C110020CC560708BC560708A2
:102D580013B5184844F0C0FB174B1B7873B1EFF359
:102D68001184102383F31288BFF36F8FFFF726FFB8
:102D780084F31188BFF36F8F02B010BD0F4B1B682F
:102D8800002BF9D050B9002200230D48CDE90023CB
:102D980042F2107200230AF097F9EDE70928EBD107
:102DA80007480AF0B7F9074802B0BDE8104009F033
:102DB800D9B800BFC43600202F490020BC360020F7
:102DC800682800203C11002010B5064B04461B68FB
:102DD80098472146A060044844F06FF9BDE81040C8
:102DE800FFF7B6BF8401002054100020044A054BA9
:102DF8009B1AB1EBD30F34BF52F831000020704753
:102E080034550708BC5607082DE9F04F8FB0C1F3B9
:102E18004A2604AF0D469046B8607B600C0D002E24
:102E280061D04FF000090A234FF0040B07F1140A90
:102E3800FE60C7E90799C7F824900093CDF808B059
:102E4800CDF804A007F11C034A464046F968FFF78D
:102E580099FAB0F5006F03461CD36C468AB0D8F8CF
:102E6800041004AB24481A46C3E9050140F2FF7177
:102E7800D9614FF400711984204B42F8103F4FF488
:102E880012514B461E48FFF7BFFFA5462C37BD46DB
:102E9800BDE8F08FC0F30A0604F11700184420F0CB
:102EA800070080083B60FFF76BFE66F35325044676
:102EB80080B13B6800F11001C7E908390A23F961BC
:102EC800CDE901AB009340460E4AF96807F11C03AF
:102ED800FFF758FA66F353252A4620467B68B968F7
:102EE80044F03EFBD2E704F1170020F00700800809
:102EF800FFF746FE0446EDE7151408080400000134
:102F0800BC5507083B7505082DE9F04F87B0054605
:102F1800DDE9106BDDE9127A884614469946BFB19F
:102F280010213B465A460020CDF800A0CDF814A049
:102F380043F01FFDB0F5006F01460BD340F2FF735D
:102F48000221184A184807B0BDE8F04F44F061BBA9
:102F58003946384604F0070305F00704E40044EA5C
:102F6800831444EA402444EA065406F1170008444E
:102F780020F0070080080391FFF702FE054640B1E4
:102F88003FB13B465A460399CDF800A0103043F0B4
:102F9800F0FC4B4622464146284607B0BDE8F04FB4
:102FA80044F0DEBA54140808BC550708406820B13C
:102FB800034BC01A40F3CF0070474FF0FF30704703
:102FC800345507080EB403B503AB53F8042B014678
:102FD8000448019301F0ECF902B05DF804EB03B08A
:102FE800704700BF7D760508CA0605D48B064CBF1E
:102FF80002490349FFF7E6BF704700BF273A0808B0
:10300800113308082DE9F04F8BB099469DF8588088
:10301800179B044607930D46DDE918A31A9F0692ED
:103028000593B8F1000F00F0BC80834B07F0020B4A
:1030380013F80830089307F48073099344F06EFA84
:10304800024600287AD020467C49FFF7BBFF064697
:10305800BBF1000F08D017F0440F71D12A46204663
:103068007749FFF7AFFF064407F0010353B1754BEB
:10307800204653F82820744B7449002A08BF1A4682
:10308800FFF7A0FF07F48073002B07F0080318BFB1
:103098004FF00009002B7FD06D4B204653F82820B5
:1030A8006C49FFF78FFF0546069B2BB11A46204651
:1030B8006949FFF787FF0544B9F1000F0DD0089B58
:1030C800002B6CD06549664BB8F1040F18BF194640
:1030D8004A462046FFF776FF054462483544079B79
:1030E8001BB12246604943F0ECFD059B002B00F024
:1030F8008E80059B3946102B28BF10232046994601
:103108000026FFF771FFB54252DC00263346204601
:103118001AF803205549FFF755FF0136102E4DD0F8
:10312800710703D120465249FFF74CFF4E453346FD
:10313800EDD320464F49FFF745FFEEE7064687E700
:103148004D4B186800288ED04C4B4FF47A7B1B6887
:103158004FF03C0CB5FBF3F5B5FBF0F14FF46163B0
:1031680000FB11550BFB05F5B1FBF3F2B5FBF0FEC7
:1031780003FB121100FB1E55B1FBFCF30BFB05F51D
:10318800B5FBF0F50CFB131120460091CDE901E5E4
:103198003B49FFF717FF66E707F0080584E7304962
:1031A80096E7B9F1010F45460CBF2E48354896E71A
:1031B80020462F49FFF706FF0136A4E700262046E0
:1031C8003149FFF7FFFE33461AF803202046A2F1E3
:1031D80020035F2B28BF2E222C49FFF7F3FE013670
:1031E800102E0DD0720703D120462149FFF7EAFEC1
:1031F800B1453346E8D820461D49FFF7E3FEEEE720
:10320800059BCA44B3EB090305937FF472AFB8F189
:10321800000F0AD0FB0704D520460B4A0B49FFF7DD
:10322800D1FE39462046FFF7DFFE20460BB0BDE849
:10323800F04F44F012BA00BFDC4308089A1408089B
:103248009E140808FC5A07088C140808CF3B080885
:10325800105B0708C4140808CA1408089114080861
:10326800951408087D760508B9430108CE140808A6
:103278001843080816430808D0360020CC3600202A
:10328800A8140808AB760508D4140808DD3908081E
:1032980042F20F7373B58B4228BF0B46056804468C
:1032A800052168460D4A3FF07FF9064663682846BF
:1032B8000B225B680A4944F0C2F9636832466946E2
:1032C80028465B6844F0BBF963681B2228465B68A4
:1032D800044944F0B4F902B070BD00BFCD28080815
:1032E800D0430808B443080800210123064A904245
:1032F80006D8064A01B901231360054B18607047C8
:10330800012140085B00F2E740420F00CC36002064
:10331800D0360020F8B50D460446064F4618B4428C
:1033280001D12846F8BD14F8011BBB6801485B6849
:103338009847F4E7F8520708014B036000207047EC
:10334800585B07082DE9F34205460E4600244FF066
:103358001409084B084F1B680193019BA34202DC28
:1033680002B0BDE8F0823868314609FB0400A8477E
:103378000134F2E7585B07089001002070B5104B44
:103388000D461C68B4B10F4B196800238B4202DB51
:103398006FF0010070BD224612F8146B864202D00D
:1033A80014460133F2E7E06847F044FE28B10020F4
:1033B8002C60EFE76FF00C00ECE76FF01200E9E724
:1033C80090010020585B070810B5436888B0029345
:1033D80083680C46CDE9033200230A68C068CDE94A
:1033E8000623054901AA059346F0DFFA079808B9AC
:1033F800059B236008B010BD3D7805082DE9F8430A
:103408000646FDF795FD0546EFF31188102383F373
:103418001288BFF36F8F114B1C68D3F804909C423D
:1034280008BF002434B988F31188BFF36F8F204692
:10343800BDE8F883A7683846FDF77AFDA84206D1AB
:103448002A463946304661F04FFB0028EBD04C4500
:1034580001D02468E6E70024E5E700BF94010020D6
:103468002DE9F0410E461546FFF7C8FF044628B37C
:10347800C3681BB35F690FB3062E07D0072E20D091
:103488002A4631463B46BDE8F0411847838A3BB996
:103498002A463146B84750B9A38A0133A38206E0C9
:1034A8004FF6FF72934204D00133A3820020BDE897
:1034B800F0810121114A124844F0A2F86FF015007A
:1034C800F5E745B12A7832B10022828231462A4690
:1034D8005B699847EAE7A38A012B08D12A460721A6
:1034E8002046B8470028E2D1A38A013BD6E70BB1B2
:1034F800013BDAE70221034ADDE700BF301508087F
:10350800545507085215080810B5044608B18068D4
:1035180038B9104A1048012144F072F86FF01500CC
:1035280010BDFFF76BFF08B10C4AF3E7A082EFF379
:103538001181102383F31288BFF36F8F084B5A68E9
:10354800C4E9003214605C6081F31188BFF36F8FA7
:10355800E6E700BF701508085455070889150808DC
:103568009401002080B505460E461746984609F096
:10357800CFFA034600F0E8FC0446DFF8189042460C
:1035880049F8003039463046A84754F8090000F099
:1035980055FC00BF0800000008B50348034A002195
:1035A800121A44F0B9F908BDC0130020304C0020AD
:1035B800074808B5074A0849121A44F0AFF9BDE8A8
:1035C80008400648064A0749121A44F0A7B900BF3E
:1035D80000000020A81300200CA508080000002007
:1035E800000000200CA508082DE9F84F80460C467D
:1035F80000AF00296AD0D1E90012E9468AB0A36871
:103608006D464FF0050A6E463948CDE90723CDE9E6
:10361800050146F810AF002332464FF421513548D2
:10362800FFF7F2FBD4E90312CD466369AD46324891
:10363800C5E90723C5E90501C5F810A000233246EE
:103648004FF421512B48FFF7DFFBCD46E3690121F9
:103658002A4A284843F0DDFF0121294A254843F03A
:10366800CFFF264600254FF00A0ADFF8A4B0E94646
:10367800D6E908C0D6E90A138EB06A46CDF81CC050
:1036880005F1010CCDE908C0A81CCDE90A01E91C27
:10369800CDE905B5CDE90C1342F810AF002345F28A
:1036A800400114480435FFF7AFFB102DCD4606F155
:1036B8001006DCD1236E0121124A0E4843F0A9FFFF
:1036C800A3690121104A0B4843F0A3FFB8F1010F89
:1036D80007D1EFF305830D4A41460648103B43F0F6
:1036E80098FF2146404608F075F8BD46BDE8F88FBA
:1036F800C1150808EC550708F01508081F16080832
:103708002E160808AB160808BA160808E81608089E
:103718006816080830BFFFF7FDBF00BF2DE9F0416C
:1037280005460B4EDFF83080324606EB0807CC1B07
:103738002046084961F08DF9A01942460021083C4D
:1037480061F0ADF9C5F8904007F10800BDE8F081D7
:1037580000000000CC5607080800000010B5244CF3
:103768002449254844F0E7F8A36A99013ED5224840
:10377800224944F0E0F81E20A36ADA0104D51E4865
:103788001F4944F0D8F81F20194CA36ADB0204D55E
:1037980019481C4944F0CFF80220A36A1C0304D539
:1037A8001548194944F0C7F82120114CA36A590358
:1037B80004D51148154944F0BEF82220A36A9A039B
:1037C80004D50D48124944F0B6F82320084CA36AE2
:1037D800DB0304D508480F4944F0ADF82420A36A58
:1037E8006FEA03436FEA1343A36210BD1D20C3E7CA
:1037F80000ED00E0FB160808EC5507081317080849
:1038080026170808401708086A17080888170808BC
:10381800AD170808C717080870B506460D46294CA5
:1038280029492A4844F087F8A36ADB0647D5274880
:10383800274944F080F81120A36A1C0704D52348BF
:10384800244944F078F812201E4CA36A990712D52F
:1038580021491E4844F06FF8636BA26A120609D525
:1038680001211E4A194843F0D4FE1EB1A36A23F071
:103878008003A3621320134CA36ADE0704D5134800
:10388800174944F058F81420A36A9C0604D50F4839
:10389800144944F050F815200A4B9A6AD10658BFCB
:1038A8009A6A9A6A920642BF5A6A22F400525A6287
:1038B8009A6A42F0FF029A6200232B7070BD1020B2
:1038C800BAE700BF00ED00E0F2170808EC5507085A
:1038D800081808083B1808084E1808086618080849
:1038E8007C1808089B18080870B506460D46284C31
:1038F8002849294844F01FF8A36AD9043CD526482A
:10390800264944F018F81720A36A1A0504D5224856
:10391800234944F010F818201D4CA36A9B0512D5C2
:103928001D48204944F007F8A36BA26A100409D582
:1039380001211D4A184843F06CFE1EB1A36A23F406
:103948000043A3621920124CA36A590504D51248F2
:10395800164943F0F0FF1A20A36ADA050ED50E487F
:10396800134943F0E8FF1B20094A936A43F47F4355
:10397800936200232B7070BD1620C5E7A36A9B04D1
:10398800F2D505480B4943F0D6FF1C20ECE700BFF1
:1039980000ED00E0CA180808EC550708E018080808
:1039A8003B180808F11808080A1908081F19080818
:1039B8003A1908089B180808F0B59DB0664B0546EB
:1039C8005868002600AFC0F3080386F31188BFF3D8
:1039D8006F8F02F07F44B4F17F4F07D102F00C04DF
:1039E800082C0ED15D495E4843F0A5FF5D495C484F
:1039F80043F0A1FF00210846FFF7F6FD7437BD46E6
:103A0800F0BD14074CBF0D460126002DEED0002254
:103A1800FA71DA1E092A7ED8DFE802F00575787196
:103A28007D7D7D7D7D7B50494D4843F084FF00239B
:103A3800494CFB71E36A9A0705D54C49484843F05D
:103A48007AFF00242DE0E36A002B01DA4849F5E704
:103A5800E36A5B00F5D54749414843F06CFF636969
:103A6800AA6943F480736361BFF34F8FBFF36F8F0D
:103A780032F8023C626922F480726261BFF34F8FB0
:103A8800BFF36F8F03F47F42B2F55F4F21D1DBB2F2
:103A9800022B1ED12B680121374A314843F0B9FD6A
:103AA8002C68FB79002BA9D16822294607F1080068
:103AB80060F0CFFF7B6A002E4AD0C3F3080222B918
:103AC8006FEA53236FEA43237B62204607F108011C
:103AD80092E7214B9A6AD2B222B10120F91DFFF771
:103AE8009BFE0EE09A6A12F47F4F04D00120F91D64
:103AF800FFF7FAFE05E09B6AB3F5803FA1D3FFF715
:103B08002DFE0446CDE70020F91DE8E70020F91D49
:103B1800EEE71A4992E71A4A6C4610F4F87F8AB021
:103B2800184918BF11466A46103B07934FF40073B3
:103B38001548ADF82030154BCDE9050142F8103F86
:103B480000234FF411510648FFF75EF9A54678E7C0
:103B58006FF30803B8E700BF00ED00E0801908081C
:103B6800EC550708AB190808E7190808FE190808F2
:103B78001F1A08082D1A08084C1A0808681A080895
:103B880067190808521908088C1A08080400000167
:103B9800064B5A6942F010025A615A6942F480622F
:103BA8005A615A6922F008025A61704700ED00E034
:103BB800EFF30880EFF3098101B57246FFF7FCFEC9
:103BC80001BD00BF0A4880F30888102080F31188DF
:103BD80008484FF40061401880F30988EFF3148017
:103BE8000221084380F31488BFF36F8F00F07AF83E
:103BF80050C70020305F0020BFF34F8F0549064BA8
:103C0800CA6802F4E0621343CB60BFF34F8F00BF72
:103C1800FDE700BF00ED00E00400FA051EF0040F08
:103C28000CBFEFF30880EFF30980816911F8021CDB
:103C38000229FFD001B5724643F072FE01BD00BFF4
:103C48000028ACBF00F16040064B4FEA0111C9B231
:103C5800ABBF00F5614000F00F0080F80013195465
:103C6800704700BF14ED00E040B2002807DB0123D5
:103C78004109034A00F01F00834042F82130704791
:103C880000E100E040B200280CDB012206494309AC
:103C980000F01F008240203341F82320BFF34F8FEC
:103CA800BFF36F8F704700BF00E100E0054B42098A
:103CB80053F82220012300F01F0003FA00F01040FF
:103CC800704700BF00E100E0044B054A23F07F0382
:103CD8009360BFF34F8FBFF36F8F704700000108E9
:103CE80000ED00E008B5FFF7EFFF104BD3F8882090
:103CF80022F47002C3F88820D3F8882042F4A00286
:103D0800C3F888204FF04042C3F83422BFF34F8FE6
:103D1800BFF36F8F0023E1EE103AFFF73DFCFFF78A
:103D280047FC00F0F3F807F081FE00BF00ED00E06B
:103D38008189203A41F0020181814FF47D41C0F828
:103D4800DC101360009B08495360019B21F00101BE
:103D58009360029B9161D3604FF08073D36100231D
:103D68000265C0F8943070476D350108104B9B68A8
:103D780083421AD1EFF30580B8B9EFF3118110220D
:103D880082F31288BFF36F8F9A8922F002029A8118
:103D9800EFF3148323F0040383F31488BFF36F8FC6
:103DA80081F31188BFF36F8F70476FF0150070476C
:103DB800D43B00200E461546002300B5E1EE103A2C
:103DC800EFF3148323F0040383F31488BFF36F8F96
:103DD800BFF36F8F0C4BD0F8902098600B4B1A6094
:103DE800D0F8803083F30B882C4686F309880020AE
:103DF800034B98472046002100220023014C20470E
:103E0800657905086D350108D43B0020003700208E
:103E18001022014B1A61704700ED00E0054B9A69CA
:103E28009B689A421FBF044A536843F0805353600B
:103E3800704700BFD43B002000ED00E0084B9B68B2
:103E480083420BD1EFF3058343B1064B5A6842F026
:103E580080525A605A6A22F400425A6247F0A6BB5E
:103E6800D43B002000ED00E025498A6882F8DDE0B7
:103E78004FF030001044EFF3098C80E8F01F1EF07B
:103E8800100F03D102F19C0080EC108A102080F3FF
:103E98001288BFF36F8F1B4F4FF000668A698A60E4
:103EA8003E60D2F89000184C206092F9DDE0D2F81C
:103EB80094000023C2F8943080F311881EF0100F8C
:103EC80003D00023E1EE103A03E002F19C0090ECED
:103ED800108AEFF3148323F0040383F31488BFF3E9
:103EE8006F8F02F1300090E8F01F8CF3098802F11F
:103EF800000004B543F02BFDBDE804407047000006
:103F0800D43B002004ED00E00037002000231021FE
:103F18000348C2180133722B82F80013F9D1704795
:103F280000E100E008B5EFF30583064A103B02EB19
:103F3800C30152F8330049688847BDE80840FFF7D5
:103F48006DBF00BF940C0020014800687047000056
:103F5800003700201FB50121094B0A4A0A4800F022
:103F68000FF90023064A0393084B0121019301A886
:103F7800D31A029300F00EF905B05DF804FB00BFF8
:103F880000000C2000000020AC5B0708C0130020D4
:103F98000A7A0B6810B562F304031C46CB68520911
:103FA80023F01F0343EA4203044A43F00103C2F823
:103FB8009800C2F89C40C2F8A03010BD00ED00E0A7
:103FC80010B50A4BD3F89030C3F30723013B98424E
:103FD80008D901210346064A064843F01AFB6FF048
:103FE800150010BDFFF7D4FFFBE700BF00ED00E0B0
:103FF800A31A0808D45507082DE9F04F8946144636
:1040080006464FF000084F4D85B0C84527DAD6F868
:1040180004A0BAF1000F44D0BAF11F0F17D91AF053
:104028001F0F14D1D6F800B01BF01F0F0FD1584640
:1040380043F0A8FC07460AEB0B00013843F0A2FC4A
:10404800874210D06FF015073F4A3B4601E04346D0
:104058003E4A01213E4843F0DCFA6FF01504204641
:1040680005B0BDE8F08F17F1160FEDD0BC42EBDDBF
:10407800C5F89870D5F89C10C5F89870D5F8A03098
:1040880021F01F0143F01F0BD6E900321A44994270
:1040980002F1FF3A1AD1D34507D13146F8B243F0BD
:1040A8007AFC08F101080C36AFE73146C5F898707C
:1040B800D5F89C30E0B263F30402C5F89C2043F0C5
:1040C8006AFC10F1160FC8D0441CEAE7C5F89870CE
:1040D800D5F8A020013B23F01F0302F01F02134371
:1040E800D3453146E0B2C5F8A030E8D043F053FCE0
:1040F80010F1160FB1D0C5F89870D5F89C209DF82E
:1041080008300BF1FF3B62F304038DF80830D5F853
:10411800A0309DF808205B0863F347128DF808204B
:10412800D6E900321344009323F01F035B44A3EB4A
:104138000A03013023F01F036946C0B20393FFF757
:104148003FFFBEE700ED00E0EF1A0808C91A0808AB
:10415800D45507080522044BC3F89420BFF34F8FAA
:10416800BFF36F8F704700BF00ED00E0BFF35F8FB4
:104178000022024BC3F89420704700BF00ED00E016
:1041880010B5034C2278FFF737FF207010BD00BF31
:10419800314900202DE9F74F294D8A4606464FF050
:1041A8000008AB46274FD0451BDAD6F80490B9F182
:1041B800000F3FD031680846019143F0E3FB0199B5
:1041C800044609EB0100013843F0DCFB84424FF060
:1041D80014021D4B08D002FB08F36FF015024BF8D0
:1041E800032003B0BDE8F08F14F1160F2C60F8D04F
:1041F8001978A142F5DD02FB08B0C7F89840C7F866
:104208009840D7F89C4000F10801007B64F3040053
:104218000871D7F8A0000C79400860F347140C71B6
:10422800D7F89C1021F01F016960D7F8A01021F081
:104238001F01296108F1010814350C36B3E700BFE6
:104248000437002000ED00E031490020F0B5534963
:10425800534DD1F890302C68C3F307239C4287B0A4
:1042680000F299800020FFF781FF4E4BC1F8C03063
:10427800844216D14C4D01A82C70FFF75DF800263A
:1042880007464A4CB74213D100202B784349D1F84E
:104298009020C2F30722934277DBFFF75BFF0020F1
:1042A80046E0696801EB0011FFF772FE0130DFE7B5
:1042B8000199300101EB0613DA682240B2F1807FE0
:1042C80052D00AD8B2F5001F34D0B2F5800F3ED0D4
:1042D800B2F5801F12D00136D4E7B2F1006F43D097
:1042E800B2F1805FF7D15A689B680958013B22F008
:1042F8001F00034423F01F03012032E05A689B6823
:104308000958013B22F01F0003440120844623F092
:104318001F0340EA4C10CDE902218DF8100002A9D4
:1043280028780593FFF74CFE00282ADA6FF015006D
:1043380007B0F0BD5A689B680958013B22F01F007E
:1043480003444FF0020C012023F01F03E1E75A68F1
:104358009B680958013B22F01F000344022023F008
:104368001F034FF0000CD4E75A689B680958013BBB
:1043780022F01F0003444FF0030C012023F01F0319
:10438800C7E72B7801332B70A5E7C1F89830C1F83F
:10439800A00001337BE74FF0FF30C9E700ED00E0F4
:1043A800B85B0708AAFF4400314900200000F0FF6D
:1043B800F0B587B007460E4614460021102268461D
:1043C8001D4660F06CFB02238DF80230054B2A462F
:1043D80021466846CDE9047601933EF077FA07B0A6
:1043E800F0BD00BFD779050808B5024B1B68984790
:1043F800002008BD18370020034B044A1860937842
:1044080043F0020393707047183700209C01002086
:1044180008B5054842F0A5FC002383F31188BFF3D3
:104428006F8F0423184602DF211B080808B50649C8
:10443800064821F00701C1F1005202F5402242F07E
:1044480046FA002008BD00BF43E800201C370020C2
:104458004FF0FF324FF0FF33014807F08BBC00BF2D
:10446800AC010020014807F0F7BC00BFAC010020F8
:1044780038B50546FFF7ECFF2A460821074842F001
:104488006CF9044628B925B1FFF75EFD0C22044BF0
:104498001A50FFF7E7FF204638BD00BF1C37002041
:1044A8000C00000038B504460D46FFF7D1FF214641
:1044B8002B460822074842F0D2F9044628B925B10C
:1044C800FFF742FD0C22044B1A50FFF7CBFF2046A2
:1044D80038BD00BF1C3700200C00000010B5044692
:1044E800FFF7B6FF21460348FDF78CFEBDE81040F4
:1044F800FFF7B8BF1C37002070B541690446867ABB
:104508000A4D59B1437ADB0706D42C2303FB065323
:104518005B6A1B689B689847002363612C202146CF
:1045280000FB0650BDE8704046F061BF90110020C6
:104538002C22024B02FB0030704700BF9011002074
:104548002C21827A054B01FB02339A6A1B7F801A61
:104558001B3323F00303B0FBF3F0704790110020E6
:1045680038B52C24827A064B04FB02335B6AD3E904
:1045780001240C601568FFF7E3FF04FB005038BD09
:10458800901100202DE9F04385B005466846904615
:104598001C46039147F061F9DDE90067EFF31189E3
:1045A800102383F31288BFF36F8F6B8B002B41D0DE
:1045B8002A8B9A4225D900220023284607F09CFC22
:1045C8000446F0B189F31188BFF36F8F039B002B6A
:1045D80041D032463B46684647F064F92C21A27A1E
:1045E800254B204601FB02335B6A03A91B681D6843
:1045F800DDE90023A847606170BB2046FFF77CFF18
:1046080024E0698B4B1E6B8389F31188BFF36F8F8E
:104618002B7F2A8BAC6A1B3323F00303521A02FB4D
:104628000344154B154AEB1A9B105343A3722B7F77
:10463800E372CBE789F31188BFF36F8F23464246B5
:10464800284607F059FC04460028BFD1002420461C
:1046580005B0BDE8F0836361012300252381039B36
:1046680029466382E27A656004F1180060F017FA5F
:1046780063692582E360EAE790110020A38B2EBAD4
:10468800F8B500242C260F4D00B9F8BD476800F195
:104698000802D2E8EF3F591EC2E8EC1FBCF1000F38
:1046A800F7D1DBB2012BF0D1837AC46006FB035348
:1046B80044601B6A13B198473846E5E7FFF71CFFCB
:1046C800FAE700BF90110020F7B506460D461446DC
:1046D800124F384646F0AEFCE0B1BB68314638466A
:1046E8001B68AAB29847002802DB002003B0F0BD7F
:1046F800002CFBD1AC42F8D22F1B042F28BF042773
:1047080005F0F0FF3A46019001A9301960F0A1F9CF
:104718003C44EFE76FF01200E8E700BFA452070837
:1047280038B5044608F0D0F9204643F0CCF9A06922
:10473800C8B194F86C30DB070DD50221154A16482C
:1047480043F0BFF96FF07705201D43F0C3F908F077
:10475800CFF9284638BD46F06DFC38B901210F4A1B
:104768000D4843F0AEF96FF01205EDE7204600F072
:10477800ADFF05460028E7D10146242204F12800B0
:1047880060F08DF994F86C3043F0010384F86C30D4
:10479800DAE700BF391B080884560708631B0808B6
:1047A80070B5044608F090F9204643F08CF994F867
:1047B8006C30DA070DD40221254A264843F081F9E6
:1047C8004FF0FF35201D43F085F908F091F9284690
:1047D80070BDC3F340019B0707D502211E4A1D483F
:1047E80043F06FF96FF07705ECE7A06944F0EAFD54
:1047F8000646A06944F076FE054628B10121174A0D
:10480800144843F05EF9DDE7A36F4BB1314620460B
:1048180043F03AFB0546A0B1A06944F08BFED1E70E
:10482800A06944F007FEA0670028EFD101210C4AD7
:10483800084843F046F9A06944F07CFE6FF00B0588
:10484800C0E794F86C3043F0020384F86C30B9E7A1
:10485800861B080884560708AC1B0808D21B0808E2
:10486800EE1B080838B590F86C3004469B0708D44E
:104878000221144A144843F024F96FF077052846BA
:1048880038BD43F020F90021204601F0B9F820B1E5
:1048980001210E4A0C4843F014F9A06944F04AFE7D
:1048A800054620B101210A4A074843F00AF994F85D
:1048B8006C30201D23F0020384F86C3043F00AF9B1
:1048C800DDE700BF0A1C080884560708311C0808E1
:1048D8004F1C08082DE9F04385B006460C46904663
:1048E80043F0FAF80546B8F1000F07D0304643F018
:1048F800F8F8012810D1B5FA85F56D090134294673
:104908003046E2B243F0D9FA814650B90121234634
:10491800324A334842F07DFE0024204605B0BDE807
:10492800F0834768B8F1000F09D03868796801AB9F
:1049380003C33A7A01AF1A7007238DF80530F18D59
:104948007B883046994228BF194643F008FC044644
:104958000028E1D0038A428A4169D21AC36800F16B
:104968000C085B1AD21A3B7839469A4228BF1A4675
:10497800404643F07BF8D9F80C90B9F1000F08D104
:10498800218AF38D9942C8D94046C91A43F089F85B
:10499800C3E7D9F8040083681B6B13B9D9F80090F2
:1049A800EBE7294698470028F8D0071F57F8041F57
:1049B8000029F3D008780028F0D0628A238AA2EB75
:1049C800030C6269E3689B1AACEB0302904294BF44
:1049D800024692B2404643F049F8E7E77F1C0808D0
:1049E8006456070838B50446806F43F020F805463A
:1049F80043F001F82046294601F04AFA044638B146
:104A080004480121044A42F0FBFD2846FFF738FE1E
:104A1800204638BD64560708A51C080838B580210B
:104A28000446806944F029FD054678B101462046D0
:104A380001F02EFA044638B106480121064A42F030
:104A4800DFFD2846FFF71CFE204638BD6FF00B043B
:104A5800FAE700BF64560708C41C080800232DE9BC
:104A6800F04F93B005930B7E044633F080060F4653
:104A780015460AD00121AD4AAD4842F0C1FD6FF09C
:104A88000406304613B0BDE8F08F82B10846FFF740
:104A9800F7FD7B7EDA0704D49D07F2D53B7E002B19
:104AA800EFD1204613B0BDE8F04FFFF79BBF4A7E19
:104AB80000F12809900705D5802B09D13846FFF762
:104AC800DFFDDEE7910700F03184002B40F02E84F3
:104AD800D3071ED53B8A082B12D1FA6839461368CA
:104AE8000020A3625368C9F8043042F0A7FF05907C
:104AF80080B18F4801218F4A42F082FD059805E078
:104B08008B4801218C4A42F07BFD3846FFF7B8FDFF
:104B18001EE00597FFF718FA002394F82850874AF3
:104B280015F0600F8350C5F341131CD0032B40F0E0
:104B380064836FF08505FFF707FA804B1B58002B3D
:104B480000F09A83002D00F0698305980028DDD1D4
:104B5800484643F0F9F80346A069002B00F0218489
:104B6800802100F027BC484643F0EEF894F829303D
:104B7800002840F02C81013B0A2BDAD801A252F818
:104B880023F000BFCB4C01083B4B0108514D0108F5
:104B98003B4B0108B94B01083B4B01083B4B010853
:104BA8003B4B01081F4C01083B4B0108934C010883
:104BB800A069618D03697F2993F88030B9D8A28DE7
:104BC800002AB6D1E28D002AB3D1EE06B1D194F80D
:104BD8003020022A02D14FF0FF35ACE71D070BD574
:104BE800C9B243F0E7F8054648B1638D0121544A3C
:104BF8004F4842F00EFD9EE7012384F8393094F8BF
:104C08003030012B05D1638D1BB984F83030002575
:104C180091E70123F9E7204642F05EFF628D0146E5
:104C2800FF2A86D8E38D002B83D194F82830D80644
:104C38007FF47FAF94F83030002BCCD092B9618DDF
:104C480094F838308B42E2D02046C9B200F0D8FE42
:104C5800638D054668B1012100903A4A344842F014
:104C6800E2FC68E72046D2B243F04DF90028E6D1CD
:104C7800B1E7002B14BF02220122052184F830205D
:104C880020461A4643F0B4FAC1E705F01F05012D86
:104C98007FF44FAFE38D002B7FF44BAF628DFF2A7B
:104CA8003FF647AFA18DFF293FF643AF94F8303068
:104CB800022B90D12046D2B2C9B243F0D4F90546AE
:104CC80039E7E38DA68D002B7FF433AF94F83030AD
:104CD800002B80D0012B02D1002E7FF47CAF15F081
:104CE8001F0515D0022D92D1B4F82A80B8F1000F13
:104CF8008DD1F6B23146204601F032F9421C054604
:104D08003FF419AF42463146204643F023F812E7F4
:104D1800002E7FF460AF638D012B7FF478AF94F899
:104D28006C3066F3C30384F86C3070E7E71C08083E
:104D3800645607081F1D0808081D08080C00000015
:104D4800411D0808631D0808A38DE28DDEB2002A04
:104D58007FF4EFAE628D022A11D105F01F053543AD
:104D68004FEA13217FF4E5AE0122A06943F002F86F
:104D780000287FF4DEAE012384F8393047E794F841
:104D8800301000293FF427AF012902D1002B7FF40E
:104D980022AF15F01F050FD0022D7FF438AF002A7F
:104DA8007FF435AF3146204601F0B8F8431C05467C
:104DB8003FF4C1AE0122A6E7002B7FF40CAF012A15
:104DC8007FF425AF94F86C3043F00803ABE70A2B67
:104DD80063D8DFE813F00B00620062006200620033
:104DE80062003A006200DD016200F201E38D022BED
:104DF80053D194F83030002B4FD0012BA18D01D125
:104E080000294AD115F01F050ED0022D17D0002613
:104E18000221204643F0A3F9054618B131460C306B
:104E280042F035FE0595F2E6002936D194F86C304B
:104E38009E0806F00206C3F300131E43E8E7204667
:104E4800C9B243F0B0F90646E2E7618DED064FEAD4
:104E58001123C9B207D0002320460AA90A9342F0B9
:104E6800C2FF0A9DDEE7013B0E2B16D8DFE813F0E0
:104E78000F003000380015001500D200360015006C
:104E88001500150015001500150015000F01204626
:104E980042F022FE18B1012818D00025C2E7266F7B
:104EA800002EFAD0B4F82E8033782046984528BFD3
:104EB8009846414643F053F905460028B2D0424689
:104EC800314605F10C0042F0D1FDABE7666FE7E72C
:104ED80000222046FFF7FEFC0546A3E70122F8E77B
:104EE8000A462046032142F083FE80460028D4D09B
:104EF80042F025FFE58D98F81530B8B998F8146098
:104F08008DF82930AE428DF8286028BF2E46D8F893
:104F1800103031461B882046ADF82A3043F01FF97F
:104F280005460028B9D032460AA9CAE74FF0000A58
:104F3800B44A8DF81130D8F808308DF810A01A400E
:104F4800B14B9A4255D1102106A804F09DF8061ECF
:104F580036DB0AAB102E984628BF1026AB4806AAA7
:104F6800564503F1020334D8B6000236F6B28DF87E
:104F78001060AE4228BF2E462046314643F0EFF877
:104F88000546002889D0022EB34628BF4FF0020BF1
:104F98005A46A6EB0B06C34600F10C0A504604A974
:104FA80042F064FD730808EB56025A4528D1F00711
:104FB8007FF538AF504618F8031042F060FD31E72E
:104FC80058367FF46AAF0121914A924842F018FBA3
:104FD80063E712F8011B0AF1010A4FEA111C01F0FC
:104FE8000F0110F80CC0415C03F802CC03F8011C57
:104FF800B6E798F81460D8F810808DF81060B8E714
:1050080050461BF8011BCDE9022342F040FDDDE9C3
:105018000223CAE7204642F05FFDD4E91C5300286A
:1050280008BF1D460A2300268DF82830062320468F
:10503800CDF82A60CDF82E608DF8293042F051FD68
:1050480001287FF42AAF002D3FF4ECAE6B88204690
:10505800ADF82A302B798DF82C306B798DF82D30FE
:10506800AB798DF82E30EB798DF82F306B7C8DF87D
:105078003030E68D9DF828309E4228BF1E463146C6
:1050880043F06DF8054600287FF44DAFCAE6204688
:1050980042F022FD20B101287FF4FFAE636F00E0EB
:1050A800236F002B3FF4F9AE5B88B3F5007F7FF6E2
:1050B800F4AE594B04F14C060A9300238DF82C30BA
:1050C800E36C9E4208BF0023BDF82A2093B1597DA6
:1050D8000F2908D1197D0A44ADF82A209DF82C2003
:1050E80001328DF82C20226D9A4201D01B68EBE723
:1050F800BDF82A20B4F82E802046904528BF904657
:10510800414643F02CF8054600283FF4C6AE9DF80A
:10511800282000F10C0A424528BF424650460AA9F9
:1051280042F0A4FC9DF82830434594BFA8EB03083F
:10513800A8EB0808B8F1000F3FF474AED4F84CB0EF
:10514800B3453FF46FAEBBF1000F3FF46BAE9BF875
:1051580015300F2B15D19BF814205046424528BF17
:105168004246DBF8101042F081FC9BF814304345AE
:1051780094BFA8EB0308A8EB0808B8F1000F3FF4A8
:1051880051AE236D5B453FF44DAEDBF800B0DAE776
:1051980094F83030002B3FF480AEE18D01297FF484
:1051A8007CAE94F83860204642F0D9FF05460028C6
:1051B8003FF438AE31460C30FFE605F01F05012DEF
:1051C8007FF46BAE204642F08CFE00283FF465AEBB
:1051D800A38D4268FF2B3FF660AE12799A42FFF426
:1051E8005CAEDAB20F2A3FF658AEE18D01297FF4A2
:1051F80054AE234493F83A60D5E7204605A942F017
:10520800F2FD5CE500FF020000030200E14308082C
:10521800861D080864560708050F050046F01BFBA5
:105228000A220023FBF718FE644BD3E8AF1F41F2B4
:105238008732461A9642624A39D9D3E8EF6F8E42CE
:1052480004D1C3E8EC0FBCF1000FF6D12FD1D2E89E
:10525800EF3FC2E8E15F0029F9D123B10221594AA1
:10526800594842F0D6F90221584A574842F0C8F93D
:10527800FEF76AFE564B1D58002D7FF466AC7B7E08
:10528800E28DD9071BD5484642F05EFDB8B9BAB1E0
:105298002946A06944F0DDF80146059000283FF44E
:1052A80057AC204613B0BDE8F04F00F0F1BDD2E88E
:1052B800EF3F0133C2E8E13F0029D9D0F7E73AB917
:1052C8002046FFF7ABFB00287FF442ACFFF7E9BBB1
:1052D800484642F039FD059D18B92846FFF7D0F930
:1052E800EEE7002D3FF434AC2946204600F0D0FD0F
:1052F80008B128460AE4A069036993F8801011F000
:1053080004017FF4CEAB44F0B8F8054600283FF41A
:105318001FAC0146204600F0BBFD00283FF4C1AB9E
:1053280001212C4A284842F06BF9E2E752077FF541
:105338000FAC002B3FF4C2AB3846FFF7A1F994F845
:105348003930002B3FF49DAB94F82930052B0CD154
:10535800618DA069C9B242F02DFD054628B1638D63
:1053680001211D4A184842F054F994F82930032BBA
:1053780011D1638D022B0ED1A18D00220E0A314668
:10538800A06942F0F7FC054628B101213346134ACB
:105398000D4842F03EF900232E4684F83930FFF7D5
:1053A80070BBE38D002B3FF4DBAB0599003918BFC8
:1053B8000121C90143F064FFFFF773BB2C370020BC
:1053C80028370020A81D080864560708BC1D0808CF
:1053D8000C000000E51D0808411D0808091E080802
:1053E8000B7810B4062B14D10369D3F89C20EFF383
:1053F8001184102383F31288BFF36F8F00204B684A
:105408001860506A60B9C2E9083384F31188BFF3A1
:105418006F8F0022002304485DF8044B45F009BF54
:1054280003605362F1E700BF0C11002030B589B06A
:10543800002200230024CDE906236FF007034FF470
:105448008062CDE90334CDE90144154B1549009438
:10545800154807F03DF81549134846F0A2F8144BD3
:1054680014498B4207D30020134B14498B420CD3A9
:10547800002009B030BD03F11402D2E8EF0FC2E8F2
:10548800E54F002DF9D11833EBE703F11402D2E808
:10549800EF4FC2E8E50F002DF9D11833E6E700BF5A
:1054A8002155010830530020A02800206E39080833
:1054B800E81200204813002048130020A8130020F9
:1054C80038B50D4642F00DFD30B90121BDE8384030
:1054D8000F4A104842F094B8C46804B938BD2B7814
:1054E800032B05D0052B0ED0022B08D02468F4E737
:1054F800606883685B69002BF8D09847F6E76068B6
:1055080083689B69F7E760688368DB69F3E700BF36
:10551800301E0808745607082DE9FF4110274FF080
:10552800FF334FF0FF32644801A906F0BFFB039B2D
:105538001B69D3F89C40236A93B1EFF3118287F378
:105548001288BFF36F8F216A29B1606A0B688142A4
:10555800236208BF636282F31188BFF36F8FC9B9F2
:105568009DF80430062BDAD0072BD8D801A252F8C0
:1055780023F000BFC1550108B5550108E9550108D8
:10558800C75501081D5601080B5601082755010883
:10559800B15601080B7E20465D06D1F81E2002D1C7
:1055A800FFF75CFAC7E742F0ECFCC4E700220121F0
:1055B800204642F01DFEB2E700221146F8E794F8B3
:1055C8006C3043F0040384F86C3094F83030022BCC
:1055D80003D1204601A9FFF773FF00220321E7E763
:1055E80094F86C3023F0040384F86C3094F830306D
:1055F800022B03D1204601A9FFF762FF00220221F6
:10560800D6E794F83030022B89D1204601A9FFF75C
:1056180057FF84E794F86C30A66923F0040384F8F4
:105628006C30D6F808803369A033D3E8AF3F9A07C7
:105638001ED53046D8F83C309847D8F82430002199
:10564800304698470546D8F840303046984795B1D7
:105658001A4A01211A4841F0D3FF002204212046AA
:1056680042F0C6FD002D3FF45AAF2A4607219FE7B6
:105678004FF0FF35ECE72946204600F0C1F9054612
:1056880008B1104AE5E7A06943F016FF831E5842A7
:10569800584194F86C3084F8305023F0680343EA9A
:1056A800401384F86C30D8E70121074A044841F0D8
:1056B800A7FF0621029A7BE70C1100205F1E08084D
:1056C800745607088D1E0808B91E080838B5024622
:1056D80005460C49806943F04DFF044630B101216D
:1056E800094A0A4841F08CFF204638BD85F8380041
:1056F800284600F043F904460028F5D0A86943F08D
:1057080068FFF1E7E9530108C91E0808745607083D
:10571800F8B501231D460C68002C35D063F07F02D4
:10572800D6B202F07F02103224FA02F7FF0716D52C
:10573800046824FA02F7FF0708D433461348012106
:10574800134A41F066FF6FF01500F8BD05FA02F242
:1057580024EA020404600C6824EA02040C60DC40B9
:10576800E6070ED5026822FA03F4E40700D4E5E759
:1057780005FA03F422EA040202600A6822EA040233
:105788000A600133102BC6D10020DEE7A4560708B3
:10579800F01E08082DE9F04F0026536891B0D46830
:1057A8000A900891069202930E96039674B9039B89
:1057B800029A09339BB293701B0AD370069B167129
:1057C800DC68002C40F0C780A346AEE04FF0000A2A
:1057D8006068CDF83CA083681B6B002B00F0AC80A0
:1057E80008999847002800F0A7803546C4E903AA1D
:1057F800A0F1040959F8043F0BB11A789AB9B542D7
:1058080040F29780E3680F9A1343E3606068836807
:105818009B6A002B00F0928098478346002800F08E
:105828009080534A7DE05A780B2A08BF9D70D9F8BA
:1058380000305A78042A10D1E2680F990A43E260CE
:10584800DA78002A5CD101229D702369AA401343AB
:1058580001352361EDB2CDF83CA0D9F800707B7812
:10586800052BC7D16FF0120B4FF001080A9B9B69FB
:10587800099379793A790E9B42EA0122ADF83620EC
:1058880097F902205FFA88F1002AACBF424641F03E
:1058980080010493B7BF4BB24FFA88F321F080021E
:1058A8000793A8BF0793049BB8BF103223FA02F0EE
:1058B800C0072CD40F9B23FA02F20593D30726D4F2
:1058C800BB79FA78099800930DF136030B9143F0F0
:1058D8004DFC0B998346D0B9079BB970002B4FF04C
:1058E8000103BCBF21F0800110318B400498059959
:1058F800BDF8362019431843CDE90E01BA8079E77F
:105908006A1E9A700FA90EA8FFF702FFA3E708F115
:105918000108B8F1100FACD1BBF1000F3FF46AAF2A
:10592800144A0121144841F06BFE584611B0BDE8F5
:10593800F08F6FF0150BF3E7354667E76FF0850BCF
:105948006FE76068089942F0ECFA039B2E4603441F
:10595800246803932AE7E36804F10C01A3600EA806
:10596800FFF7D6FE08B924682BE76FF0150BDCE7C4
:10597800311F08080D1F0808A456070870B5836969
:1059880005461B69026F93F88030C3F34113022B5D
:105998000CD0032B0CD0012B0CBF10230823D37180
:1059A800EE6D3EB96E6DBEB9344611E02023F6E7C0
:1059B8004023F4E7324601212846FFF7EBFE044670
:1059C80040B173685B790B4A01210B4841F021FE15
:1059D800204670BD3668E4E7324600212846FFF7C6
:1059E800D9FE044618B173685B79044AECE7366857
:1059F800D9E700BF551F0808A4560708781F0808EC
:105A08002DE9F04105460E4642F066F895F8383023
:105A1800804633B3284642F064FA0746F0B101469F
:105A2800284642F0CEFA10220446002105F13A0039
:105A38005FF035F8002385F83830FF683FB984B146
:105A480019491A4842F02CFA2046BDE8F0817868D6
:105A580083685B6A03B198473F68EFE76FF03C04DF
:105A6800EEE71EB985F838600024EDE73246414676
:105A7800284642F022FA074690B10246284642F0EC
:105A8800CAFA04460028DFD185F83860FC68002C83
:105A9800EAD0606883681B6A03B198472468F6E710
:105AA8006FF03C04D0E700BF311C08085C560708BB
:105AB8002DE9F04105460F461446D2F8048042F01D
:105AC800F3F995F86C30D9070BD54749474842F0A8
:105AD800E7F96FF00F07281D42F0EDF93846BDE8E9
:105AE800F081012F0AD1284641F0FBFF30B9404927
:105AF8003E4842F0D5F96FF08507ECE798F8073093
:105B08009A0607D5AB691B6993F880309B0701D4C7
:105B18003849EDE71FB1012F06D03749E8E7EB6DAB
:105B28002BBB05F1540603E06B6DABB905F15C06C0
:105B3800002233680BBB002FD5E91C2308BF13468E
:105B48005B7C626803F10103DBB25371D5E91C1277
:105B580008BF0A46537422E09C4206D127492348CD
:105B680042F09EF96FF01507B5E71B68DDE79C4228
:105B780001D12349F3E71B68D2E79C4221D123686E
:105B8800CAB972683360944200D1736000232360FD
:105B980063685B7902211B4A144841F03AFDA16809
:105BA800B9B1284642F03EF8074668B116490F4891
:105BB80042F076F98FE7136073689C4208BF726001
:105BC800E4E71A461B68B5E7A06842F0B8F888F819
:105BD80006000023236073681BB9C6E90044002748
:105BE80079E71C607460FAE7C91F08085C56070863
:105BF800EB1F0808A51F080809200808292008081D
:105C0800462008086320080880200808F8B50546DB
:105C180000AF29B301290BD1184C194E2BE063684A
:105C280028461968FBF772F9B8B11834B442F6D3AC
:105C38006C4688B06A46134BCDE905354FF40073BE
:105C4800ADF81C30104B42F8103F00234FF4E251DE
:105C58000E48FDF7D9F8A54600242046BD46F8BDF4
:105C68000B4C0C4EE2E7636828461968FBF74EF9BF
:105C78000028F2D01834B442F5D3D9E748130020ED
:105C8800A8130020B7200808030000016C56070875
:105C9800E81200204813002070B5012501F07F03A9
:105CA80011F0800F18BF10339D4090F83030044633
:105CB800022B06D001210C4A0C4841F0A1FC00201F
:105CC80070BD90F8386041F007FF32460146204623
:105CD80042F0F3F80028F2D0C0680028EFD08368BB
:105CE8001D42EDD10068F8E7D52008086C56070872
:105CF8002DE9F84305460846114616469846FFF72B
:105D080085FF0446002843D0284642F003F995F859
:105D18006C30DA0702D5204A012109E0D4F8049052
:105D280004F11407D7E8AF3FDB070CD502211B4A63
:105D38001B4841F065FC6FF00F04281D06F08CF835
:105D48002046BDE8F883D9F804301BB1AB4201D036
:105D5800144AE1E742463146284642F0AEF8A0B17F
:105D68000023236003696BB9C0E90344D7E8EF3F18
:105D780043F00103C7E8E23F002AF7D10024C9F83D
:105D88000450DAE71C600461F0E76FF03C04D4E7E4
:105D98006FF01204D4E700BFC91F0808FA200808EA
:105DA8006C5607081C2108082DE9F04F83B000AF96
:105DB8007B6097F830304C680E463B6081469046D1
:105DC80041F08AFEA36801461B6B33B96FF01504D6
:105DD80020460C37BD46BDE8F08F2046984700287E
:105DE800F4D00024051F06F10C0A55F8041F09B168
:105DF8000B782BB9002C14BF00246FF03C04E7E7A4
:105E08004B78042B0ED1002C3CD18B787A689342C6
:105E1800EBD1CB783A689342E7D10B79002BD7D0F6
:105E28000124E2E7052BE0D1002CDED0B8F1010F08
:105E380091F802B009D0B8F1020FF1D15246594693
:105E4800D9F8180042F075F904E05246D9F818005C
:105E580042F053F904460028E2D06D468AB06A46FB
:105E6800F368CDE907B3062307490990CDE905187A
:105E780042F8103F00234FF441510448FCF7C4FF97
:105E8800AD46A5E70024A3E75C2108089C5607084F
:105E98002DE9F0410B7E0C465906054637D16BB308
:105EA80041F05AFE40B11B4801211B4A41F0A8FBB2
:105EB8004FF0FF30BDE8F0812846D5F87080268A7B
:105EC800EF8D41F009FEF8B1421E534253419B0148
:105ED800228A9AB1BE42324628BF3A46E98D91429B
:105EE8000CD9B2FBF3F103FB11223AB994F918303B
:105EF800002BBEBF637E43F0080363762146A86982
:105F0800BDE8F04143F018BA98F80730E0E76FF0C1
:105F18001500CFE78C5607089821080870B5064683
:105F280080690C4643F0ACF9054638B10221234696
:105F3800094A0A4841F06DFB284670BD012214F059
:105F4800800F18BF24F08004736B18BF1034A24070
:105F58001A437263F0E700BFAC2108088C560708A3
:105F680070B5054680690E4643F0B5F9044638B168
:105F780002213346054A064841F04BFB204670BDD6
:105F8800314605F1340042F0AAF8F7E7C3210808C2
:105F98008C56070870B50646EFF31181102383F37A
:105FA8001288BFF36F8F1B4D2A6881F31188BFF3E6
:105FB8006F8F526892F86C20D20705D4BDE8704004
:105FC8000A22002306F036BAEFF3118283F312880F
:105FD800BFF36F8F2C682CB1696823688C422B60E3
:105FE80008BF6B6082F31188BFF36F8F44B160689C
:105FF80004F10801C36998472146074845F0B6F8F7
:106008002B6833B13046BDE870400022002306F00B
:10601800D9B970BD303700209810002030B585B050
:10602800CDE90012054600220023144803A905F013
:10603800A3FD0246E8B9DDE90001039B5D60083372
:1060480083E80300EFF31180102383F31288BFF372
:106058006F8F039B1A600A4A516861B9C2E900331D
:1060680080F31188BFF36F8F00220023054806F0E4
:10607800A9F905B030BD0B605360F1E79810002016
:10608800303700200000002073B5102504698DF812
:106098000710EFF3118685F31288BFF36F8F012283
:1060A800206C0DF1070141F024F986F31188BFF344
:1060B8006F8F012812D045F06EFAC8B10122104B3B
:1060C800D3E8EF1F002903D1C3E8E02F0028F7D158
:1060D80004D102210B4A0C4841F092FA237F2BB1DC
:1060E8000A22002304F1480006F06CF902B070BDE2
:1060F800A37E002BE2D000210A2045F054FBC8E71C
:1061080038370020ED2108085456070838B5002410
:1061180005690E492B6C05F14800C3E90144DC60B0
:10612800AB6BC3E90144DC6045F029FA05F178005E
:10613800074945F0F8F9074905F1280045F0F3F952
:10614800284642F07AF8204638BD00BF816201082F
:10615800C9630108956401082DE9F34103690646FE
:106168000D46D0F804801C690F7E002A32D00B8AB5
:1061780071323E480BBF022101213D4A3D4A00933E
:106188003B4641F050FA30462F7E42F0CAF887422B
:1061980004D1042104F1880042F077F930462F7EBB
:1061A80042F0CDF8874204D1052104F1880042F07D
:1061B8006CF930462F7E42F0A6F8874203D104F1ED
:1061C8008C0005F031FF2946404602B0BDE8F04199
:1061D80041F0E6BF42F0A5F8B84214D12A8AE9682E
:1061E800A06B41F086F828B1236A1BB104F128009E
:1061F80006F078F804F18800042142F046F904F129
:10620800780006F06FF830462F7E42F098F8874203
:1062180015D1236A1BB104F1280006F063F80521A3
:1062280004F1880042F031F9237F9BB900234FF431
:106238007A7204F1480006F0C5F801232377304646
:106248002F7E42F060F88742BDD104F18C0005F042
:1062580089FEB8E7236C5A89DB889A42EFD000227E
:10626800002304F1480006F0ADF8E8E754560708A3
:106278000C220808302208082DE9F04750F8483C5D
:1062880000F140075B68054600213846D3F80090C6
:1062980042F033F8002864D00121384642F02DF846
:1062A800804600285DD155F8083C5A89DB889A4217
:1062B80003D115F82D3C002B53D0D7E8EF4F44F00D
:1062C8002003C7E8E23F002AF7D114F0200448D1A0
:1062D800484642F034F8002282460023224841F022
:1062E8008FFB064650B93846052142F0CEF82846BD
:1062F800BDE8F0470A22002306F064B880F818A029
:1063080015F82C3C33B1428AC16855F8080C41F0A5
:1063180010F80446214606F10C0041F0A1FB5CB1DF
:10632800D9F8040042F08FF8B4FBF0F303FB1044F3
:10633800B4FA84F84FEA58183146484605F82D8CC7
:1063480041F016FF68B10121084A094841F058F99F
:106358003046FEF795F93846BDE8F047052142F08A
:1063680094B8BDE8F08700BF9011002051220808BA
:106378005456070838B503461B6940685D68AC6821
:10638800A37A84F8223094F82D3084F82330A37649
:10639800696849B1237C3BB941F044FC30B1012123
:1063A800054A064841F02CF9002038BD686841F0DC
:1063B800C6FC2074F8E700BF632208085456070893
:1063C80070B550F8782C00F110045268034600218B
:1063D8002046156841F091FF00284DD00121204644
:1063E80041F08BFF002847D153F8402C6868938808
:1063F800918916695B1A9BB2F61A42F024F8B042EA
:106408003AD8D4E8EF3F43F01002C4E8E12F00295E
:10641800F7D1DB0606D5BDE870400221174A1848B7
:1064280041F0EEB8284641F07CFF002206460023E2
:10643800144841F0E5FA0446F0B10676686842F07F
:1064480002F8638A984203D2686841F0FCFF83B27D
:1064580021462846638241F08BFE68B1284641F008
:1064680060FF034606480121074A41F0D2F820465A
:10647800BDE87040FEF704B970BD00BF8D22080862
:106488005456070890110020AD22080838B550F876
:10649800083C044633B9BDE8384001212A4A2B4854
:1064A80041F0AEB850F8283C00F160055B68022165
:1064B8001A68002383828383284641F01EFFB8B1FF
:1064C80054E9023110699847637D1BB104F150000B
:1064D80005F008FF0521284641F00FFF98B9637FB2
:1064E8006BB10022002304F1200005F06BFF0AE0E5
:1064F8000321284641F001FF0028E1D1E4E714F820
:106508000D3C002BEDD10221284641F0F6FE38B1B2
:106518002369DA885B899A4202D0204605F0E2FEB8
:106528000321284641F0E9FE60B1A2699388918968
:1065380012695B1A9BB29A4204D02046BDE83840E3
:1065480005F0D0BE38BD00BFD2220808545607084F
:10655800D3B5002600270446CDE90067054841F079
:1065680053FA28B1230658BF0023047658BF038284
:1065780002B0D0BD141200202DE9F04383B00023EF
:106588004FF0010805691C4C1C4E02AF28602B77A0
:1065980085F8203005F12409B442234601D30020B0
:1065A80019E095F820201034CAB16C4688B01B68F1
:1065B80002AA1349C2E905134FF400739383114BE0
:1065C80042F8103F104800234FF4E251FCF71CFC3E
:1065D8006FF00B00A5460437BD46BDE8F08385F88B
:1065E800208054F8043C4846009354F8101C54E9A1
:1065F800032342F016FACFE7B4B80808C4B808086D
:106608003423080803000001AC5607081FB5CDE97C
:10661800010103924FF0FF324FF0FF3301A9034805
:1066280044F007FE002005B05DF804FBDC100020F4
:106638001FB500230190CDE902334FF0FF324FF030
:10664800FF3301A9024844F0F4FD05B05DF804FBEE
:10665800DC1000202DE9F041044617460E4600687C
:1066680042F047F831463A468046FFF771FFD4F8C2
:106678007B300546DB1B0146C4F87B30206841F0BF
:1066880077FD88B10B4A434601210B4840F0C1FF12
:106698003146204642F0F8F82846FDF7F1FF20463B
:1066A800BDE8F04142F0BCB8A37F0133A377BDE851
:1066B800F08100BFAD220808AC5607082DE9F84F55
:1066C8000446006842F02AF84FF030090746E37F95
:1066D800012B1ED82368D3F810B0D3F804A09BF878
:1066E800616009FB06B62436304642F0C0F93146EF
:1066F80002468046504642F027F89BF81F30054670
:1067080033B1A8EB00023146504642F01DF8054669
:106718000DB9BDE8F88F204641F0D3FF2A4601465F
:1067280006463846FFF714FF05460146206841F043
:106738001FFD80B101213B46094A0A4840F069FF24
:106748002846FDF79DFF3146204642F09DF8BDE8FA
:10675800F84F42F065B8E37F0133E377B7E700BF4E
:10676800AD220808AC5607082DE9F04FB94F89B09B
:106778004FF0FF324FF0FF33B74805A905F096FAFE
:10678800059E069D3469002D40F09080257704F120
:10679800240694F820309D42C0F2828004F1180348
:1067A800D3E8EF2F22F00202C3E8E12F0029F7D146
:1067B800D3E8EF1F21F00401C3E8E21F002AF7D154
:1067C80004F11803D3E8AF3FDB07D1D5237F022BB1
:1067D80000F08E81032B00F0878153BBDDF814A0F5
:1067E800DAF81050EB7F23BB504641F097FF814603
:1067F800284641F066FF4FF40072014606464846B7
:10680800FFF7A6FE80460146504641F0B1FC00283D
:1068180000F0668101214B46904A914840F0F9FE0C
:106828004046FDF72DFF3146284642F02DF841F04D
:10683800F7FFA37F002B9BD1237F012B40F07D81A5
:10684800302304F1630694F86150304694F86210DE
:1068580003FB054500F060FA2435024631462369FA
:10686800284600F077FA0646C4F88400284642F025
:10687800F4F88146284642F0F5F88046284642F06A
:10688800F6F8E26D3044002A40F03B81002840F0E1
:106898003381284642F012F9003818BF01202CE154
:1068A800304642F0D1F80135303672E7DDF81C8009
:1068B800D6F804A095F81890B8F1000F21D02B8ACB
:1068C80018F1710F6648009308BF02214B4616BFA6
:1068D8000121644A644A40F0A6FE304695F81880C3
:1068E80041F01CFF804540F0EF80E37F013BE377F8
:1068F8002046696941F0C8FF2946504641F050FCDE
:106908005EE7304641F00AFF484540F09580237F16
:10691800D5F80C80B5F810B0002B49D1BBF11F0F8A
:1069280042D1D8F80030BB423ED1414604F154036D
:1069380008F11C0251F8040B914243F8040BF9D1F9
:106948000A881A808A7842219A70552384F873300D
:10695800532384F8743084F87630A36DE26DC4F85C
:1069680077300023C4F8803094F86030C4F87B2076
:106978009A0684F875100FD194F8612094F82030A5
:106988009A4209D294F86230013B0F2B04D80123B4
:1069980084F87F302377A0E7206841F0B5FE022312
:1069A80084F87F300423F5E7204641F039FF94E767
:1069B800032B92D1302394F8619003FB0949D4F852
:1069C800803009F124095B44C4F88030BBF1000F22
:1069D80016D0484642F04BF890B141465A464846D0
:1069E80042F057F8804628B902215B461F4A1C48E6
:1069F80040F00FFED4F87B30A3EB0803C4F87B30DB
:106A0800D4F88020E36D9A420DD2484642F02FF820
:106A180000287FF462AFD4F88020E36D9A4202D256
:106A2800206841F087FE484642F048F8003818BF11
:106A3800012084F87F00B5E7304695F8189041F0BA
:106A480058FE81457FF449AF237F052B10D184F888
:106A58001C8042E755534243DC100020AD22080851
:106A6800AC5607080C220808302208084B230808EF
:106A7800022B7FF432AF4FF030092A8AD4F88030E5
:106A880094F861801344C4F8803023681969D3F8F6
:106A980004B091F8613009FB0311243108460391D1
:106AA80041F0E5FF03990246584641F04DFE0028A3
:106AB8007FF413AFD4F87B3013B1206841F024FE83
:106AC80009FB08402430AFE7304695F8188041F0BC
:106AD80010FE804502BFA37F03F1FF33A37707E7CA
:106AE800EB7F0133EB77A4E62046FFF7E7FDA0E64E
:106AF800204641F0D9FE9CE6022084F87F0004235A
:106B08001AE094F9601040B90029206802DA41F0CF
:106B1800FBFDBEE641F00EFEBBE6002914DA90420A
:106B280002D8B9F1000F06D1206841F0EDFD02232B
:106B380084F87F30E3E702232377237F022B0ED1EB
:106B4800204641F0B1FE13E6904202D8B8F1000F9A
:106B580003D1206841F0EEFDE9E70323ECE7032BBE
:106B680003D12046FFF7AAFD02E6042B7FF400AE0E
:106B7800A37F2BB101211D4A1D4840F041FDF7E5D7
:106B8800206841F0B6FD8046204641F09AFD054652
:106B9800024604F1730304F17F0153F8040B8B429E
:106BA80042F8040BF9D11B782946137040460D2290
:106BB800FFF7CEFC06460146206841F0D9FA78B1C5
:106BC8000C4A434601210A4840F023FD3046FDF7B0
:106BD80057FD2946204641F057FE41F021FEC7E502
:106BE800A37F0133A37705232377C1E57123080821
:106BF800AC560708AD220808802938B50D4614465A
:106C080021D083290DD019BB8023537183230320FE
:106C1800117193710023E07023706570A3700430C4
:106C280038BD0223137101235371002393710A2382
:106C3800D37108224168A0185DF068FF064B0E204A
:106C48001B882382E6E7044B02201B889380E1E738
:106C58006FF08500E4E700BF174308082DE9F0410D
:106C68008769D0F82480BA4228BF3A46B2FBF8F4C4
:106C78000646C2692346006840F037FE0546C0B99B
:106C8800B7FBF8F7A7420BD1002205213068FCF7C3
:106C9800E7FB28B101210A4A0A4840F0B1FC012566
:106CA800F3692344F3613DB10020074BB362BDE8AB
:106CB800F08100240125E7E7706A6043F7E700BF29
:106CC80092230808AC5607080203000C81420B46C1
:106CD80007B509D302210D4A0D4840F09AFC6FF020
:106CE800150003B05DF804FB6AB101391144814213
:106CF80001D28B4207D90221009305481346054A61
:106D080040F091FCEBE70020EBE700BFA92308085F
:106D1800AC560708C02308080C290346084616D1B4
:106D28001B78252B12D009D8122B10D8084A42FA02
:106D380003F313F0010F08BF0620704703F0FD02AC
:106D4800282A03D05A2B08BF0A2070470A20704708
:106D5800F6FFFBFF2DE9F041984690F82C3086B0FD
:106D680023F00C0380F82C300023C0E9043383613E
:106D7800062A04460F460B7840F010810BBB4B796E
:106D88005B0724D490F82C309F070DD402234FF4CE
:106D980068521946002584F8283084F8291062853D
:106DA800284606B0BDE8F08141F0BDFD0028EDD1D0
:106DB800002319461A46EDE70223052145F202325F
:106DC800E8E7032B36D14E7916F0040604D00223E7
:106DD80005214FF41052DDE790F82C308DF807604C
:106DE80043F0040380F82C307023ADF8043090F899
:106DF80029300D7903F00F038DF806300A23122D80
:106E080028BF12258DF80B30438D2A465BBA4046C1
:106E180001A98DF808608DF809608DF80A6003965D
:106E2800ADF81030ADF81260ADF814605DF011FEE9
:106E3800A662B5E71B2B00F0898009D8122B1AD05F
:106E48001A2B61D00121B24AB24840F0E2FBBEE7FA
:106E58001E2BF7D14B795E07B9D40B7913F00303D6
:106E680000F09780012BA3D190F82C3043F0010358
:106E780080F82C309CE74B795E07A8D490F82C302A
:106E880043F0040380F82C304A7812F002061FD130
:106E9800D5078B7822D5B1F8035042461946FFF73B
:106EA800ABFE6DBAADB285420BDAB7F803506DBAD6
:106EB800ADB200231A4684F8283084F82960628528
:106EC8006EE742462046B978FFF796FE051EF0DACF
:106ED800022305264FF410520025ECE72BB10221BE
:106EE8008D4A8C4840F095FBF2E7B1F803504146D3
:106EF8006DBAADB241F04DFD232DD6D9414620469D
:106F080041F047FD2425D4E74D7915F004057FF4B9
:106F18005EAF90F82C3043F0040380F82C308B7867
:106F28003F2B0ED1CE78002ED2D10D790323042D1C
:106F380028BF042540462A4601A901935DF089FD32
:106F4800B7E7022305264FF41052B4E74B795907E7
:106F58003FF53DAF3B791A090CD19A070AD5DB07F3
:106F680015D494F82C3003F00303032B3FF424AF1B
:106F7800002305E094F82C209707C2F34003F0D5CE
:106F880094F82C2063F3410284F82C2010E70123A5
:106F9800F6E790F82C2063F30002F5E70A2A7FF45D
:106FA80051AF2A2B1AD8222B7FF64CAFA3F123021C
:106FB800072A3FF647AF01A151F822F03B700108BC
:106FC8004D6E0108BD7001084D6E01084D6E010837
:106FD800257101084D6E01087D7101085A2B7FF457
:106FE80031AF4D7A15F004057FF4F1AE90F82C30EE
:106FF80043F0040380F82C308B783F2B40F0DD8081
:10700800CE78002E40F0D9804FF4C063CDE9013628
:10701800B1F8075040466DBAADB2082D28BF082513
:1070280001A92A465DF015FD3246334684F828202A
:1070380053E07B7A13F004037FF4C9AE01AEADF8D8
:107048000430B370082390F82C208DF8073042F0F4
:10705800040280F82C2041F066FC0028B5BF4FF0F0
:10706800FF3302220322236A8DF80C20A8BF1BBA23
:107078000293636A31461BBA8DF80D30C3F30722B9
:10708800C3F307438DF80F3094F82C308DF80E2099
:1070980043F0040384F82C30B7F8075040466DBA23
:1070A800ADB20C2D28BF0C252A465DF0D2FC00237A
:1070B800A36275E67E7A16F004067FF488AE90F82F
:1070C8002C3043F004039D0780F82C3009D40226A5
:1070D8004FF46853002584F8286084F82960638594
:1070E8005EE641F020FC0028F1D1236A03B1013BA0
:1070F80094F82C10626A1BBA12BA41F0040184F8A1
:107108002C100825C8F80030C8F804200023E2E74E
:1071180007240808AC560708EA2308087B7A5807AA
:107128003FF555AE94F82C30D7F8026043F00403CD
:107138009907B7F8075084F82C307FF527AE20461A
:1071480041F0F1FB00287FF421AE6DBA36BAADB23A
:107158002A463146206AFFF7B9FD20B102230521EE
:107168004FF4045216E6174B2361636AE6616B43DA
:10717800A3611DE67B7A5A073FF529AE90F82C30BB
:10718800D7F8026043F00803B7F8075080F82C30AE
:107198009B077FF5FBAD41F0C6FB00287FF4F6ADF9
:1071A8006DBA36BAADB22A463146206AFFF78EFD6F
:1071B8000028D3D1044B6361D7E7022205264FF498
:1071C800105333E7FD890508656C010810B504699B
:1071D8000346204640F8143B0122002144F02BF9D5
:1071E80004F12C00024944F09EF9002010BD00BFB4
:1071F8008573010838B503461B6940685C681B69DC
:1072080025685A681AB19A680AB1DA683AB913480F
:107218000121134A40F0F4F96FF0150038BD10331E
:10722800D3E8EF1F41F00101C3E8E21F002AF7D1BC
:10723800216909B90020F1E72B7A002BFAD140F037
:10724800F1FC28B10121074A044840F0D9F9F1E7D7
:10725800206940F074FD2872ECE700BF94560708D7
:10726800222408086322080838B5046940680068C1
:1072780004F11005D5E8AF5FED071FD40BB15D68C9
:107288003DB9104A1048012140F0BAF96FF01500D5
:1072980038BD90F820501DB1DD680DB90B4AF1E7F3
:1072A80085791DB19D690DB9094AEBE7C4E9021258
:1072B80063600274120A42740020E9E76FF07700F5
:1072C800E6E700BF4C240808945607086B24080812
:1072D8008A2408082DE9F347D0F804A006698846EF
:1072E80015467768DAF8044006F11003D3E8AF3F93
:1072F8009B073BD5236960685B68D3F8009040F032
:10730800EBFB00220023012829460CBF99F81B90AB
:1073180099F81490DAF80C00CDE90023424640F0C1
:1073280073FB054650B90121124A134840F068F929
:107338006FF00B04204602B0BDE8F087014680F8E4
:107348001890204640F014FF044618B12846FDF76F
:1073580097F9EFE7FB69002BECD14FF0FF324FF0C4
:10736800FF3306F1140004F039FEE3E76FF00C0474
:10737800E0E700BFAB2408089456070870B550F83A
:107388002C3C5C6865681C38D0E8AF3F9B0725D566
:107398002B6968685B681E6840F09EFB0022012824
:1073A8004FF00003A0680CBF96F8296096F8226099
:1073B80040F026FB044630B9094A0121BDE8704077
:1073C800084840F01DB901460676284640F0D0FE30
:1073D80020B12046FDF754F9034AEEE770BD00BF1F
:1073E800C624080894560708E024080807B5084A80
:1073F80092E80300CDE9000106488268126822B1CC
:107408006946904703B05DF804FB6FF05700F9E751
:10741800D05607081C5107081F2808B5034606D987
:1074280009480121094A40F0F4F8002008BD01206C
:10743800074A00FA03F3D16833EA0101F6D012696A
:10744800934318BF0020F1E764550708152508087D
:1074580000200246012100F01F021F2808B501FA8A
:1074680002F2034606D90648064A40F0D2F86FF001
:10747800150008BD044B0020DA601A61F9E700BF67
:107488006455070815250808002002462DE9F04133
:10749800054600264FF001080E4F6B78F4B2A34260
:1074A80001D8BDE8F0812B781C442046FFF7B4FFD3
:1074B80068B12046FFF7CEFF57F834303BB107EBF1
:1074C800C40204F01F04516808FA04F09847013612
:1074D800E3E700BF7C370020014B1954704700BF19
:1074E800300C0020034670B1B0FA80F2C2F11F02DE
:1074F800D2B206498856064AD2F880100B43C2F821
:107508008030FCF7B1BBFF22F3E700BF300C00204E
:1075180000200246034AD2F8803023EA0003C2F86A
:107528008030704700200246032921D8DFE801F0A7
:10753800020C10190F4B1A6822EA00021A605A68E6
:1075480022EA00025A6070470A4B1A680243F5E7BC
:10755800084B5A6802435A601A6822EA00021A6005
:107568007047044B1A6802431A605A6810435860FF
:10757800704700BF0020024630B5B0B1B0FA80F3C2
:10758800C3F11F03DBB20B4850F833408C4204D1DF
:1075980000EBC3056D68954205D044B940F8331037
:1075A80000EBC3004260002030BDFF23EBE76FF023
:1075B8000F00F9E77C37002060B1B0FA80F3C3F11F
:1075C8001F03DBB20021044A42F8331002EBC30266
:1075D80051607047FF23F5E77C370020C300074A56
:1075E800C0F38100183052F8202003F018000F2350
:1075F8008340134023FA00F0704700BF0020024682
:10760800F8B504690D4600AFA034D4E8AF3FC3F322
:107618008003994218D1164A164B6E4688B0002945
:1076280018BF13466A461449CDE905134FF4007391
:10763800ADF81C30114B42F8103F00234FF4E451D1
:107648000F48FBF7E1FBB5464DB1D4E8EF3F43F0F7
:107658000403C4E8E23F002AF7D1BD46F8BDD4E8E8
:10766800EF3F23F00403C4E8E23F002AF5D0F6E731
:10767800552508085D250808642508080300000149
:10768800445607082DE9F0470546894690461F46A7
:10769800D0F808A041F0A3FC0446D0B1067FF30758
:1076A8000AD590F8203018480121184A3FF0B1FF58
:1076B8006FF07700BDE8F0873B464246494641F007
:1076C8004CFC48B994F820300121114A0E483FF08B
:1076D800A0FF6FF01200EDE79DF8203026F00606B7
:1076E80084F82180678484F824302677DAF8183003
:1076F800214628469847B0FA80F3227F5B0963F356
:1077080000022277D6E700BF445607087625080806
:107718009025080870B50546866841F060FC044667
:10772800D8B1037FDB0709D490F820300C48012139
:107738000C4A3FF06EFF6FF0770070BD0146F369A9
:107748002846984738B1237F03F00103227F63F36B
:1077580000022277F1E70346F8E76FF01200ECE742
:1077680044560708B22508082DE9F3411746D0F812
:1077780008800546D8F83C300E469847002200237A
:1077880039460B48FCF7FEFE044670B901213B461A
:10779800084A094800963FF046FF2846D8F8403086
:1077A8009847204602B0BDE8F0810676F5E700BFAD
:1077B80040120020CD2508084456070813B5036970
:1077C8000C46D3F8A40091F8201043F071F894F80F
:1077D800203048B101210090084A09483FF023FFB2
:1077E8006FF0040002B010BD5B0601D10020F9E77C
:1077F800237F43F002032377F8E700BFFB2508083F
:107808004C560708F8B591F9203091F82060002B04
:1078180001DB0020F8BD7306FBD047684C8CB7F835
:107828004830C4F30A04A34294BF03330334006905
:107838008CBFA3089B08D0F8A440402B98BF5B00DE
:10784800D4F8E8049D008AB9A84224BF401BC4F8B4
:10785800E80491F820100022204601F07F0143F04F
:10786800BBF80028D5D06FF00400D3E7BA68121A25
:10787800AA4207D20A4832460A4941F012FF6FF07D
:107888000B00C7E720469AB206F07F0143F0A4F840
:107898000028E8D1D4F8E8342B44C4F8E834B8E731
:1078A8004C56070829260808F7B54668036974681E
:1078B800D3F8A45064009834A1B20746A40028461F
:1078C80043F0A9F8C5F8E84401241022002128460D
:1078D80043F082F8D5F8E8344033C5F8E8347368E3
:1078E8009C420ED3284642F0F5FE054680B1174962
:1078F8000246174841F0D5FE6FF00404204603B055
:10790800F0BDE1B20022284643F066F80134E6E70C
:1079180002460146009040233846FFF7B3FE04466E
:1079280028B12A460B490A4841F0BBFEE6E7024661
:107938000090402380213846FFF7A4FE044608B192
:107948008022EFE73069FCF78FF9D7E74C26080863
:107958004C5607086126080838B504460369D3F869
:10796800A45043681869FCF78DF900212046FFF7F9
:10797800D1FE38B10C490D4841F098FE6FF004046F
:10798800204638BD20468021FFF7C4FE0446002863
:10799800F0D1284642F0BBFE02460028F0D0044948
:1079A800024841F07EFEE9E77B2608084C560708A6
:1079B8009E26080838B503690546D3F8A440204632
:1079C80043F004F8024630B10D490E4841F069FE13
:1079D8006FF0040038BD0021142043F0E4FE204677
:1079E80042F0F7FF04460028F2D101462846FFF787
:1079F80007FE22460221284641F02BFB2046E9E7F4
:107A0800B22608084C56070870B50369456804464D
:107A1800D3F8A40042F049FE024618B11A491B489F
:107A280041F03FFE6668F069D8B14368984704465C
:107A3800B8B117490246154841F033FE002C19DB4E
:107A480000F0F8FB024618B11249104841F029FE2F
:107A58002869FCF72BF910B12869FCF713F9002005
:107A680070BD0D48716983685B6843B90B49074865
:107A780041F01CFE0A49054841F018FEE0E7984726
:107A88000028DDD0F2E700BFD22608084C560708C8
:107A9800E82608083B2708081C5107080627080895
:107AA800222708082DE9F04103690646D3F8A450B7
:107AB800476800F08BFB044638B12E4902462E4831
:107AC80041F0EFFD2046BDE8F08176682B4896F836
:107AD8004A30D0F80880012B13D97169D8F81830CA
:107AE800083153B92649244841F0E0FD2549224888
:107AF80041F0DCFD6FF00404E4E7224698470028D3
:107B0800F0D1D8F8003071690BB91F49EBE71B4871
:107B1800984704460028F8D1F06950B1036898479F
:107B2800064630B119490246134841F0BAFD002E05
:107B3800DCDB40F2E442002128465CF0B0FF3B6801
:107B480028462B607B682B7140232B723B6B6B7232
:107B58007B6BEB7102F06EFE024620B10C490648C1
:107B680041F09FFDC6E7284642F0D1FD0028A9D084
:107B7800C0E700BF592708084C5607081C510708DA
:107B880076270808D027080898270808B327080880
:107B9800E82708082DE9F04F064600274FF0280A85
:107BA8004FF0400BD0F810904568D9F8A4808BB0FE
:107BB8006B68BB4256D800274FF0280A4FF0400B9D
:107BC8006B68BB4200F2858099F8803023F06A0325
:107BD80043F06A0389F880306B6B2BB999F88030D1
:107BE80043F0010389F88030C8F8E46408F5C061FF
:107BF80008F5BA600823042243F008FBD5E91012FF
:107C080008F59E684FF0000A4FF0000B6FF007036D
:107C180001200027CDE90330CDE906AB4046CDE988
:107C28000177514B009604F053FC3168404643F00D
:107C3800B8FCEB6898473946A86909AA42F080F968
:107C4800041E07DB099B3A461979186842F08AF93D
:107C5800041E6BDAA31C69D044492246444841F00B
:107C680020FD30E00AFB07F1EB6B17F0800F0B44A7
:107C78009A7E07F07F000CBF42F0400242F02002DB
:107C88009A769A7E83F8207050B942F001029A766B
:107C9800EB6B5FB1EB6BB5F848200B441A8307E038
:107CA80022F00E0242F00E029A76F3E7A3F818B01B
:107CB800EB6B3046194441F0A4F9044638B12D491C
:107CC8002B4841F0F3FC20460BB0BDE8F08F01379C
:107CD8006EE70AFB07F1AB6B67F07F020B4483F892
:107CE80020209A7E7C0642F020029A760BD1D2B2EE
:107CF80042F001029A76AB6B67B1AB6BB5F84820DE
:107D08000B441A8308E09A7E22F00E0242F00E021B
:107D18009A76F2E7A3F818B0AB6B3046194441F0F5
:107D280070F904460028CAD1013749E7A86A08B99A
:107D38000024C8E7283543F07DF930B90E490C48CE
:107D480041F0B4FC6FF01504BDE74FF4B0112846BC
:107D580041F066FC0028EBD00849054841F0A6FC34
:107D68006FF00404AFE700BF517E01081828080827
:107D78004C560708FC27080836280808522808081F
:107D880073B5D0F8A46008460C46154641F030F9A2
:107D980018BB94F82030298A802BEA680B4602D158
:107DA800402928BF4023D018C91AE86029823046E4
:107DB80094F8201042F062FD58B194F82030012167
:107DC8000090074A07483FF02EFC6FF0040002B00D
:107DD80070BD0121204641F00FF90020F7E700BFF0
:107DE8006F2808084C56070813B591F820300C4640
:107DF800D0F8A400DBB9537EDB071ED4538AC0F841
:107E0800EC34538A402B28BF4023D26894F82010C2
:107E180042F00FFD68B194F8203001210090084A23
:107E280008483FF000FC6FF0040002B010BD538A10
:107E3800EBE70121204641F0DFF80020F5E700BF1D
:107E4800A02808084C5607082DE9F3470746036998
:107E5800D3F8A4604FF0FF334FF0FF3201A906F5C5
:107E6800BA6003F023FF9DF80430012B5FD0022B8A
:107E780007D0002BEED1384606F29C4141F01CF9A0
:107E8800E8E79DF80590D6F8E48449F0800A514661
:107E9800404641F0A4F80546002141F0ADF82846D7
:107EA80041F0CAF804460028D4D019F07F0F18D141
:107EB800038AB3B1402B28BF4023C26880213046D3
:107EC8001D4642F0DBFC024620B13F493F4841F0E5
:107ED800E8FBBFE7238A5B1B2382E3682B44E3604C
:107EE800B8E7204641F0ACF8814660B1204641F041
:107EF800ABF8E26800235146304642F0BFFC024628
:107F08000028A7D0E1E7284641F092F84A46014602
:107F1800404641F0AAF8284641F08EF8024600286B
:107F280098D02946D8F81000FFF72AFF92E79DF865
:107F38000590D6F8E48449464046BDF806A041F0CD
:107F48004EF8054641F078F8044648B920494A46B3
:107F58001E4841F0A6FB2146284641F04DF879E736
:107F680051460C303FF07CFDB9F1000F17D1BAF142
:107F7800400F14D1228AD6F8EC349A420FD2E06826
:107F8800638A61699B1A411A5B1A402B024428BF15
:107F98004023304695F8201042F04BFC5AE728461B
:107FA80041F046F800220146404641F05EF8284676
:107FB80041F042F8024628B12946D8F81000FFF7E8
:107FC80013FF47E70146C7E7D02808084C560708BB
:107FD800F9280808F7B591F82150036905F0030559
:107FE800D3F8A4706B1E022B4FF001020C4688BF19
:107FF8000025FFF707FC064698B9628C2B463846E1
:1080080094F82010C2F30A0242F0B7FB48B194F882
:10801800203001210090044A04483FF004FB6FF02F
:108028000406304603B0F0BD122908084C5607086C
:1080380013B503690C46D3F8A40042F08BFB40B19A
:108048000121009023460448044A3FF0ECFA6FF0FF
:10805800040002B010BD00BF4C5607083B290808B1
:1080680037B5036905460C46D3F8A40091F82010EB
:1080780042F0B7FB024630B92146284603B0BDE8B6
:108088003040FFF7BFBB94F8203001210090044A2C
:1080980004483FF0C8FA6FF0040003B030BD00BFD9
:1080A800692908084C56070873B5036905460C4644
:1080B800D3F8A40091F8201042F031FC58B194F89C
:1080C800203001210090164A16483FF0ACFA6FF0B4
:1080D800040002B070BD237F60F34103237720467C
:1080E80040F0AAFF064608B90020F2E7204640F013
:1080F8007FFF94F92030002B07DA0028F4D13246AC
:1081080021462869FFF73CFEEEE70028ECD132460D
:108118002146286902B0BDE87040FFF765BE00BF80
:10812800932908084C56070837B50D46044642F00F
:108138009DFB01238DF805508DF80430ADF806003D
:108148000022002301A904F5BA6043F072F818B1BF
:108158000249034841F0AAFA03B030BDC329080810
:108168004C560708002307B5ADF8063002238DF8F2
:1081780005108DF804300022002301A900F5BA602B
:1081880043F057F818B10349034841F08FFA03B098
:108198005DF804FBC32908084C560708002307B5F7
:1081A80001930022002301A900F5BA6043F041F8C9
:1081B800002803DA0349044841F078FA03B05DF86F
:1081C80004FB00BFC32908084C56070838B54FF010
:1081D800FF324FF0FF33124803F000FF0446C0B9E6
:1081E800104D2B685A1C2A6083B90F4BDA6802F4C9
:1081F8004032B2F5003F0ED26FF0040401210B4A61
:108208000B483FF0FDF92B68013B2B60044803F055
:10821800A9FE204638BD1A6942F080521A61F5E776
:108228006C110020DC39002000080246F6290808F5
:108238002C56070810B54FF0FF324FF0FF330A48AD
:1082480003F0CCFE044660B9084A1368013B13608A
:1082580023B9074A136923F080531361024803F0D6
:1082680081FE204610BD00BF6C110020DC390020C3
:1082780000080246074B1A6822F004021A605A687E
:10828800D207FCD40222DA601A6842F001021A60AE
:10829800704700BF00040340044B1A6822F0010233
:1082A8001A601A68D207FCD4704700BF0004034064
:1082B8000D4A0E49936813F4000308D0936813F429
:1082C80000030CD1D2F8F42051F8230070479068CD
:1082D800000207D4D2F8F430C3F30333F4E7936809
:1082E8001B0FF1E79268EFE7000C0246D05F070822
:1082F80038B50B880D46C3F30B03122B144636D83A
:1083080013B96FF0850031E0013B112BF9D801A2B8
:1083180052F823F097830108CB830108658301088D
:108328000B8301080B830108B3830108AD8301089F
:108338000B8301080B8301089183010891830108CD
:1083480091830108918301089183010891830108B1
:10835800B783010897830108978301084FF4FA400F
:1083680020602B68B3F5805F2ED2002038BD882BA3
:108378000AD003F67473C3F30B031C2BC1D8164A37
:1083880022FA03F3DB07BCD5144B1868E8E7FFF7BC
:108398008FFF4FF42023A0FB0303400B40EAC340A8
:1083A8004008DDE7FFF784FFDAE70D48D8E7FFF775
:1083B8007FFF4FF42023A0FB0303400B40EAC34098
:1083C800CEE74FF40040CBE7C3F313330133B0FBE0
:1083D800F3F02060C9E700BF11011111C8060020A1
:1083E800006CDC0237B5A84CA84BE26902F00C021D
:1083F8001341D80700F14381FFF75AFF236AA44AC3
:1084080003F00F03D35C20FA03F5A24BDA6842F4B9
:108418004032DA60DA681104FCD59F48854201D2FF
:1084280003F072F8984CD4F8943043F00403C4F87D
:108438009430D4F8943003F004030093009BFAF7C7
:10844800D9F9D4F8F03023F0180343F01003C4F836
:10845800F030D4F8F03043F00103C4F8F030D4F829
:10846800F0309A07FBD5D4F8F03043F08003C4F815
:10847800F030854CD4F8F0301B05FBD5FAF7D8F965
:10848800A36843F40003A360A36823F0704343F098
:108498008043A360236843F040032360236843F0CC
:1084A80008032360236843F001032360764B1A68AE
:1084B8005407FCD5D3F8942050070BD4D3F8942054
:1084C80042F00402C3F89420D3F8943003F0040374
:1084D8000193019B6C4CFAF78DF9D4F8F03043F016
:1084E8008063C4F8F030D4F8F0301901FBD5FAF7FE
:1084F8009FF9236843F480532360634B1A689204FE
:10850800FCD5DA6902F00C020C2A1AD11A68540553
:1085180007D41A6842F480721A605B4A13685805D7
:10852800FCD5594BDA6922F0030242F00102DA6104
:10853800DA6902F00C02042AFAD11A6A22F00F0250
:108548001A62514B1A6822F080721A609A6A22F0F5
:10855800030242F001029A624E4AD16821F4802156
:10856800D160D46814F48044FBD19A6A464922F455
:1085780070429A62494B4A4A1B699342B6BF494ABC
:10858800102393FBF2F38A6A03EBD37322F470424D
:108598005B1042EA03338B623E4BDA6842F4802276
:1085A800DA60DA685104FCD5FFF782FE3E4AA0F58E
:1085B8007413A3F51063934205D93C4B394A03441D
:1085C80093425ED20C24304B9A6A22F470629A620B
:1085D8009A6A22F00C0222439A625A6B6FF30802DD
:1085E80042F04F025A639A6A22F010029A625A6B5A
:1085F80022F4FE0242F480325A639A6A42F400324C
:108608009A625A6B22F0FE4242F080725A639A6A6A
:1086180042F480229A621A6842F080721A601A68DC
:108628009201FCD5DA6A22F00302DA621A6B22F0B0
:1086380003021A631A6A22F00F021A621A6A22F0F7
:1086480070021A621A6A22F4E0621A625A6A22F006
:1086580070025A62DA6942F00302DA610A4AD3699F
:1086680003F00C030C2BFAD10B4CA54202D3204685
:1086780002F04AFF00200E4B1C6003B030BD002002
:10868800BCE66FF02100F8E7000C0246FEEFFFFFA2
:10869800524408080008024600688909D05F0708A4
:1086A8000020A10700127A0000093D00FFED85FFB8
:1086B800C8060020192808D8054BC34013F0010F3D
:1086C8000CBF6FF08500002070476FF08500704781
:1086D800CEFC060208B5074842F0ACFC38B10648A3
:1086E800FBF78AFE0448FAF735F8002008BD6FF05A
:1086F8001200FBE7F8520708058701080A2838B571
:108708000446074D04D1AB680D2128465B6898479D
:10871800AB6803485B68E1B29847204638BD00BFA4
:10872800F8520708064A11680B6823F004030B6027
:108738005068044B196883685B6803B11847704731
:1087480078050020E405002010B5094BD3E9004066
:10875800084B196883681B6803B19847236843F07E
:1087680004032360236843F00803236010BD00BF9F
:1087780078050020E405002008B5EFF311811023E7
:1087880083F31288BFF36F8F0120094B93F84820B9
:1087980083F8480081F31188BFF36F8F32B9FFF770
:1087A800D3FFBDE808405E20FBF75EBA08BD00BFF6
:1087B8007805002038B54368056939486860196844
:1087C80083681B6853B19847044650B1012123467A
:1087D800344A35483EF01DFF204638BD6FF0570437
:1087E800F4E7012205F10800114642F024FE0122B7
:1087F800214605F1200042F01EFE05F138002B4904
:1088080042F091FE072385F86130042385F8623031
:108818000F2385F84C300C23224685F84D3021462D
:108828005E2085F85E4085F85F4085F8604085F8F1
:10883800494085F84A4085F84B403FF080F81C4B8A
:108848001C491B681A681D6922F07C4222F07F02CD
:108858008A42D86806D14AF2B0218D4202D116491F
:10886800884211D0196821EA0201144A0A431A60A1
:108878004AF2B0221A61104ADA601A6822F080427D
:108888001A601A685200FCD41A6842F004021A608E
:108898001A6842F008021A60FFF76EFF9CE700BFF3
:1088A8001C510708412A08085C5507080F99050854
:1088B80078050020000DF000BB7C0100000DF040A1
:1088C800F8B58378C678EFF3118E102484F31288F4
:1088D800BFF36F8F057890F801C05B1B33409A4255
:1088E80088BF9AB2AF1837402C4607708EF31188AC
:1088F800BFF36F8F8F188F421BD165450CD1EFF3F3
:108908001181102484F31288BFF36F8F04784470A8
:1089180081F31188BFF36F8F01799B1A994294B242
:1089280005D342F038FE68B1084803F0DBFC204666
:10893800F8BD00EB040E9EF805E0013401F801EBE8
:108948003440D8E7FFF718FFF1E700BFB005002073
:1089580070B50D4614460CB9204670BD4FF0FF3275
:108968004FF0FF330B4803F039FB224629460A48EB
:10897800FFF7A6FF064630B94FF0FF324FF0FF333E
:10898800064803F02BFB0348A41B03F0EBFAA4B240
:108998003544E0E780050020D60500209805002032
:1089A80010B51D4B01461B68EFF31184102282F3AA
:1089B8001288BFF36F8F5A68500605D45A68D207D9
:1089C8001DD46FF00A0015E01A6842F080421A6060
:1089D8001A6822F080421A600A221868400005D4FA
:1089E8005868400602D458684007E7D5013AF4D1E0
:1089F8006FF0040084F31188BFF36F8F10BD5A68BD
:108A08009207F5D4586810F04000F1D19B680B60CC
:108A1800002BEFD1D5E700BF780500202DE9F743FB
:108A2800D8078846144605D43148FFF749FF03B0F4
:108A3800BDE8F083002A37D0EFF31185102383F3C4
:108A48001288BFF36F8F5E20FBF730F906465E2071
:108A5800FBF718F985F31188BFF36F8F0EB9FFF78D
:108A680073FEDFF89490D9F800305A68510713D490
:108A78005B685A0610D44FF0804325461D4FC7F84F
:108A88008831D9F800305B68DB070FD4BFF34F8F0C
:108A980020BF40BF20BFF4E701A8FFF781FF0024F3
:108AA80016B35E20FBF7E0F82046C0E701A8FFF701
:108AB80077FF4FF080420346C7F8882188B9291FFD
:108AC800019A89B2002DEBD0A94203D1002BD8D04E
:108AD8000192D6E7013DADB208F805200123120A3C
:108AE800F0E7002DCDD1DBE7FFF71CFEDCE700BF88
:108AF800C105002000E100E0780500202DE9F743DA
:108B080001A8FFF74DFF002843D1042780460146FE
:108B1800264C019A94F84B3094F84CC094F84AE0EB
:108B2800A3EB0E053CEA05055FFA82F91ED194F81D
:108B3800601094F85F6094F861508E1B35EA060661
:108B48002AD108B184F84B30B8F1000F00D0019257
:108B58005E20FBF797F8FFF7E5FD002384F848301F
:108B6800134803B0BDE8F04303F0FCB9E01880F8FF
:108B78004E90012001330CEA0303013F4FF0010836
:108B88004FEA1222CCD108B184F84B300192002967
:108B9800E6D103B0BDE8F083661801310D4086F8D0
:108BA8006390012184F86050E7E700BF7805002052
:108BB8009805002000487047745D0708044BB3F817
:108BC800A0379B020B60002318464B60704700BF1C
:108BD8000000FA0B07B50346054A00910548012134
:108BE8003EF021FD6FF0150003B05DF804FB00BFF7
:108BF800A72A08087455070873B506466422002397
:108C0800684642F02AFEDDE9004533691B681A6AA6
:108C180012F0FA0212D01A6A02F0FA021A626FF01F
:108C2800040002B070BD22462B46684642F03AFE68
:108C3800DDE9003213430CBF0122002233691B68AF
:108C4800186A10F48030ECD0002AECD00A230121F5
:108C5800024A03483EF0DDFCE1E700BFD12A0808DC
:108C68007455070838B5036905461C6849B1FFF70C
:108C7800C3FF58B12869043003F074F96FF0040099
:108C880038BDA36A002B06DB0020F9E7A36A43F08E
:108C98000043A362F8E7034BA36003F18833A360A2
:108CA800F2E700BF2301674573B5012306460D4669
:108CB800144640F0F7FE50B90A482B4601210A4AEB
:108CC80000943EF0B0FC6FF0150002B070BD3CB1EE
:108CD80022462946304602B0BDE8704040F0BFBE8B
:108CE8002046F2E774550708E52A0808F7B51C4638
:108CF80017460123224605460E4640F0D3FE58B9D2
:108D0800012100943346154A15483EF08CFC6FF05B
:108D18001504204603B0F0BD002CFAD0286940F0B5
:108D280070FE00212846FFF79DFF98B9314623467B
:108D38003A46284600F0B8F8064601212846FFF7CB
:108D480091FF002E14BF344604462869043003F00E
:108D580009F9DEE76FF00406EFE700BF102B0808FB
:108D6800745507082DE9F84F494B17461B680D46FF
:108D7800824603F001084FF0000BFFF78DFA013F20
:108D8800DFF82091434E2F44AF420CD3DAF810306D
:108D98001C68A36A002B0EDA01213F4A3F483EF0C7
:108DA8002FFC6FF0040BB8F1000F01D0FFF762FA47
:108DB8005846BDE8F88F5046FFF71EFFB0F1000B8C
:108DC800F1DBDAF810301B681B6C9B0252D54FF6AA
:108DD800FD70B9F8A010226C4B1E9BB2834202F4BE
:108DE800801250D8B5EB412F2CD26B0B002A43D1FF
:108DF800A26A22F40062A262A26A504642F002020B
:108E0800A262A26A22F47E72A262A26A42EAC30342
:108E1800A362A36A43F48033A362A36AFFF7ECFE5C
:108E2800DAF8103083461B681B6C13F4001FA36A22
:108E380014BF334023F002030028A362B3DB05F517
:108E48000055A1E7B5F5801F0BD332B1A36A23F40F
:108E58000063A3626B0B803BCEE7A36A43F4006315
:108E6800F7E701212B460E4A0C483EF0D2FB6FF083
:108E7800150B98E76B0BBFE7B5F5801FE6D2A26A22
:108E880042F40062B7E7B5F5801FAED3DDE700BF57
:108E980000040340FDF7FFFF612B08087C55070815
:108EA8006E2B08080007FA0B2DE9F84F00249846A6
:108EB800324B0D461F6806469146A346FFF7ECF96C
:108EC80007F0010705F10065D8450DD93369D3F8D6
:108ED80000A0DAF82830002B0CDA0121284A2948AA
:108EE8003EF08EFB6FF004040FB1FFF7C3F9204684
:108EF800BDE8F88F3046FFF77FFE041EF4DB2BF049
:108F080003024A44111F0B460C3253F8040F00BBEE
:108F18009342FAD1DAF8283043F00103CAF828302E
:108F2800DAF828302B4651F8040F914243F8040B25
:108F3800F9D13046FFF760FEDAF82830041E23F036
:108F48000103CAF8283005F11005CDDB0BF1100B31
:108F5800BAE7284600230468013408D005F17845AB
:108F68000121094A07482B443EF053FBBAE7013375
:108F7800042B00F10400EED1CCE700BF000403404D
:108F8800612B08087C550708872B080830B5104C5A
:108F9800104D0C60236813B12B68136030BD036952
:108FA8001B68196C1B6C9B020FD54FF6FD700A4BA2
:108FB800B3F8A030591E89B281428CBF4FF4807338
:108FC800DB0823604FF40053636001232B60E4E760
:108FD800E4390020E03900200007FA0B2DE9F843B6
:108FE800D0F8049090460746D9F808000D461E466A
:108FF8003FF083FFB8F5001F044616D12846D9F87C
:109008000840FEF7EBFA84420CD129463FF075FF81
:109018000446FEF77FFA2046FEF7CEFA00212046E6
:10902800FEF782FA0020BDE8F883B8F5800F20D05B
:10903800B6F1806F19D0B6F1C06F18D0B6F1007FC5
:109048001AD102263A4620460E49FEF795FAB0B9DB
:109058002846D9F808103FF055FF20463146FEF75C
:1090680063FA2046FEF73EFADCE70126EAE7032624
:10907800E8E76FF08500D6E76FF01500D3E76FF0EB
:109088000F00D0E7159C05080C291FB528BF0C2137
:109098000C460A4BD3F8082712BA0192D3F80427D2
:1090A80012BA0292D3F800370A461BBA01A90393F1
:1090B8005BF0CFFC204604B010BD00BF0000FA0BE7
:1090C800174AD2F8F430D2F8F410C3F30073490108
:1090D800D2F8F4104FEA4303D2F8F42048BF43F023
:1090E8000103890048BF43F0100352000C4A48BFEF
:1090F80043F01003D2F8F410D2F8F420090148BF65
:1091080043F00403002A074AB8BF43F08003926B78
:10911800520748BF43F0800303600020704700BF38
:10912800000C02460008024680B500AF8AB06A46C5
:10913800094B0791CDE905304FF40073ADF82030A5
:10914800064B42F8103F00234FF411510448F9F739
:109158005BFEBD4680BD00BFB52B080804000001BA
:10916800AC5507082DE9F74398460B7A164643F0A5
:109178000403046907460B720D460B460122B242EE
:109188001AD904F118094FF0FF324FF0FF3348465F
:1091980002F024FF384640F09AFD041E2DDA012122
:1091A80023461A4A1A483EF034FA484602F0DAFED4
:1091B800204603B0BDE8F0830AD2197A187D81EA07
:1091C800000C1CF0010F01D040071CD589071AD4E8
:1091D80001320C33D2B2D2E7012E0CBF002305F1C5
:1091E8001403CDE90038384695E80E0040F012FE29
:1091F800041E04DB013E0C35F6B2002EECD13846D5
:1092080040F067FDD1E76FF01504D1E7C92B0808D6
:10921800AC55070808B50121034A04483EF0F0F9A7
:109228006FF0040008BD00BFE52B0808AC5507081F
:109238000023F7B542680446066923480F46D568F7
:109248005168926801938368012ADB6833D9083131
:109258004BB91E4A01211E483EF0D2F96FF00404B2
:10926800204603B0F0BD01AA98470028F1DB376318
:1092780006F118074FF0FF324FF0FF33384602F07F
:10928800ADFE2B68204623F001032B6096F8621090
:1092980040F0E0FC2046019900F0BEF8041E06DB11
:1092A80096F861301BB12B6843F001032B603846F8
:1092B80002F058FED4E70BB9064ACBE701AA984753
:1092C8000028D4DAF8E700BF1C510708032C080867
:1092D800AC550708312C0808F8B5044646680569F6
:1092E80000274FF0FF320021284642F0A4F820461C
:1092F8003368984785F8607085F86270012205F137
:109308001800114642F097F8204600F051F8B3686B
:10931800012B25D831691F4B994230D014D81E4BE8
:1093280099422ED01D4BCB1A5942594189002046EB
:1093380041F01001FFF77CFF041E26DA0121184ACC
:1093480018483EF05DF913E0174B99421BD003F51E
:10935800C31303F5206399420CBF0A210021E6E7F5
:1093680012487168836808319B691BB96FF004045F
:109378002046F8BD3A4698470028CBDAF6E706219A
:10938800D5E70221D3E70821D1E70123002485F896
:109398006030EDE740420F00A0860100801A060009
:1093A8005F2C0808AC55070840E133001C5107083A
:1093B80037B545680021286A01AA40F0C1FD041E9E
:1093C80007DB019B00221979186840F0CBFD041EC9
:1093D80008DA012123460C4A0C483EF01AF92046C7
:1093E80003B030BD0A48696883681B683BB901212E
:1093F800084A06483EF004F96FF00404EFE798477E
:1094080004460028EBD0F2E7832C08089C5507088F
:109418001C510708A12C08082DE9F04F4FF00C0E3D
:1094280044680369002085B00393A36AE568DFF800
:109438002881DFF82891DFF828A1DFF828B1029306
:10944800029B8342039B1B6B01930DD1C3F3420222
:10945800012A39D0022A66D03A4A3B4801213EF017
:10946800CFF86FF015001DE00EFB00F7D4F824C00C
:10947800364A0CEB0706736893421DD015D853453E
:109488001CD0A3EB0B02534253419B00019A53405B
:1094980013F00E0F16D15CF807308B4212D1B36867
:1094A80000202B6105B0BDE8F08F434508D04B453F
:1094B8000CBF0A230023E9E70623E7E70223E5E7D1
:1094C8000823E3E70130BBE741F25C2E4FF47A6CE6
:1094D80040F2E2474FF4FA7602201D4B421EB1FBE0
:1094E800F2F2B3FBF2F2BCFBF2F4013CFF2C23D8FE
:1094F800BEFBF2F808F1FF38B8F1FF0F1CD8B6FB35
:10950800F2F9B9F10F0F17D8B7FBF2F2013A0F2AA7
:1095180012D8023848EA094343EA007343EA02537F
:1095280043EA0423BCE740F2145E4FF4167C4FF480
:10953800FA7740F27716CFE701301128CED1054AE5
:109548008BE700BFEB2C0808A455070840420F0022
:1095580000CA9A3B662D080840E13300404B4C0096
:10956800A0860100801A060043681B6803F1080200
:1095780052E8002F42F0010203F1080040E8002100
:109588000029F3D1174A93421ED002F18052934228
:109598001AD0154A934217D002F18052934213D041
:1095A800124A934210D002F1805293420CD0104AD2
:1095B800934209D002F18052934205D00D4A93425A
:1095C80002D0B3F1502F03D15A6842F040025A60DA
:1095D80053E8002F42F4807243E800210029F7D1B4
:1095E800704700BF00380140004400400048004078
:1095F800004C00400050004043681B6803F108021B
:1096080052E8002F22F0010203F1080040E800218F
:109618000029F3D1174A93421ED002F18052934297
:109628001AD0154A934217D002F18052934213D0B0
:10963800124A934210D002F1805293420CD0104A41
:10964800934209D002F18052934205D00D4A9342C9
:1096580002D0B3F1502F03D15A6822F040025A6069
:1096680053E8002F22F4807243E800210029F7D143
:10967800704700BF003801400044004000480040E7
:10968800004C0040005000400129034608461AD00B
:1096980002290BD0C9B91B680D4A934217D002F1B1
:1096A80080529B1A18BF0123180370471868084B8B
:1096B80098420AD003F1805398420CBF4FF40050EF
:1096C8004FF440507047002070474FF400507047E7
:1096D8000024004638B51D46094B6C0833F81220A3
:1096E8000023F7F7B9FB090241EA106100022018CC
:1096F8002A464FF0000341F10001F7F7ADFB38BDF2
:1097080038FF07082DE9F04782B0436880460C46C9
:109718001D6800AF002945D0586819698368DB685F
:109728006BB13A1D9847061E0CDA0121344A3548B8
:109738003DF066FF30460837BD46BDE8F0876FF05C
:109748005706F2E7304B9D4203D003F180539D4208
:109758002BD10026D7F80490DFF8BCA02346484652
:109768000021B2B2FFF7B6FFA0F5407050452BD9E3
:109778000136102EF2D16D468AB0D8F800306A460C
:1097880022490794CDE905134FF40073ADF8203052
:109798001F4B42F8103F00234FF411511948F9F7B5
:1097A80033FBAD466FF01506C4E72B6823F400437E
:1097B8002B607B6803EB5403B3FBF4F30F2BDAD96C
:1097C8009BB2EB600026B5E7EB6A484623F00F032F
:1097D8003343EB620F4B33F8162000231946F7F793
:1097E8003BFB002306464FF4807C1946600822465E
:1097F800E6FB0C01F7F730FBC0F31300E860E1E784
:10980800312C08083C56070800240046AA2D0808F1
:109818000400000138FF0708FFFC0F002DE9F8439A
:1098280007460E7940683B69012E0D460468D3F857
:10983800008014D0B31ED3F1000949EB03094FEAA5
:1098480089296979FFF720FFAA790346022A09D0F6
:10985800042A01D0002E6AD04FF4805005E04FF45E
:10986800C069EEE7002E5FD00020A6F1030CBCF122
:10987800010F04D86FF085031846BDE8F8830EB1D0
:10988800042AF7D0B3F5805F53D0B3F5405F52D0C8
:10989800002B0CBF012303239942EBD1494640F02A
:1098A800B5FB8242E6D1EB7953B3012B45D1244B6A
:1098B8009C4225D003F180539C4221D0214B9C42ED
:1098C8001ED003F180539C421AD01F4B9C4217D0E4
:1098D80003F180539C4213D01C4B9C4210D003F1DF
:1098E80080539C420CD01A4B9C4209D0B4F1502FA3
:1098F80006D0184B9C4203D003F180539C42B9D147
:109908002368294623F001032360384640F000FD10
:1099180003460028AED1226842F00102226095E891
:10992800030088E80300A7E74FF08050AAE7304615
:10993800A8E70023B0E70223AEE7032BB7D099E7E7
:10994800003801400044004000480040004C0040FE
:1099580000500040002400462DE9F04383B0D0F8C1
:1099680004908046D9F80400D9F81010836800AF35
:109978001B687BB19847054670B90021D9F82400C7
:109988003A1D40F0DDFA051E0EDA28460C37BD46B2
:10999800BDE8F0836FF057050121644A64483DF043
:1099A8002FFE002DF1DBE8E77B68002219791868A3
:1099B80040F0D8FA051EE8DBD8F80460D8F8103073
:1099C80034681D68236823F001032360B06841F000
:1099D80031FB38B90121574A55483DF011FE6FF067
:1099E8001205D2E7D6E902018368DB6803B198471C
:1099F80054E8003F43F00C0344E80032002AF7D152
:109A08002946404640F084FC054610B16FF0150524
:109A1800BBE7337E1BB1A36843F00803A360737EE2
:109A28001BB1636843F400436360B37E1BB1636892
:109A380043F480336360F37E1BB1636843F40033FF
:109A48006360337F002B5AD03B4B9C423CD003F1E0
:109A580080539C4238D0394B9C4235D003F1805317
:109A68009C4231D0364B9C422ED003F180539C420D
:109A78002AD0344B9C4227D003F180539C4223D0F8
:109A8800314B9C4220D0B4F1502F1DD02F4B9C421B
:109A98001AD003F180539C4216D06C4688B06A46AF
:109AA800D8F800302A49CDE905134FF40073ADF812
:109AB8001C30284B42F8103F00234FF4E2511C4859
:109AC800F9F7A2F9A546A1E7D8F804301A6893680F
:109AD80043F4804393602368727F23F0787343EAEA
:109AE800425323602368B27F23F4F81343EA024306
:109AF8002360F37F1BB1A36843F40043A36096F887
:109B080020301BB1236843F000532360236843F0DF
:109B180001032360E3699A02FCD5E3695B02FCD583
:109B28004046D9F8283098472FE700BFC12D0808CC
:109B38003C560708E12D0808003801400044004061
:109B480000480040004C00400050004000240046FF
:109B5800FC2D08080300000170B50B6806469888BC
:109B680040F0B2FC04280C46D1E91B15034610D07E
:109B780002280AD1012A01D9012D0AD8328E92B2BF
:109B880009B105B10A80022508E0032A12D9032D7C
:109B980012D9326B09B105B10A600425B5FBF3F59A
:109BA800226F2AB1954213D91649174840F0C8FCCC
:109BB800284670BD012A02D9226F012ADED896F8FC
:109BC8003020D2B201B10DB90125E9E70A70FBE7EF
:109BD800521B22677AB9A26D04F15C010832A265B2
:109BE800E26D04F15800013AE26504F1700240F0B8
:109BF80047FCE066DCE7E26E002AD9D005FB0322C9
:109C0800E266D5E7592E08080C5607082DE9F843EF
:109C180006460C4604274FF0020891F87C9023680A
:109C2800988840F051FC04280346626E17D0022839
:109C38000FD1B9F1010F02D9A16E01290FD8002A5D
:109C480039D0A16E01B1118889B2B8FBF3F531841E
:109C58000CE0B9F1030F1FD9A16E03291FD9CAB1AE
:109C6800A16E01B11168B7FBF3F53162A26E2AB19A
:109C7800AA4224D21F49204840F062FC636F5B1B54
:109C8800A9EB050515F0FF09636701D0002BC6D1C4
:109C9800BDE8F8831146E6E7B9F1010F02D9A16ED4
:109CA8000129CCD84AB1A16E01B11178C9B20125F8
:109CB80086F82010DAE71146C6E71146F6E7521B88
:109CC800A2667AB9226D04F1540108322265626DE8
:109CD80004F15000013A626504F1680240F0D0FBDB
:109CE8006066CBE7626E002AC8D005FB0322626675
:109CF800C4E700BF592E08080C56070808B502B972
:109D080033B10448044940F01BFC6FF0850008BDDE
:109D18001846FCE70C560708772E08082DE9F04787
:109D2800044600AF006940F04BFC0121606840F038
:109D380032FC002802DA10F1860F15D1656800217F
:109D48002846266940F027FC041E0BDB3248A96828
:109D580083681B685BB19847044658B12F4930485F
:109D680040F0EEFB04EAE470BD46BDE8F0876FF012
:109D78005704F3E74FF00108B5680835D6E9023211
:109D880003EBC203A5F108029342EBD955F8080C7E
:109D980041F050F9034615F8041C55F8080CBBB9F6
:109DA8006C468AB06A46006807914FF400711D4DF1
:109DB800ADF820101C49CDE9055042F8101F4FF4AA
:109DC80011511748F9F720F8A5466FF01204C9E7B2
:109DD80035F8023CD0F810E0DA0754BF43F4B0136A
:109DE80083F4D013DEF800C023F4801208FA01F9D6
:109DF800DB074CBF4CEA09032CEA0903D0F808A09A
:109E0800CEF80030DAF800309847002805F1080548
:109E1800B4DA0446A6E700BF1C510708A52E0808B7
:109E28000C560708C02E0808040000012DE9F04F61
:109E380087B080460E469B469146056900AF32B909
:109E48002BB9002630461C37BD46BDE8F08FB388D5
:109E58009A0400F123814FF0FF324FF0FF3305F1F0
:109E6800100002F0BBF86E600023C5E9113385F8D5
:109E78004C30D8F81030D8F804A0FB601B68DAF82A
:109E880000409E42B28840F01581130508D5B9F10B
:109E9800000F00F00C814FF4C121204640F0E1FA98
:109EA800B08840F011FB0346B9F1000F40F075810E
:109EB800C5F8509000226A6505F1540105F1680261
:109EC80005F15000FB6040F0DBFAFB686866BBF107
:109ED800000F40F06B81C5F858B00022EA6505F123
:109EE8005C0105F1700205F1580040F0C9FA002143
:109EF8000B46E866686D2964834240F06081002360
:109F08001A46D5F85CC0624540F0608199422CBF82
:109F180029662B66AB6E3BB92B6F2BB96B6F1BB9E0
:109F2800AB6F002B00F03F8223687B60E3683B60E7
:109F3800D8F80430BB601B68FB60FA681B68D268FD
:109F480003F4006302F4C022134340F046814946FB
:109F5800304640F0D3FA59468146304640F0CEFAB2
:109F680081454E46B8BF0646002EC0F2B580BB6894
:109F78001B6AB342C0F03B81FB68D8F810101B681D
:109F8800DB0702D5F86840F091FAFB68FA685B686D
:109F98006FF30F0333435360C1E91D66D8F80430EB
:109FA8001B681A6842F001021A60DA68500200F170
:109FB8002581D8F810603068002840F028817B6837
:109FC80003F400693B6803F4C02349EA0309AB6E54
:109FD8002BB92B6F1BB96B6F0BB9AE6F3EB329460C
:109FE800204640F00FFB636913F4787300F01C817E
:109FF8006E468AB06A46934905919349CDE906139E
:10A008004FF40073ADF82030904B42F8103F002316
:10A018004FF411518E48F8F7F7FE6369B5465A06B2
:10A0280003D5A36943F04003A3616FF00406D8F891
:10A038000430D8F810901C686369D90700F15F8173
:10A04800E3685A0240F172818249204640F047FA9B
:10A05800002800F057812368D80740F153816368CE
:10A068009BB26BB9D9F800309B88C3F34513192B01
:10A0780006D821FA03F3DB0702D5204640F016FA8A
:10A088002368E26803F4006302F4C0221343B3F5C3
:10A09800C02FDAD1204640F009FAD6E7AB69002B89
:10A0A8007FF4D9AE6B689E427FF4D5AEDCE64FF400
:10A0B800C021F2E6DAF81010C2F34513022918D0CD
:10A0C800032919D0012931D1043B1C2B8CBF002353
:10A0D8000123ABB96FF0850695F84C3013B1002E0B
:10A0E8003FF4AFAE00236B6005F1100001F03AFFBA
:10A0F800A8E6043B0C2BE9E7082B01D0102BE9D18B
:10A10800100448BFE368544842BF23F4601343F483
:10A118000023E3608368DAF80810DB685BB94F490D
:10A128004B4840F00DFA6FF00406D5E74C49484813
:10A1380040F006FACEE707F1140298470028EEDB54
:10A1480000217B69306823FA01F2824240F22D81B6
:10A1580001310929F7D16C468AB06A4607931B0A70
:10A16800089305233F49CDE9051042F8103F002325
:10A178004FF421513648F8F747FEA5463BE04FF427
:10A18800C02143E11BB1E36823F0105366E1E368A3
:10A1980023F0105343F0005360E1D9F800202A65FA
:10A1A800002A3FF487AED9F8042084E6DBF80020C3
:10A1B800AA65002A3FF491AEDBF804208EE62A6DEA
:10A1C80002EBC30252680133114495E6A86D00EB17
:10A1D800C20040680132034495E6B3F5C12F30460A
:10A1E8000CBF4946594640F089F90646BCE61E4967
:10A1F800174840F0A5F96FF015066DE71A6842F4A4
:10A2080000721A601A6891053FF5D3AEFAE7037D2C
:10A21800002B3FF4D4AE0121083040F0A9F933688F
:10A22800186940F0D8FECAE6B9F5C12F7FF4CFAE61
:10A23800AB6EDBB100212268E36800295CD102F42F
:10A248000069C0E6642F08084044080804000001BB
:10A258000C560708000202021C5107080C2F0808B8
:10A26800E42E08086F2F0808382F08082B6F002BDA
:10A27800E0D0DAF80060304640F031F901460028B5
:10A28800F9D1304640F012F92B689888C30712D4E8
:10A298000B46D5F85CC0634524D140F015F991FB15
:10A2A800F0F300FB131323BBB1FBF0F173686FF3FA
:10A2B8000F03194371604FF4C021304640F0D1F8C4
:10A2C800336843F001033360F3685A02B2D5336848
:10A2D80043F40073336033689B05ABD47369180784
:10A2E800A8D4F8E7AA6D02EBC302526801331144FF
:10A2F800D1E76FF015019EE76FF0150697E694F821
:10A30800303099E6D8F810A0DAF8003073B11A7D29
:10A3180062B1998811F4805B08D1186940F05BFE3E
:10A32800DAF800005946083040F022F963699905C7
:10A3380042BFA36943F40073A361A36943F0100308
:10A34800A361A36943F04003A361A36943F0080331
:10A35800A36163686FF30F036360D9F800309B88CB
:10A36800DA0402D4204640F0A1F899F84C3033B909
:10A37800C9F8406009F1280001F0F4FDACE6D9F80D
:10A38800443023B131464046D9F848209847D9F897
:10A3980000309B8813F400537FF49EAEC9F8043054
:10A3A80009F11000E8E71E4696E6204640F07EF8E0
:10A3B8004B4AA36852F8212023F070431343A3604B
:10A3C8009AF82530DB0703D5E36843F40043E360DC
:10A3D800B38813F0020FE36814BF43F0007323F04F
:10A3E8000073E360B38813F0040FE36814BF43F00D
:10A3F800807323F08073E360B18811F4006105D0A5
:10A40800B9F1000F3FF4BBAE4FF4C121204640F034
:10A4180028F8B38813F0100FE36814BF43F400035F
:10A4280023F40003E360A36823F48003A360B388E4
:10A43800327D03F0010322B99AF8252091077FF5B0
:10A44800A1AE33B9E368DA005EBF236843F48053F2
:10A458002360E36823F0105343F08063E360B3881C
:10A46800204913F0010FE36814BF23F4800343F479
:10A478008003E360B288A368C2F34512043A51F836
:10A48800222023F01F031343A360E368DAF81C209B
:10A4980023F00F031343E360E368DAF8182023F08E
:10A4A800F00343EA0213E360B288DAF81430C2F327
:10A4B80045120732D20893FBF2F3012BB8BF0123F0
:10A4C800FA68094982F87C30DBB2A268013B51F88E
:10A4D800233022F4F0721343A360FB681E60DFE4AC
:10A4E800A45E07085C5F07081C5F07084FF0E023BD
:10A4F80010B599691C699B6900B103600B4A0C4847
:10A508001268002908BF1146002B08BF134614F42F
:10A51800803F01D1994205D20168114401604FF092
:10A52800E021096900681044C01A10BDD03A002023
:10A53800C43A002010220B4B002083F823204FF44C
:10A54800C862094B1A604FF47A52084B1A60084BDC
:10A5580043F67F6218604FF0E0235A610722986142
:10A568001A61704700ED00E0CC3A0020D03A002094
:10A57800C43A0020684620F007018D46F1B540F046
:10A5880083F804460020FFF7B1FF1348134A036815
:10A59800D2E900515B1941F10001C2E900310027FD
:10A5A8004FF47A520E4D0760D5E900619B1BB3FB4F
:10A5B800F2F002FB00F39B1941F10001C5E90031FB
:10A5C800084B21461F6002F07BFCF9F727FCBDE829
:10A5D800F1408546704700BFC43A0020883000200B
:10A5E80080300020C83A00202DE9F341804601A8B8
:10A5F800FFF77CFF00272849284AD1E90034C3180F
:10A60800274844F100041760D0E90020B3EB020C9E
:10A61800C1E90034234E64EB0004234BBC42356887
:10A6280018681ADB4FF47A5E204B1B6813EB08039B
:10A63800A3FB0E3247EB07080EFB0822B3EB0C0313
:10A6480062EB04029842974107DAB3F1807F72F116
:10A658000002A8BF6FF07F4318464FF0E0230022A6
:10A66800306001389C6958619A61114A536803F057
:10A67800807343F000735360019BD1E90020A3422B
:10A6880038BF5B191B1B9A1840F10000C1E9002074
:10A6980002B0BDE8F08100BF88300020C43A002035
:10A6A80080300020D03A0020CC3A0020C83A002060
:10A6B80000ED00E010B5084B00201C68074B1B6834
:10A6C800E41AFFF713FF4FF47A532044B0FBF3F07A
:10A6D800034B186010BD00BF883000208030002078
:10A6E800C83A002038B53FF0CFFF064B044600209B
:10A6F8001D68FFF7FBFE84F31188BFF36F8F2844B2
:10A7080038BD00BF8830002030B53C4AD369916A13
:10A7180013F00C0305D00C2B3FD101F003010129E4
:10A728003BD19168090254BFD2F8F42092683449A9
:10A7380054BFC2F30332120F51F82200002B5AD033
:10A748002E49B7EE006A8C6A8B6A8D6AC3F30323BD
:10A758008A6B013307EE903AC2F3CC03C5F30012BB
:10A76800534306EE903A04F00304022CB8EEE77A5D
:10A77800FAEEE96A1FD0032C1DD04B6BC3F3080314
:10A7880007EE903AF8EEE77A77EEA67A06EE900AA8
:10A7980077EE867AB8EE666A1AE0D26902F00C02A1
:10A7A800042A06D0082B27D000200C2B23D1002008
:10A7B800C6E71448F9E74B6BC3F3080307EE903A72
:10A7C800F8EEE77A77EEA67A77EE867A9FED0E6A4C
:10A7D8000A4BC6EE076A5B6B67EEA67AC3F306639D
:10A7E800013307EE103AB8EEC77AC7EE876AFCEE77
:10A7F800E67A17EE900A30BD0248FCE7000C0246E4
:10A80800D05F07080024F4000024744B08B5FFF754
:10A818007BFF054B054A1B6A03F00F03D35CD84046
:10A82800034B186008BD00BF000C024652440808DC
:10A83800C8060020F7B5044610B390F895340568AB
:10A8480003F0FF021BB980F894243FF02CFF032388
:10A8580084F89534324B20689D4204BF0023A371CD
:10A8680040F035F9237C251D8DF8003095E80E0061
:10A87800206840F0E8F8014630B1022384F89534A6
:10A888000125284603B0F0BD206840F026F90028CD
:10A89800F3D101270246267904F11403C1B28E428E
:10A8A80003F1240321D800210A4604F51573C8B220
:10A8B800864203F1240326D8237C8DF8003095E8DE
:10A8C8000E00206800F00AFC05460028D5D10123B7
:10A8D800607484F89534237B012B02D1204640F024
:10A8E8009EF8206840F002FBCBE723F80A0C43E906
:10A8F800072203F8237C03F8241C03F8202C43F8D0
:10A90800142C0130CAE743E9072203F8232C03F883
:10A91800240C03F8202C43F8142C0131C7E700BF9E
:10A92800000004422DE9F04F066889B0044630461D
:10A9380040F018FB0390002840F06F81206840F039
:10A94800E3FA002800F06981D6F808382068C3F3D4
:10A958000D23C4F8D43440F0D7FA870748BF2268DB
:10A9680006F5006542BF536903F00203536120688E
:10A9780040F0CAFAC0062DD52268936923F0100367
:10A988009361D6F8208008F4F013B3F5802F08F00F
:10A998000F0740F0458147F6F07318EA030F14D00B
:10A9A800242303FB0747C8F30A194A463046D7F859
:10A9B800601240F03AFAD7F860324B44C7F8603278
:10A9C800D7F868324B44C7F868322268936943F075
:10A9D80010039361206840F097FA010300F1338176
:10A9E800206840F091FA42030CD5206840F098FAAC
:10A9F80027464FF0000A049006F5106B049B002BC5
:10AA080040F0EB81206840F07FFA002813DA6B6889
:10AA180023F001036B6094F8CC34012B40F085825D
:10AA28000021204684F8CC1440F00CF822685369C1
:10AA380003F000435361206840F066FA03050AD525
:10AA4800AB68DF0702D520463EF0A5FE22685369B1
:10AA580003F400635361206840F056FA000115D5ED
:10AA68002268536903F00063536194F8CC34002BD7
:10AA780040F05F820121236884F8CC145B6D204686
:10AA8800C3F38303C4F8D0343FF0DCFF206840F000
:10AA98003BFAC10433D56B68102123F001036B60C6
:10AAA800206840F048F84FF67F3106F510632279A8
:10AAB8000398824200F24182EB6943F00113EB6193
:10AAC800E37B002B00F05682D5F8843043F00B036B
:10AAD800C5F884306B6C43F00B036B64D6F8003810
:10AAE80004F29C4223F4FE63C6F80038A17920687A
:10AAF80000F0E4FC2268536903F480535361206832
:10AB080040F002FA820416D5206840F02FFA206837
:10AB180040F05CF8E0712768FFF778FEE2790146BB
:10AB2800384600F06BFA20463EF0FDFD2268536976
:10AB380003F400535361206840F0E6F9030707D592
:10AB480020463EF046FE2268536903F0080353612D
:10AB5800206840F0D9F9070600F11782206840F014
:10AB6800D3F9C0020CD5A046012706F5126923794E
:10AB7800BB4200F228822268536903F480135361B0
:10AB8800206840F0C1F981022AD523464FF0010C14
:10AB980006F53261207960451DD993F87C72086802
:10ABA800012F40F02682002880F22382D4F8D42492
:10ABB80082EA1040C20700F11C8283F87B72B069F8
:10ABC80040F08000B0617069000600F112826B6885
:10ABD80043F400736B602268536903F400135361F4
:10ABE800206840F091F9410007D520463EF0C7FDA6
:10ABF8002268536903F080435361206840F084F968
:10AC080042070AD523685D686B0702D520463EF0E7
:10AC1800BCFD226853682B43536009B0BDE8F08F30
:10AC2800B3F5402F7FF4D1AE0822304604F29C41A0
:10AC380040F0FBF8242303FB0747D7F86832C8F332
:10AC48000A184344BFE6206840F062F9A24600278C
:10AC5800049006F53068049B002B3FF4C1AE049BBA
:10AC6800DB0779D55FFA87FB5946206840F060F921
:10AC780010F0010F81461FD00123C8F80830206862
:10AC880094F806C000F5306303EB4713BCF1010FDD
:10AC9800016C9A6840F08B8012F0080F07D0B34817
:10ACA800814209D9120407D54FF4004203E012F09B
:10ACB800200F5AD020229A6019F0080F21D00823BB
:10ACC800C8F808302368A9491A6C03F5306303EB08
:10ACD80047138A42986804D9000444BF4FF40040DF
:10ACE800986020460592FDF759FA059A9F498A42CD
:10ACF80007D9A179012904D1206804F29C4200F007
:10AD0800DDFB19F0100F1CBF1023C8F8083019F02C
:10AD1800020F14D07369190642BF6B6843F480634D
:10AD28006B609AF85732012B06D10023594620460A
:10AD38008AF857323FF00CFD0223C8F8083019F0A2
:10AD4800200F1CBF2023C8F8083019F4005F1CBF6F
:10AD58004FF40053C8F80830049B01375B0804938C
:10AD680008F120080AF1240A75E7DFF800C26145F6
:10AD780001D9120498D41A69DAF87432C2F31202AB
:10AD88009B1ACAF868326FB9D4F864222AB901212B
:10AD980004F29C4200F092FB04E0D4F860221A44CA
:10ADA800C4F8602259462046FDF7BEF984E7DFF86B
:10ADB800C0C1614507D111043FF576AF9206F1D5C0
:10ADC80020229A60EEE7002FECD1D4F86432002BF1
:10ADD800E8D1394604F29C42DCE7049BDA0740F1EB
:10ADE8009B805FFA8AF319462068079340F0A9F818
:10ADF80010F0010F804620D001216B6B0AF00F0282
:10AE080001FA02F223EA02036B63CBF80810A17976
:10AE180001290DD1D7E9072313443B62BAF1000F8A
:10AE280006D1636A23B9206804F29C4200F046FB0D
:10AE380020465FFA8AF1FDF795F918F0080F1CBF54
:10AE48000823CBF8083018F0100F1CBF1023CBF8DC
:10AE5800083018F0400F1CBF4023CBF8083018F01A
:10AE6800020F10D0514630463FF065FEFB7D012BA6
:10AE780006D100232046FB755FFA8AF13FF069FC92
:10AE88000223CBF8083018F0800F45D0D7E90932F3
:10AE98009A4241D8A3EB0208FB692168984528BF6C
:10AEA800984601F5106308F1030803EB4A1305916E
:10AEB8004FEA98080693069B9969D7E9093289B23F
:10AEC800414527D393420BD80121059B0AF00F0077
:10AED800D3F83428814022EA0102C3F834281BE061
:10AEE800A3EB0209FB69079A994528BF9946A379FC
:10AEF80005980093396A1FFA89F33FF083FF3B6A8C
:10AF080009F103084B443B62BB6A4FEA98084B447B
:10AF1800BB62D0E79342D7D9049B0AF1010A5B08C8
:10AF2800049324370BF1200B68E520463EF042FCE1
:10AF38007CE520463EF02FFCA8E599601A6820338E
:10AF480022F4001243F8202CC3F8E811D3F8E021CA
:10AF580022F40012C3F8E021D3F8E02142F00062A5
:10AF6800C3F8E021039A01320392A0E50A30544F56
:10AF78000A31544F6B6943F4005343F02B036B6160
:10AF88002B6943F00B032B61A8E501222427B36941
:10AF980004F2572023F08003B36106F53263217968
:10AFA80091427FF6DBAD07FB02F1415C012907D135
:10AFB800196841F000611960196841F08041196011
:10AFC80001322033EBE798F83C30D9F80020012B08
:10AFD80009D1002A07DA67F07F01204688F83B305C
:10AFE800C9B23FF0CCFC013708F1240809F1200967
:10AFF800BDE50CF1010C24332031CBE5022A4AD1FE
:10B00800274B284A0B44934239D9274B274A0B44EC
:10B01800934236D9264AA1F57403A3F510539342F7
:10B0280031D9244AA1F18373A3F5E74393422CD382
:10B03800214B224A0B44934229D9214B214A0B44E4
:10B04800934226D3204B214A0B44934223D3204AD0
:10B05800A1F1B773A3F5585393421ED31D4B1E4A53
:10B068000B4493422CBF06230723C26822F4705274
:10B07800C260C26842EA8323C360002070470F237E
:10B08800F3E70E23F1E70D23EFE70C23EDE70B239E
:10B09800EBE70A23E9E70923E7E70823E5E700BF29
:10B0A800405327FFFF340C00401E1BFF3F420F0098
:10B0B8007F4F120020D6130060B6E5FE5FE316004E
:10B0C80000D3CEFE40771B00C05BB3FEC0912100C9
:10B0D80020753800E05459FEE09C410084B02DE909
:10B0E800F843044609A880E80E00002319469DF895
:10B0F80024809DF82E7003F14002013304EB820294
:10B108000F2B5160F7D104F50066002F64D17368E6
:10B1180043F002037360A36B23F40013A363236853
:10B1280043F040032360236843F080032360002535
:10B1380003212046C4F8005E3FF041FD102120465F
:10B148003FF0F9FC014620463FF018FD0843C0B225
:10B15800401B18BF01202A464FF090414FF0006C69
:10B168004FF67F3E356104F510637561F561A845BA
:10B1780037D800224FF0904511464FF0006C4FF63B
:10B188007F3E04F5306390453DD8336923F48073DE
:10B1980033610023A3616FF0804363619DF826301B
:10B1A8001BB9A36943F01003A361A2691F4B1343A2
:10B1B800A3619DF82A301BB1A36943F00803A3617A
:10B1C800012F01BFA36943F0804343F00403A36147
:10B1D800BDE8F84304B07047A36B43F40013A363BE
:10B1E800A5E7D3F80090B9F1000F0ADA3DB9C3F822
:10B1F80000C01A610135C3F808E02033B7E71960C9
:10B20800F7E71A60F5E7D3F80090B9F1000F0ADA0A
:10B218003AB9C3F800C019610132C3F808E0203315
:10B22800B1E71D60F7E71960F5E700BF00383C801B
:10B2380030B54A780B78012A00EB431300F500601B
:10B2480029D1D3F80029002A0BDAD3F8002942F0D3
:10B258000062C3F80029D3F8002942F08042C3F8FD
:10B26800002901240A78C56B02F00F0204FA02F2E1
:10B2780025EA0202C2630978C26901F00F018C4015
:10B2880022EA0402C261D3F80019174A0A40C3F837
:10B298000029002030BDD3F8002B002A0BDAD3F8A0
:10B2A800002B42F00062C3F8002BD3F8002B42F0C9
:10B2B8008042C3F8002B01240A78C56B02F00F0204
:10B2C80004FA02F225EA0242C2630978C26901F06F
:10B2D8000F018C4022EA0442C261D3F8001B034AE2
:10B2E8000A40C3F8002BD4E7007833EC0078F3EF7A
:10B2F800F7B54B7891F800C0012B6D4D6D4E00EB02
:10B308004C1440F089800F6904F510633FBB1F6936
:10B318003D401D611D6945F400251D611D693540CD
:10B32800012A1D614DD1CA6902B15A610B79012BFD
:10B338000CD1D0F8083813F4807FD4F800390CBF4A
:10B3480043F0005343F08053C4F80039D4F800396F
:10B3580043F00443C4F80039002003B0F0BD1F696E
:10B368003E401E611E6935401D610D698E68BCF145
:10B37800000F0CD1B54288BF0E611D6945F4002548
:10B388001D610D691E69C5F312053543C8E73544CB
:10B39800013DB5FBF6F5484FD3F810C0AEB207EA49
:10B3A800C54545EA0C051D610D79012DE9D11D69D9
:10B3B80025F0C0451D611F69750705F0C0453D436F
:10B3C800DEE7D4F8003943F00443C4F800390B79B8
:10B3D800012B0DD00B69002BBED001230A78D0F8C1
:10B3E800344802F00F0293402343C0F83438B3E7DF
:10B3F800D0F8083813F4807FD4F800390CBF43F034
:10B40800005343F08053C4F8003900920B8A0A783D
:10B41800C9683FF0F7FC9FE7D4F8107B04F5306368
:10B428003E401E611E6935401D610E698D68BCF184
:10B43800000F27D106B10D610D621E69C5F3120513
:10B4480035431D611D6945F40025012A1D6102D19E
:10B45800CA6802B15A610B79012B0CD1D0F80838AF
:10B4680013F4807FD4F8003B0CBF43F0005343F043
:10B478008053C4F8003BD4F8003B43F00443C4F8BD
:10B48800003B69E7002ED8D02E44013EB6FBF5F606
:10B49800B6B275430D62084D1F6905EAC6453D43BE
:10B4A8001D610D6A1E69C5F312053543CDE700BF5E
:10B4B800FFFF07E00000F8FF0000F81F30B5114C4F
:10B4C800056C00F53063A54203D9D0F8004B002C79
:10B4D80016DB00241C611C69012944F400241C614A
:10B4E8001C6944F018041C611C6944F0C0441C61C8
:10B4F80001BF5A61D0F8003B43F08023C0F8003BFD
:10B50800002030BD0A30544FA8B1304BDA6802F43D
:10B518004032B2F5403F10D12D4B984250D92D4BB7
:10B5280098424FD92C4B984235D92C4B984216D972
:10B538002B4B984231D901207047DA6802F4403227
:10B54800B2F5003F0DD1274B984239D9264B984286
:10B5580038D9264B98421ED9254B9842EBD803235D
:10B568001CE0DB6803F44033B3F5803F0AD1214B7C
:10B57800984225D91B4B984224D91F4B98420AD987
:10B58800194BEAE71D4B98421AD91D4B984219D915
:10B598001C4B9842CFD8022300E004231A490A68BA
:10B5A80022F00F021A430A600A6802F00F0293425F
:10B5B8000AD0086800F00F00C01A18BF01207047B1
:10B5C8000023EBE70123E9E7002070470008024663
:10B5D8000048E8010090D00300D8B8050020A10772
:10B5E8000068890940787D0180F0FA02C068780413
:10B5F80000E1F50520BCBE0060343C0200127A0070
:10B608000024F40000366E01002002400F4BF0B514
:10B618001F6800230E4D9F4202D16FF0150011E004
:10B6280015F8016BB0EB461F4FEA46140BD304F133
:10B638002006B04207D2041B0020064D55F82330DF
:10B648000B601470F0BD0133E5E700BF086C070814
:10B658006B4408080C6C07084FF6FF73984237B51F
:10B6680017D00DF1030201A9FFF7D0FF034680B9F7
:10B6780001999DF80340084A507928B115688D4210
:10B6880002D11579A54205D00133202B02F1080219
:10B69800F2D1002003B030BDD43A00204FF6FF733A
:10B6A800984270B504460E46154607D102211D4A38
:10B6B8001D483BF0A5FF6FF015000AE0FFF7CCFF2F
:10B6C80040B1194823460221184A3BF0A2FF6FF007
:10B6D8000F0070BD2A4631462046FFF797FF30B16C
:10B6E80002212346124A10483BF093FFE3E7034642
:10B6F800104911F83340DA0054B10133202BF8D146
:10B70800094802210C4A3BF084FF6FF00B00E0E788
:10B7180034680A4941F833402B7811440B710123EE
:10B728004B71D6E7B52F0808B4550708D82F080875
:10B7380006300808D93A002033300808D43A0020E7
:10B74800F8B51B4B0D460446002219465E793EB3F8
:10B758001868A04224D11879A84221D101EBC2036C
:10B7680000225A7101232069AB400168D4F808C04F
:10B7780021EA03010160DF4329462046DCF8003056
:10B78800984786300AD12269A168136820463B4051
:10B7980013600B684FF48032294698473046F8BD4D
:10B7A8000132202A03F10803D0D10026F6E700BFB2
:10B7B800D43A002010B50446F7F758FA0348012197
:10B7C800034A3BF01DFF20463FF03FFCEC550708BD
:10B7D800693008082DE9F84304460D4600AFEFF339
:10B7E8001188102383F31288BFF36F8F04282A4A25
:10B7F80098BF2A4BE9468AB09668117C98BF53F8DF
:10B8080020306A4688BF264BCDE9073140F2013324
:10B818002448ADF82430244BCDE9050442F8103F04
:10B8280000234FF431512148F7F7EEFACD4645B1E0
:10B83800EB69C3F3080323B101211D4A1B483BF000
:10B84800DFFE2EB130463FF0AFFE08B1037803B9F2
:10B858001848E9468AB06A46174B0790CDE905367D
:10B8680040F20133ADF82030144B42F8103F00236A
:10B878004FF411510D48F7F7C7FA2946CD4620462F
:10B88800FFF798FF88F31188BFF36F8F3046F8F7FA
:10B89800D5FABD46BDE8F883D43B00201060070800
:10B8A800793008088F30080805000001EC550708B2
:10B8B800B730080887300808D830080804000001A5
:10B8C80038B50A4B53F82040013053F82050A542B0
:10B8D80000D838BD606830B1037EDB0701D43FF083
:10B8E80088FB0834F3E723689847FAE724600708D9
:10B8F800012270B52C4B2D4C2D4D86B01A70AC42E0
:10B908001CD30320FFF7DCFF0420FFF7D9FF294CE5
:10B91800294D2646AE4204F1300413D301F0D4F881
:10B92800244CAC422AD301F0E3F83AF060FD234AF4
:10B93800938923F00103938106B070BD54F8043B4A
:10B948009847DCE754F80C3C059354F8103C0493F2
:10B9580054F8143C039354F8183C029354F81C3CD4
:10B96800019354F8203C009354E90A2354E90C014C
:10B97800F5F746FC54F8303C5E65CAE7D4E90A237B
:10B98800B3F1FF3F08BFB2F1FF3F05D052EA030110
:10B99800206803D100F078FD3034C2E70849183038
:10B9A80001F0A6F9F8E700BF32490020C0530708A4
:10B9B800C4530708C8530708F85307087031002014
:10B9C800CFB60508E02370B5134E012203FB0066CD
:10B9D800002386B0CDE904230F220193CDE902327A
:10B9E80018234FF4A0720D4D0D4903FB0055044672
:10B9F80002FB00110B4B30460095F5F701FC337C38
:10BA08002C7423F004033374074B013403EBC42371
:10BA1800EE606B6006B070BD90300020D43B002013
:10BA280030670020E5B10508305F00207FB50020B1
:10BA3800FFF746FF2D4B03F5006282F3088883F376
:10BA48000A88F0232A4C2B4D84F822300023E37710
:10BA580023766376A37684F82030636A43F4E02380
:10BA68006362F8F795F8F8F7D3F94FF0FF33A3625C
:10BA7800E362F8F7EBFBF8F76DFAF7F759F81E48A9
:10BA880000F0DEFCF6F70AFF1C4CAC422AD301207A
:10BA9800FFF716FF02201A4CFFF712FF01F00CF80F
:10BAA800184B00259C61184B45F6E062059301236D
:10BAB8001649CDE903532046154BCDE901550095AC
:10BAC800F5F79EFB0646237C204623F004032374E7
:10BAD8003FF09FFD2846FFF775FF314620460C4A88
:10BAE800F8F768F954F8043B9847CEE7305F002030
:10BAF80000ED00E0C053070850320020BC5307088F
:10BB080070310020D43B0020F4130808706800202E
:10BB1800F9B8010838B5064C064DAC4201D30020EF
:10BB280038BD2046D4E901123FF0D9FA1434F4E7BD
:10BB3800B4100020C810002030B5054B85B0DDE9F1
:10BB480008450293CDE900453FF087FA05B030BDBE
:10BB58006367050838B5064C064DAC4200D338BDBE
:10BB680020463FF0E1FA0028F9D11C34F5E700BF80
:10BB780098100020B410002073B50C46EFF3118123
:10BB8800102585F31288BFF36F8FC5685DB12560F6
:10BB98002B68C360836901338361002081F31188B6
:10BBA800BFF36F8F11E052EA030603D16FF00B0069
:10BBB8002560F3E7CDE900230246083000F088FE4F
:10BBC80018B9034B9B685B69236002B070BD00BF66
:10BBD800D43B0020F7B50E4604469DF82010EFF33D
:10BBE8001187102080F31288BFF36F8F256AE068F1
:10BBF800854245D22568AC4219D0C5B128463FF0E8
:10BC0800F8FA05F1180001F003F93146A2686869ED
:10BC180058F01FFF00232846C5F8983000F0D4FCE0
:10BC280004F10800394600F0DBFD002036E0A26888
:10BC3800D9B13146E06958F00CFFE369A2681344B2
:10BC48006269E361934201D12369E361236A1021A8
:10BC58000133236204F124003FF09CFE0028DFD169
:10BC680087F31188BFF36F8F18E0A0692369314605
:10BC7800984208BF6069801AA06158F0EAFEE5E7BB
:10BC880052EA03010CD0084904F1080089684E61A2
:10BC9800CDE900233946224600F01AFE03B0F0BD74
:10BCA8006FF02200DCE700BFD43B0020F7B5044664
:10BCB8000846EFF31186102181F31288BFF36F8FC6
:10BCC800216A00293BD0A268A16958F0C2FEA36985
:10BCD800A268256813446269A361934204BF23697B
:10BCE800A361236AAC4203F1FF33236236D02846AE
:10BCF800002D34D000273FF07CFA05F1180001F040
:10BD080087F86969A268E06958F0A3FEE369A26848
:10BD1800284613446269E361934204BF2369E361DF
:10BD2800236A01332362C5F8987000F04DFC04F1D2
:10BD38000800314600F054FD384603B0F0BD52EA21
:10BD4800030111D00A4989684861CDE900233146C9
:10BD5800224604F1080000F0BBFDEEE7002086F360
:10BD68001188BFF36F8FE8E76FF02200F7E700BF95
:10BD7800D43B00202DE9F341044617461E46EFF355
:10BD88001188102383F31288BFF36F8F304BC2687A
:10BD98009B6872B18068984217D057EA060216D19C
:10BDA80088F31188BFF36F8F6FF00F0002B0BDE802
:10BDB800F08193F90E1001322161C4E9023288F34F
:10BDC8001188BFF36F8F0020F0E72169F3E793F93B
:10BDD8000E1090F90E30994230DA9942A8BF1946F0
:10BDE8003FF05FFA054622464146CDE900761948FC
:10BDF80000F06EFD0028E6D0EFF31186102383F3E0
:10BE08001288BFF36F8FA068D0B1236821699C4264
:10BE18000AD04BB193F90E309942A8BF19466FF07A
:10BE28007F039942B8BF19463FF03BFA40B131460B
:10BE3800084800F0D5FC6FF00A00B7E70025D2E704
:10BE4800002DF4D186F31188BFF36F8FF3E700BF9D
:10BE5800D43B002033490020F8B583680546002B01
:10BE680040D0234A926893423FD1C368012B03D93B
:10BE7800013BC3600020F8BDEFF31187102383F363
:10BE88001288BFF36F8F016980683FF00AFA2C6847
:10BE9800A54207D10023C5E9023387F31188BFF310
:10BEA8006F8FE7E7002CF5D0D4E900320026136045
:10BEB8005A60237CC4E9006623F002032374A66059
:10BEC80004F1180000F0A4FFAC6094F90E3020468D
:10BED8002B61C4F8986000F077FB3946054800F0FC
:10BEE8007FFCC7E76FF01500C5E74FF0FF30C2E7EA
:10BEF800D43B00203349002073B51546EFF3118673
:10BF0800102282F31288BFF36F8F0468B4B12368DC
:10BF1800426823F00303944208BF43600360236828
:10BF28009B0704D0656820463FF060FD2C4686F3E9
:10BF38001188BFF36F8F204602B070BD55EA030227
:10BF4800F5D000F1080231461046CDE9005300F063
:10BF5800BFFC0028EFD1024B9B685C69EBE700BF90
:10BF6800D43B002070B5EFF31186102383F31288B9
:10BF7800BFF36F8F0468A0421CD0DCB1D4E9003253
:10BF8800002513605A60237CC4E9005523F002039E
:10BF98002374A56004F1180000F03AFF2046C4F8A5
:10BFA8009850656100F010FB3146BDE870400A48C2
:10BFB80000F016BCD0E902329A4218BF01330221C0
:10BFC800836010303FF0E6FC0028EDD186F311883D
:10BFD800BFF36F8F70BD00BF3349002013B5EFF377
:10BFE8001181102484F31288BFF36F8F846844B1E1
:10BFF800013C846081F31188BFF36F8F002002B089
:10C0080010BD52EA030406D181F31188BFF36F8F84
:10C018006FF00F00F3E7CDE900230246014800F076
:10C0280057FCECE733490020F8B50546EFF31187D4
:10C03800102383F31288BFF36F8F00262C68A54264
:10C048001AD0CCB1D4E90032002613605A60237CA0
:10C05800C4E9006623F002032374A66004F1180003
:10C0680000F0D6FE6FF00A0366612046C4F89830E7
:10C0780000F0AAFA0126E1E700230221AB6005F1EE
:10C0880010003FF087FC28B926B987F31188BFF361
:10C098006F8FF8BD3946BDE8F840014800F0A0BBF5
:10C0A800334900202DE9F04F04464FF0FF3A4FF096
:10C0B800FF3B614E85B0EFF31187102383F312889D
:10C0C800BFF36F8FD4F8E4505DBB022104F1FC008C
:10C0D8003FF0C1F900287FD004F1F409D4F8F450F6
:10C0E8004D4500F08680002D00F08380D5E90032B0
:10C0F8004FF0000813605A602B7CC5E9008823F0D4
:10C1080002032B74C5F8088005F1180000F080FEC2
:10C1180001232846C5F89830C5F8148000F054FA71
:10C12800DCE7D4F8E8202B689542C4F8E43008BF6F
:10C13800C4F8E830D4F8FC3043F00203C4F8FC300B
:10C14800EB6823F0040343F00103EB606B6887F3AB
:10C158001188BFF36F8F28469847EFF31187102394
:10C1680083F31288BFF36F8FEB68D80623F00102C0
:10C178004AD4EA60EB689A0717D5306823F00203BF
:10C18800EB6090B10022036878B141688D4249D1D3
:10C198000368002A40D172683360904200D173600E
:10C1A800002340F8083BFFF7DDFED4F8FC3023F00D
:10C1B8000203C4F8FC30DB053CD4D4F8E430003B7F
:10C1C80018BF012387F31188BFF36F8F002B3FF44B
:10C1D80072AF3FF00AFA6EE7D4F8FC30D90608D5FA
:10C1E800C4F8FC0087F31188BFF36F8F05B0BDE872
:10C1F800F08F00233946CDE900AB029304F1EC023D
:10C208000E4800F08BFC56E723F01103EB6005F1B4
:10C218001000FFF7A7FEADE713607368984208BFE8
:10C228007260BDE702461BB1196818460B46ABE7BA
:10C238001946FAE70023C5E7FC3B002033490020F4
:10C24800F8B5C36804469A070E46C3F3400542D4BE
:10C258005F0742D40B680BB983680B60E368D807A3
:10C2680042BFA36802253360376858BF012557B31A
:10C278001B4B9A68D7F8E0309A421ED13FF08BF9F1
:10C2880080F00100C0B2D7F8FC30D907C3F38002B0
:10C298001CD5F2B1F8B100232360D7F8E83073B9A0
:10C2A800C7E9394438463FF000F9E36843F004032E
:10C2B800E3603368A3602846F8BD0020E3E71C600C
:10C2C800C7F8E840EEE76FF0150506E06FF01205D5
:10C2D80003E01B07DFD56FF00F0500233360EAE7A3
:10C2E800D43B0020014601483FF039B950330020C3
:10C2F800F0B50446002089B00E9DC4E9390004F168
:10C30800EC00C4E93B0004F1F400C4E93D0055B376
:10C318002879002840F2011008BF0120C4F8FC0069
:10C3280000204FF0FF364FF0FF37CDE90330CDE95D
:10C338000100CDE9066720460C4B009400F0C8F8D0
:10C3480055B1296811B120463FF02BF96B791BB123
:10C35800A38943F00103A381204600F095F8C4F8AF
:10C36800E04009B0F0BD0120D8E700BFADC001082A
:10C3780037B501900846EFF31184102181F3128834
:10C38800BFF36F8FC16811F01E0F16D153EA020573
:10C3980008D101A9FFF754FF84F31188BFF36F8F09
:10C3A80003B030BD41F00801C160019910308161CE
:10C3B800034900F09DFC0120EEE70020ECE700BFF8
:10C3C800F3B4050801460148FFF7D2BF50330020F7
:10C3D800F0B585B00C4617461D460190EFF3118362
:10C3E800102181F31288BFF36F8F204603A90393AE
:10C3F8003FF03CF855EA0703039E09D1204601A9FE
:10C40800FFF71EFF86F31188BFF36F8F05B0F0BDED
:10C41800E3683A4643F00803E360019B0449A362DA
:10C4280004F110002B4600F063FC0120EAE700BF8E
:10C43800F3B4050801460148FFF7CABF503300208E
:10C448000123037483810023C0E92033C0F88C30B2
:10C45800014B9860704700BFD43B002008B500F03E
:10C4680069FA70B1074B9B68DB7B53B9EFF3118016
:10C47800102383F31288BFF36F8FBDE8084000F0E4
:10C48800C5BA08BDD43B002038B50446EFF3118582
:10C49800102383F31288BFF36F8F037C5B070FD5DC
:10C4A800183000F0B5FC237C204623F004032374E5
:10C4B80000F08AF82946BDE83840044800F090B9F1
:10C4C80085F31188BFF36F8F38BD00BF3349002053
:10C4D800F0B5002587B00595109DDDE91276049525
:10C4E8000F9D044603950E9D02950D9D01950C9D8B
:10C4F8000095F4F785FEB6F1FF3F08BFB7F1FF3F9F
:10C5080005D056EA070305D12046FFF7BDFF2046B0
:10C5180007B0F0BD3A46334604F11800014900F06F
:10C52800E7FBF4E7CFB605086FF00A01094A9368FC
:10C53800C3F898100849C3F894004B6843F0805337
:10C548004B60002383F31188BFF36F8F9368D3F890
:10C5580098007047D43B002000ED00E038B5184C37
:10C56800A168206A0B68814214BF1A4600224968F4
:10C578000B605960A368216A2AB9124AC3E90021ED
:10C588000B6023620AE092F90E5093F90E0085427F
:10C5980012DD5168C3E900210B605360E569094B5E
:10C5A8009D4200D005B9E568A3689D4202D028469F
:10C5B8003FF046F9A56138BD8A42DED01268DBE754
:10C5C800D43B0020F03B002070B590F91020037C8C
:10C5D800002A2FDBD9062DD11A4C63F07F0322469F
:10C5E800037452F81C3F216A934207D1C0E9002125
:10C5F800086020620FE09942F8D01B68002BF5D044
:10C6080093F90E6090F90E50AE42F4DD5968C0E916
:10C61800003108605860E569954200D005B9E568C1
:10C62800A3681A7CD20606D1DA897F2A03D9AA69B7
:10C638000AB9A36170BDAB4202D028463FF000F9A9
:10C64800A561F7E7D43B002038B590F910200146E2
:10C65800002A037C04DA03F07F0303743EF0C7FF6B
:10C668000D4D2A4652F81C4FAB68944200D004B9CD
:10C67800EC688B4207D01A7CD20604D1DA897F2A6B
:10C6880001D9A2692AB1A34202D020463FF0D8F8C6
:10C698002346AB6138BD00BFD43B0020002A2DE9FA
:10C6A800F8430CBF4FF010084FF00808027C04460E
:10C6B80018EA020F0D4665D148EA0203D2090CD1E7
:10C6C8000374B8F1080F7ED1A36813B120463EF079
:10C6D80096FF102704F118060FE003F07F03037498
:10C6E8003EF085FFEDE785F31188BFF36F8FEFF319
:10C6F800118587F31288BFF36F8F304600F088FBEF
:10C708000B30F0D0A66D04F15807B74211D04FF0A6
:10C71800000976B130463EF072FFC6F8989006F1EF
:10C72800180000F075FB3046FFF74EFFA66DB742C4
:10C73800EFD1294B9B689C4245D1EFF30587003F19
:10C7480018BF0127DFF890904B4653F81C6F9E42A4
:10C7580000D00EB9D9F80C60D9F80830B34202D02D
:10C7680030463FF06DF8B8F1100FC9F8186009D0DD
:10C7780020463BF0F1F8204600F066FA17B117485A
:10C78800FFF75EFE144B9B68A3421ED1EFF30583AF
:10C79800DBB9A289D20711D585F31188BFF36F8F52
:10C7A80083F31188BFF36F8F0423184602DFEFF37A
:10C7B8001185102383F31288BFF36F8F2846BDE8D5
:10C7C800F843FFF7B1BE0027BCE785F31188BFF334
:10C7D8006F8FBDE8F88300BFD43B002050320020A3
:10C7E80049B9EFF3058030B9054B9A699B689A42BD
:10C7F80001D0FFF799BE81F31188BFF36F8F70479F
:10C80800D43B002070B50F4D06462B4653F81C4FFD
:10C818009C4200D004B9EC68AB681A7CD20604D1FB
:10C82800DA897F2A01D9A2692AB1A34202D0204617
:10C838003FF006F82346AB613146BDE87040024838
:10C84800FFF7CEBFD43B00203349002070B5EFF38B
:10C858001186102383F31288BFF36F8F1A4CA168D7
:10C86800206A0B68814214BF1A46002249680B608F
:10C878005960A368216A2AB9144AC3E900210B60E8
:10C8880023620AE092F90E5093F90E00854216DDF4
:10C898005168C3E900210B605360E5690B4B9D4269
:10C8A80000D005B9E568A3689D4202D028463EF04D
:10C8B800C7FFA5613046BDE87040FFF735BE8A4224
:10C8C800DAD01268D7E700BFD43B0020F03B002045
:10C8D800F8B5DDE906670C461146EFF305833BB171
:10C8E800002383F31188BFF36F8F0423184602DFF8
:10C8F8000D4B0E4A98681060EFF31182102282F3F4
:10C908001288BFF36F8F9D6828463EF091FE32462D
:10C918003B4605F11800064900F0EAF92046BDE853
:10C92800F840FFF701BE00BFD43B0020043C0020C4
:10C93800CFB60508F8B50446EFF31187102383F343
:10C948001288BFF36F8F037C49B203F01F02002ADD
:10C958000CBF0126002635D103F07F032A4D03744E
:10C968003EF045FE2A46037C817363F07F0303741F
:10C9780052F81C3F286A934207D1C4E9002004609A
:10C988002C620DE09842F8D01B68002BF5D093F983
:10C998000EC08C45F6DD5968C4E900310C605C6056
:10C9A800EC69944200D004B9EC68AB689C4202D0B0
:10C9B80020463EF045FFAC6187F31188BFF36F8FC7
:10C9C8003046F8BD9B071CD585683EF010FE817384
:10C9D8002B689D4209D16B68C4E900531C606C60E8
:10C9E800EAE76A689A42F6D01B68002BF3D093F9FD
:10C9F8000E208A42F5DD5A68C4E9003214605C6092
:10CA0800DAE78173D8E700BFD43B0020034648B972
:10CA1800EFF3058232B9064A91699268914201D0D2
:10CA2800FFF782BD83F31188BFF36F8F704700BF94
:10CA3800D43B0020F8B550EA010305460C4603D163
:10CA48003EF0D3FD0020F8BDEFF31187102383F3E8
:10CA58001288BFF36F8F144E144BB0681860FFF73D
:10CA6800F3FDB0682A4623461149183000F040F912
:10CA7800B36804461A7CC3F8947042F004021A742E
:10CA88006FF00A02C3F898200A4A536843F08053AB
:10CA98005360002383F31188BFF36F8F3EF0D7FEF6
:10CAA800201A20EAE070CEE7D43B0020043C0020A6
:10CAB800CFB6050800ED00E0024B03F11C02C3E904
:10CAC80007227047D43B0020EFF31181102383F332
:10CAD8001288BFF36F8F054B9A68D37B013BD373E2
:10CAE80081F31188BFF36F8F704700BFD43B0020DC
:10CAF800EFF31180102383F31288BFF36F8F034B7A
:10CB08009A68D37B0133D373FFF77CBED43B0020F4
:10CB1800014B9868704700BFD43B0020D3B5DDE9CE
:10CB28000667089CCDE90067FFF7D2FE1CB1034BEE
:10CB38009B685B69236002B0D0BD00BFD43B002076
:10CB4800027C034612F01F0210D10A4988420DD018
:10CB58000949086868B1D9897F2909D893F90E204D
:10CB6800064B1B689A42B8BF0020704700207047E8
:10CB78001046704790300020CC060020083C00206A
:10CB88000122044BC01A044BC0105843034B1A54DB
:10CB9800704700BF30330020ABAAAAAA334900204F
:10CBA800F8B50B4B04461E7C18230A4D0A4F03FBAD
:10CBB8000655284600F02CF934B1BB5D2846E21A28
:10CBC8000649D31700F094F80023BB55F8BD00BF01
:10CBD800D43B0020303300203349002089CB0108A2
:10CBE800F8B5EFF31187102383F31288BFF36F8F23
:10CBF800124E134BB5681868A84206D13EF020FEC5
:10CC080087F31188BFF36F8FF8BD00221A60337C59
:10CC18000C4AD35C002BF3D02846FFF791FF04465B
:10CC28000028EDD02B7CDB06EAD1FFF797FCB3692F
:10CC3800AB42E5D12046FFF7B3FFE1E7D43B002044
:10CC4800043C002033490020EFF31181102383F3C3
:10CC58001288BFF36F8F0A4A536A834207D1DB6F8A
:10CC6800536281F31188BFF36F8F70471346002B0F
:10CC7800F7D0DA6F8242F9D1C26FDA67F1E700BF05
:10CC8800D43B0020024B1868984208BF0020704728
:10CC9800D006002008B50246FFF7F4FF6FF0004108
:10CCA800C8B18A4215D2D0E90230B0F1FF3F08BFBF
:10CCB800B3F1FF3F03D16FF00040801A08BD8B42EB
:10CCC80070F1000001DB0548F7E79A4201D2981A93
:10CCD800F4E70020F2E78A42EDD3EFE7FEFFFF7F9B
:10CCE800024B186808B1FDF7E5BC7047D80600206C
:10CCF800B3F1FF3F08BFB2F1FF3F2DE9F84F0446FB
:10CD08009A461546984679D00161EFF311871023AA
:10CD180083F31288BFF36F8FBAF1000FDFF8E89042
:10CD280023DBFFF7DDFF374B06461A68003A18BFCA
:10CD3800012245194AF10003521943F10003D9E9C8
:10CD48000051551943EB01080121DFF8C090C4E9EF
:10CD58000223FFF797FFD9F804A0D0B9C4E9009AD5
:10CD6800CAF80040C9F8044025E06FF00102D9E98B
:10CD78000013521A4FF0FF3161EB0303521B63EBB0
:10CD88000A03012A73F10001BCBF0122002300211C
:10CD9800DBE7D0E9022ED4E9023C93427CEB0E0B90
:10CDA80023DAD21A6EEB0C03C0E902234368C4E904
:10CDB80000031C604460FFF765FF84420DD1114BEE
:10CDC8001B68013309D111B9FFF78AFF06463046BF
:10CDD800FFF760FF0021FDF707FC87F31188BFF319
:10CDE8006F8F28464146BDE8F88F9B1A6CEB0E0200
:10CDF8005045C4E90232B1D00068AEE70025A84624
:10CE0800EFE700BFD806002048330020D0060020F6
:10CE1800F8B50446EFF31186102383F31288BFF3A5
:10CE28006F8F026872B3FFF72DFF184B5B689C4247
:10CE380008D0D2E90231D4E90275DB1941EB0501CA
:10CE4800C2E90231D4E900320025844213605A60F5
:10CE5800C4E900550ED000200D4A136823F00101E3
:10CE68008C4204BF43F00103136086F31188BFF3BB
:10CE78006F8FF8BDFFF734FFFFF70CFF2946FDF76A
:10CE8800B3FBE8E76FF01500E6E700BFD006002027
:10CE98000C3C0020EFF31182102383F31288BFF3B8
:10CEA8006F8F064B40F001001B681B1A584258410F
:10CEB80082F31188BFF36F8F704700BF0C3C0020CE
:10CEC80000232DE9F0470C46334E344DDFF8D4905B
:10CED800334F30602B60D6F80080B8F1000F10D1C6
:10CEE8004FF0FF3340462B60FFF7D4FE4146FDF775
:10CEF8007BFB84F31188BFF36F8FBDE8F047FFF722
:10CF08006FBEFFF7BFFE6FF0004330B1D0E90212E9
:10CF1800994272F10002B8BF0B464345194684BFD7
:10CF2800434641464FEAE37C38B18268B2EB030AD4
:10CF3800C26862EB0C0EC0E902AEA8EB01014FF02B
:10CF4800000A4FF01008D9F800203160D218D9F83B
:10CF5800043043EB0C03C9E90023FFF793FE0028D4
:10CF6800B9D0D0E902120A43B5D1D0E900210A604C
:10CF780051600269C0E900AA386084F31188BFF3E0
:10CF88006F8F9047EFF3118488F31288BFF36F8F88
:10CF9800C7F800A0E1E700BF103C0020D806002039
:10CFA8000C3C00204833002010B5EFF31184102307
:10CFB80083F31288BFF36F8FFFF792FE054AD2E919
:10CFC8000031C01841F1000184F31188BFF36F8F5D
:10CFD80010BD00BF483300202DE9F0410446EFF3AF
:10CFE8001186102383F31288BFF36F8F03682BB168
:10CFF80086F31188BFF36F8FBDE8F081FFF74AFF12
:10D0080007460028F4D1D4E90A586A1C48F10003FD
:10D01800022A73F1000324D33EF01DFC281848EBC4
:10D028000101012871F1000142DB3EF014FC6FF0B0
:10D038000203281848EB010183426FF000438B413B
:10D048003BDB3EF008FC6FF001022D1848EB0103B2
:10D058004FF0FF31521B61EB030320461949FFF7DC
:10D0680047FE236B01332363236A63B186F3118878
:10D07800BFF36F8F20469847EFF31186102383F391
:10D088001288BFF36F8F54F8185FA542B0D0002DF7
:10D09800AED028463EF0F2FA0023C5F8983086F361
:10D0A8001188BFF36F8F2846BDE8F0413EF0B1BA52
:10D0B8006FF001024FF0FF33CFE73A464FF00043DD
:10D0C800CBE700BFE1CF0108B3F1FF3F08BFB2F1E2
:10D0D800FF3FF8B5044616461D4618D0EFF31187F2
:10D0E800102383F31288BFF36F8FFFF791FEDDE9FA
:10D0F8000623C4E90A2300233246236320462B462D
:10D108000349FFF7F5FD87F31188BFF36F8FF8BD6B
:10D11800E1CF010870B50546EFF31184102686F3B8
:10D128001288BFF36F8FFFF773FE20B184F3118865
:10D13800BFF36F8F70BD6B6A63B184F31188BFF35F
:10D148006F8F28466B6A9847EFF3118486F312882D
:10D15800BFF36F8F05F118003EF0CAFA0028E5D03A
:10D168003EF057FA2146BDE870400148FFF738BB4A
:10D1780034490020034610B5EFF31184102282F3DE
:10D188001288BFF36F8FC1600121816000688342FC
:10D1980005D184F31188BFF36F8F002010BDD0E94B
:10D1A800003213605A600023C0E900333EF0ACFB44
:10D1B80021460248FFF714FBEFE700BF344900207F
:10D1C800F8B507460C4616463EF0E5F908B10020CA
:10D1D800F8BD0E4B9B68D3F88C50002DF7D0221D5C
:10D1E800F5D2EFF31184102383F31288BFF36F8F06
:10D1F800284647F00401B04784F31188BFF36F8FC6
:10D208000028E4D040F8045BE2E700BFD43B0020EC
:10D218000146024A0020FFF7D3BF00BF5D6705083B
:10D2280007B5064B4FF44062009305494FF0FF33B2
:10D238000448FFF75DF803B05DF804FB3C6007089D
:10D2480050C7002050330020F0B504468BB03FF0A3
:10D2580027F8042C2BD0354D286818B118F04AFC53
:10D2680000232B601CB3324B9C4220D0002601AB1C
:10D278000293304B214602A80393019641F0BEFF6A
:10D2880001983146013018F015FC0246286070B14B
:10D2980006AF3846019944F0ABFA274B214604A85B
:10D2A8000593049741F0AAFF2A68019BD65403F01E
:10D2B800ABFE3EF070FC46F0E9F83EF087FD01F069
:10D2C80017FA00221D4D1E4BD5F8F0401A7084B194
:10D2D80020460DF0E9F930B3A06807F043FBD5F814
:10D2E800F040002CF4D1D5F8F0301C46DB68002B58
:10D2F800FBD1C5F8EC400025124C02F0E1F80FF024
:10D308006BFF0DF0F9FA3EF0E1FF206818F0F2FB30
:10D3180025600D4C206818F0EDFB25600BB0BDE8CA
:10D32800F0403EF054BDE468DBE700BF943D0020C8
:10D33800E04000201BBA05089F1706086840002037
:10D3480034490020503C00204C3C0020002270B59D
:10D358000446154B00EB8105C3E900229A60264676
:10D36800306841F0FFFB022804F1040418D130684A
:10D378000E4C206098B10E483EF068FD20683EF0E3
:10D38800ADFB0C4802F05EFB01F05EFD064920682B
:10D398003EF09FFB0023236001F056FD012070BD85
:10D3A800AC42DCD10020E3E7183C0020483C0020D8
:10D3B800624408080F9D080873B506463EF007FD4D
:10D3C8000FF0C8FE18F078FA054618F081FA0446FE
:10D3D800641B00250FF0C6FEA4F580600FF0C8FEA0
:10D3E80001F086F900F034FC6B464FF400623046D9
:10D3F8001F4900953EF011FB01461E4B1E4C18605C
:10D40800009B19440EF08AF84FF4005201AB3046E5
:10D418001A4901953EF001FB0146194B1860019B22
:10D4280019440DF011F913F0D3FE2946D4F8E80099
:10D4380010F0B2F81621D4F8E80044F07DF866211F
:10D44800D4F8E80044F078F840F6B651D4F8E8008B
:10D4580044F072F8294604F1D80010F09DF8094804
:10D4680006F0E6F80122084B1A7002B070BD00BF42
:10D47800463108084C3C0020684000205D3108080F
:10D48800503C0020CC14080834490020F0B5092885
:10D498000546ABB000F0988001F044F9044638B175
:10D4A800002D69D14A4BD3F8F040003C18BF012445
:10D4B8002846FFF781FF3EF07FFC002C7ED006ACAB
:10D4C800444F01F027FD4FF40071204644F075F9F0
:10D4D8003C6001F02FF9012105463EF085FB3E4BEB
:10D4E8003E4A3F493F4841F031FC0AA800F01CFB86
:10D4F8003D493C4841F04FFC00260AAC14F8012B8A
:10D508003A493848013641F046FC202EF6D13849D0
:10D51800344841F01BFC45F0BCFF02213548FFF7B9
:10D5280015FF00233B6001F0FBFC0022002312AC36
:10D53800CDE90023284601222F4902943EF0A4FB9E
:10D54800E0B14FF47A703EF0AEFC0022002328468A
:10D55800CDE9002328490E2202943EF095FB48BBF2
:10D56800DDE9072105AB20463EF0EEFB20463EF004
:10D57800C5FB01F0BDF81DE0002499E7069841F0CD
:10D58800A0FE079A0646014605AB204601323EF04A
:10D59800CBFBD8B9079A059B9A4217D13146089810
:10D5A80057F085FA061E18BF012620463EF0A6FB56
:10D5B800002EC6D1002128463EF016FB0F4C6068AD
:10D5C800FFF742FE002363602BB0F0BD0126ECE7B5
:10D5D80068400020143C0020773108088A31080888
:10D5E800E0310808E88607088E940808FE9C0808B9
:10D5F800273A080878600708F0310808183C002026
:10D608002DE9F04F8046AB4E89B0002841D0002468
:10D61800202725463368012B00F0B480B8F1000FAD
:10D6280040F0B48001264FF4405301933EF037FC9C
:10D638000390002C40F05E814FF4C87BA1460BFBA1
:10D6480006F3012603F59C5A04930AF1080A01F02F
:10D6580005FF01F075FB05460290002800F099804F
:10D6680047F0100701F020FB934E306828B103788B
:10D678001F4002D118F03EFA3760B9F1000F04D00C
:10D68800002001F099F901F091F9284609B0BDE8A8
:10D69800F08F01F02DF801F071FB05460028B6D196
:10D6A800854FFFF789FE3EF08EFB3B68002B55D077
:10D6B8001A7822F020021A703B689A681C7812784F
:10D6C80092B1586808B105F0B3FF3B6801219B6827
:10D6D80007A80793FFF73AFE98B93B6898683EF0A9
:10D6E800B5FB764802F0AEF904217548FFF72EFE27
:10D6F80038B908217348FFF729FE10B1724802F0C3
:10D70800A1F9336818052BD500F0C0FF012827D1EF
:10D718006E484FF0000902F095F96D4B706883F878
:10D728000090FFF791FD3A68C6F804902AB1137883
:10D73800990644BF43F02003137033681A0511D5C6
:10D7480000F0A4FF441E18BF01243027336803F4F7
:10D758008073002B0CBF254601245BE72C46C3E7EA
:10D768005C48D6E71BB9242704F00104EEE714F05F
:10D77800020418BF83F480634FF0280718BFC3F36F
:10D788008024E3E702264FF440134EE70326524B6A
:10D798004BE73EF034FB059080B13EF04FFB68B19B
:10D7A80001F0ECFA054648B93EF036FB04287FF450
:10D7B8005BAF032000F070FF059D55E71CBB3EF0F2
:10D7C8001EFB08B301F0DAFAF0B944483EF086F9D6
:10D7D80001F092FA00283FD0414802F033F9B8F13D
:10D7E800000F02D03F4802F02DF9404601F0F2F94F
:10D7F8003D483EF02BFB3D4802F024F9B8F1000FFC
:10D8080001D045F043FE01243EF0F9FA2040C4B2AD
:10D818002EB101F0B3FA10B904F0BCFD06463EF093
:10D828003EFB039B049AC31A9A42054623D9B3FBCD
:10D83800FBF20BFB1235632D10D9B9F1000F04D0A0
:10D84800002001F0B9F801F0B1F8C5F5C87066B369
:10D85800B04228BF304628E02548BEE7B9F1000F9E
:10D8680004D101F0C3F8019801F0A6F80123C5F12D
:10D8780064000293EBE79A4506D23EF010FBCDE92F
:10D888000290DDF80890E2E6B9F1000F04D000201C
:10D8980001F092F801F08AF8039B5344581B16B123
:10D8A800B04228BF30460028EBD018F035F818F001
:10D8B8007DF8E6E7183C0020903D0020159D0808FB
:10D8C8006860070848600708CB930808439308086E
:10D8D800344900205C93080800303000624408088E
:10D8E800C09A08089B950808113308081396080879
:10D8F800EB9A08084FF00009B6E600BF07B5114BD0
:10D90800186820B103B05DF804EB3EF09FBA0E4BE7
:10D918001A68012A0FD19A68002A0CDD596851B19A
:10D9280009680C33C98809480091094941F00EFA81
:10D9380003B05DF804FB074803B05DF804EB02F0A0
:10D9480081B800BF483C0020183C0020E886070842
:10D95800FE3108087D990808F7B517F091FF01F026
:10D9680077F818F045F83EF024FA01F00FFA50481D
:10D978003EF0B4F83EF0CBFA01F0DCFA01F062F8C0
:10D98800B0FA80F00021400900F020FF10B908200B
:10D9980001F05EF801F056F818B901F05FF801F0EF
:10D9A80057F845F073FD3EF011FA3EF00EFA03F019
:10D9B80065FC3F483EF092F8002000F06DFE01F053
:10D9C80041F808B901F076F90125012000F0A4FE1C
:10D9D800012000F09BFE01F035F8FFF757FD3EF0FF
:10D9E800F7F9012001F024FA4FF480742846314EEB
:10D9F80014F4106754D015B92F4802F023F835787D
:10DA0800002D3ED101F01EF8FFF7FAFD0028EFD1F6
:10DA180001F018F8044600F06BFE2046FFF7CCFC36
:10DA28003EF0D1F9012001F057F901F00BF828B9BF
:10DA3800224B012101A80193FFF788FC00F0D6FFD3
:10DA48001F4800F0B9FF00F0B1FF3378012B1AD15D
:10DA580001F060FA00F0AAFC044601F061FA042023
:10DA6800FFF7F2FB00F0C2FF002000F0A5FF00F076
:10DA78009DFF012001F038F9032000F00DFE002081
:10DA8800B6E70025C4E70F4B0F4F3B6001F0DCF908
:10DA980000F012FD002304463B6001F0D5F9DEE7F3
:10DAA800002CB3D044F0F4FB384603B0F0BD00BFFF
:10DAB80062440808354900203C88080807320808ED
:10DAC800303030000F320808483C002008B50CF010
:10DAD80033FE00F02BFB042107480CF0F5FD3EF067
:10DAE800F4FB01F021FD03F00BFB06F003FDBDE89C
:10DAF80008400CF035BE00BF58410020014B187893
:10DB0800704700BF344900209FED010A704700BFED
:10DB18000000000000487047006889099FED010A6D
:10DB2800704700BF3333534038B505462021FBF713
:10DB3800ABFA041E11DA2146094839F012F900241B
:10DB480021462022074839F00CF9C4F1200228198F
:10DB58000021BDE8384056F0A2BF1F2CF0DD38BDCB
:10DB68009F320808B93208080428034607B506D8C2
:10DB780001460E4803B05DF804EB01F005BC062130
:10DB880068460B4A34F010FD052801DD39F01CFF0A
:10DB9800442200F108036B44411C684603F8082C32
:10DBA80001F0F2FB03B05DF804FB00BFE0320808A7
:10DBB800E5320808F8B5244DEB7DDB0731D52E6832
:10DBC800706801282DD9B168431ECA5C0A2A28D179
:10DBD8004A1E002B01DC1A4608E0D45C0A2CFAD055
:10DBE800013BF6E78C5C202C02D101329042F9D837
:10DBF800002B0CDD541CA04209D15C1E0C448C4245
:10DC080005D014F8017D0A2F0BD0202FF7D001443E
:10DC1800D21A11F8023C94083A2B00D10134013C85
:10DC280000D2F8BD04223046084943F0B4FD04216F
:10DC3800064801F0A9FB2B6904332B61EB7D43F007
:10DC48000203EB75EBE700BF543C002015430808BE
:10DC580020220021014856F022BF00BF20410020A9
:10DC6800002238B50B4C0546A26062754FF0FF32B2
:10DC78006B680846C4E9032363602560A1613DF031
:10DC88002DFF6B680BB90123E375BDE83840FFF73A
:10DC980091BF00BF543C0020F8B503780446DBB1BF
:10DCA8000E4FD7F8B80018B12146F3F72FF998B1FD
:10DCB8002046F3F73DF9461C304641F005FB054682
:10DCC80050B13246214656F0C4FE05491C22081DB3
:10DCD80056F0CCFEC7F8B850F8BD00BF6840002029
:10DCE800204100202DE9F347A24C06462368D3E9DA
:10DCF800011044F06BFDA5688146042D00F21182E5
:10DD0800DFE815F0050026012F01CA010A02731E7B
:10DD1800042B12D8D4E900325B689A425BD0012EFA
:10DD280000F0D481032E56D0052E58D123685D68A3
:10DD38002369ED1A0023A36099E10C2E37D18E4890
:10DD48003DF0CCFEA0693DF0C9FE226863682169F8
:10DD58009068C91A184401F017FB00252368D3E915
:10DD6800011044F033FD484503D20321834801F0F4
:10DD78000BFB236826699F68D3F80480701907EBAA
:10DD8800080138443DF08DFE8146A8EB0601B8191C
:10DD980001F0FAFA236822695B689B1A5B1BA3EB04
:10DDA8000900FFF7E1FE23692B4423616AE00D2E89
:10DDB80001D00A2E43D1A37D0BB19E420FD17048EA
:10DDC800A6753DF08BFE206843F047FD63682E463C
:10DDD8001844FFF761FF304602B0BDE8F087002322
:10DDE800A375082E01D07F2E38D126696268964225
:10DDF80048D92B462068B11AD0F808C08B4203EBEB
:10DE0800020723D1042BB4BF01270427F71B3B4685
:10DE18001CF80320194602F0C002802A03F1FF33E0
:10DE2800F6D0761A32467F1A4FF0010843F09FFD6C
:10DE3800F01BFFF799FE23699B1B2361EBE000238E
:10DE48001B2EA375CDD10123A3601BE01CF807701E
:10DE5800202F01D10133D1E70127D7E7E37D9A07C6
:10DE680017D5092E0CD0202E43D14FF000080321DE
:10DE7800206884F817802F4643F072FD0326D7E701
:10DE88000023E375E37D4FF0FF3623F00203E375CB
:10DE9800A1E7092E2DD123685A68D2B19B6822695F
:10DEA800134413F8010C15F005FD90B10426354B09
:10DEB80001930025019B21695A1C019229440122E2
:10DEC80020681F7843F034FD0135B5420770F1D161
:10DED80044E7236860689D6821692B4A091A01ABE9
:10DEE80028440EF0D1FC06460028CBD0431CE0D1D4
:10DEF80028E71F2EC6DDF7B206F0C006802E18BF31
:10DF08003B462068D4F810C001BF8368217D13F810
:10DF18000C30013103F14002D2B214BF0021C9B262
:10DF2800372A9FBFE525DB0803F006031D4188BF9C
:10DF3800002521754FF00102614498BF05F00305E3
:10DF480043F0F6FC237D0770AB429BD1013505E712
:10DF58004F2E04D05B2E40F0E480022374E70423A4
:10DF680072E7A6F13003092B10D803236675A36066
:10DF780088E700BF543C0020EA320808F33208085A
:10DF88001133080815430808E88607080023413EAE
:10DF9800A360072E3FF676AF01A353F826F000BF23
:10DFA800C9DF010829E0010869E001088DE00108DE
:10DFB8008DDE010835DD01088DDE0108D5E0010898
:10DFC800E368062B3FF75EAF574A03F1010A2D338A
:10DFD80002EB8308D8F80830002B3FF453AF2568CC
:10DFE8006668A8682169014430443DF05AFD074637
:10DFF80028466E60D8F80810C4F80CA043F08BFCD3
:10E008004FF001082268636826695568F61AED1A08
:10E01800002E3FF70DAFB8F1000F7FF49FAE26E05A
:10E02800E568002DFFF62EAF2668D4F80480B068A6
:10E038002169013D014440443DF033FD71680746C4
:10E04800A1EB08013046E56043F08AFCE268002A4B
:10E05800D6DB354B206803EB8203D3F8B810CDE745
:10E06800236825695B689D422CBF00250125002D8A
:10E078007FF708AF2368294698682369184401F098
:10E0880083F990E6226963689A427FF6FBAE002521
:10E098000126A8462F46CBE67E2E42D1637D313B32
:10E0A800072B3ED801A252F823F000BFD5E00108A3
:10E0B8002BE10108F1E0010835DD01082BE1010839
:10E0C8002BE10108D5E0010835DD01082368656802
:10E0D80098682669811928443DF0E3FC761B0025E1
:10E0E8000746A846A56093E72068216943689942D6
:10E0F80017D2012285685B1A0D4415F8016F06F0E6
:10E10800C006802E01D19A4204D143F030FC00238E
:10E11800A36022E60132F0E7462E3FF407AE482E10
:10E12800D4D0002390E600BF684000202DE9F04FCE
:10E138008BB068460A4BCDE900451968CDE90267FE
:10E14800091A8908CDE90489CDE906ABCDF820C0C4
:10E15800CDF824D00CF0B8FA0BB0BDE8F08F00BFB2
:10E168006840002070B5067804461EB14FF0FF35B0
:10E17800284670BD3DF0C1FFC31E012B05460CD8D3
:10E1880001210C48217001F0FFF8032DEED10A4857
:10E19800836E60309E600BF0B9FDA388013B9BB293
:10E1A800A380002BE4D10121044801F0EDF8638835
:10E1B800A380DDE7F7320808684000201533080817
:10E1C8002DE9F0434FF0000997B0044603A817461D
:10E1D8001D468846CDF810900BF07EFD07F001062D
:10E1E8000346002877D1F90665D5D4E90121DC205A
:10E1F80042F054FA0446B8F1010FD4F8009007D160
:10E208004FEA091140F2DF2041F0060113F048F807
:10E218002146424601A811F04FFB4946C7F3800248
:10E2280001A80AF0F7FFB8F1010F044601D1FFF782
:10E238004DFC380602D4032000F0E6F914B120465C
:10E2480044F040F84FF0FF3000F0DEF901200EF006
:10E258004BFC16F001FC1EB10121454801F094F871
:10E268000024FDB12C60ECB14FF0FF33049FAB608C
:10E2780038466F6015F0AEF9A0B16946384601AA74
:10E2880044F064FA019B6BB15A68AA60002285F8D1
:10E298002C20186843F0EAF82022014605F10C000A
:10E2A80056F034FC1EB10121314801F06DF82046CA
:10E2B80017B0BDE8F0837A0605D594E80E00DC2097
:10E2C80042F0A0F996E7BB0695D5204643F0AEF894
:10E2D80042F0F2F98EE74FF0FF3000F095F948462A
:10E2E8000EF002FC790602D5A368206898471EB193
:10E2F80001211F4801F048F8049C204609F074F8F1
:10E308001C490EF0B3F8F0B1049844F005FA0E2851
:10E3180017D0C20705D4830708D10268164B9A4262
:10E3280004D143F072FF40F480749AE7014600225A
:10E33800124809F075F81249104840F087FC01208E
:10E34800F1E70020EFE70F4B9C420DD004990B48F2
:10E3580040F054FF049B0C4918680EF087F8002819
:10E3680014BF822401247CE74FF4006479E700BFDE
:10E37800F7320808DCA00708F4980708E8860708B9
:10E38800273A0808E0400020B8A0070808B5037835
:10E398004BB901210170044800F0F6FF3DF0ADFED5
:10E3A80003380128FAD808BDF7320808F0B58BB051
:10E3B800202106A843F001FA002536483DF08EFBDF
:10E3C800079535483DF08AFB3DF097FE431E032B29
:10E3D80043D8DFE803F002353F4707990229ECD11B
:10E3E800089B1A78052AE8D15F78412F05D02B4879
:10E3F80000F0CAFF00230793E3E78024012628489A
:10E4080000F0C2FF03216846ADF800408DF80260B5
:10E4180000F0BAFF002301AA0392224A314604926F
:10E42800214A03A805923A468DF80430ADF8064013
:10E43800ADF80840FFF7C4FEC305DBD50BB0F0BD4F
:10E448001A483DF04BFB06A843F0D9F90020184BB9
:10E458001870F3E700230793B6E7C1B206A843F0A4
:10E468000BFAB1E713483DF039FB079B43B90F4856
:10E478003DF034FB06A843F0C2F94FF48070DDE7A5
:10E4880000231122012106A8FFF79AFE10F4106F4D
:10E4980096D0D3E7F9320808B13B0808D8560708E0
:10E4A800143308086DE1010895E3010811330808E1
:10E4B800354900201733080870B598B0202101A805
:10E4C80043F07BF9474E48483DF008FB47483DF08C
:10E4D80005FB45483DF002FBB28A002302B1B38236
:10E4E80005A8029306930BF0F7FB044688B9404948
:10E4F80001A83DF0E4FA012805462BD13A483DF041
:10E50800EDFA01A843F07BF920463A4B1D7018B08C
:10E5180070BD00200EF0E8FA33483DF0DFFA0699A6
:10E52800354840F06BFE029B002BD5D001A843F084
:10E5380094F90EF0EBF858B10A2101A843F09CF9C0
:10E548002E4901A83DF0BBFA0328C2D00428EDD11A
:10E5580000212CE0851E032DE5D801A353F825F0F2
:10E5680079E50108DBE4010881E5010893E5010884
:10E578001D483DF0B3FAA6E71B483DF0AFFA01A8E5
:10E5880043F03DF94FF48070C1E71D483DF0A6FA0D
:10E59800002302933DF0B1FDC1B203298DF80310A9
:10E5A80097D004290CD110483DF098FA0121002396
:10E5B800162201A8FFF704FE10F4106F8CD0A6E70E
:10E5C80001A843F059F99DF803300D2B03D10D48EC
:10E5D8003DF084FADEE701210DF1030000F0D4FEDE
:10E5E800D8E700BF68400020113308088A310808BE
:10E5F8001A33080835490020E88607085633080802
:10E608001F3308084F330808014B1860704700BFD4
:10E61800DC060020024B986A003818BF01207047BA
:10E62800684000202DE9F04106460D4600270DB947
:10E63800BDE8F08133780A2B15D1A7B901210D481F
:10E6480000F0A2FE01243319A542984604D013F81D
:10E65800012B57B90A2A08D13046214600F094FE0A
:10E6680046462D1BE3E70024EDE70D3A5742574194
:10E678000134E9E75B330808024B0348197842F094
:10E68800FAB800BF36490020FC810708014B18780A
:10E69800704700BF36490020014B1870704700BF13
:10E6A8003649002010B5064C23783BB14FF47A72F6
:10E6B800044B1A6000F020FE0023237010BD00BF39
:10E6C80037490020E0060020074B1A685AB11A683B
:10E6D800012A09BF05491A680A704FF47A7218BFEF
:10E6E80002F1FF321A607047E00600203749002027
:10E6F8004FF47A7208B5044B1A6000F0FDFDBDE8CE
:10E70800084016F057BF00BFE00600200146014848
:10E718003DF042BAC0130020014601483DF05ABA04
:10E72800C0130020024B5868003818BF01207047FA
:10E73800703C0020034B04485B68002B08BF002096
:10E74800704700BF703C0020C01300200268044BD3
:10E758009A4206BF808800F001000020704700BF81
:10E7680024B107080022002310B59CB004AC014670
:10E77800CDE9002305480E2202943DF085FA10B930
:10E7880020463DF0BBFA1CB010BD00BFC0130020EE
:10E7980070B50023164600229EB006AC0D46CDE9A2
:10E7A800002301460E22084802943DF06DFA40B954
:10E7B80032462946204605AB3DF0C6FA20463DF0D4
:10E7C8009DFA1EB070BD00BFC01300200023F0B535
:10E7D800434E444CADF5137D074630460D46636005
:10E7E800B38000F097FD06F1800045F0D3FD0D28B9
:10E7F80002D11FB915B970E0002D6CD04FF4007329
:10E80800002200930721384812AB18F07DFA00283F
:10E8180063D100F071FD3549334818F08DF90028AF
:10E828005BD13349304846F0C8FC002855D13148FF
:10E83800FFF798FF3048FFF795FF3048FFF792FF42
:10E848002F48FFF78FFF2F49274846F0B6FC2E4B7D
:10E8580003AA03F13807154618685968083303C531
:10E86800BB422A46F7D11B8839222B80274803A9A7
:10E87800FFF78EFF2648FFF775FF264B03AA03F123
:10E888001007154618685968083303C5BB422A465D
:10E89800F7D1186899889B792860A9801E4803A930
:10E8A8001622AB71FFF774FF1C490F4846F085FC30
:10E8B80098B900F021FD1A4B012523600023E3607D
:10E8C800184BC4E90156C3E93B443FF055FD2846BF
:10E8D8000DF5137DF0BD0028EDD00020F8E700BF4E
:10E8E800C0130020703C0020401400205D3308084D
:10E8F8006733080873330808863308089D33080807
:10E90800A7330808B4330808E9330808B8330808F7
:10E91800CC33080823340808DB330808E433080834
:10E92800CC140808684000202DE9F041CAB01C4604
:10E938001546509E0AB1002313700CB100232360C2
:10E948001EB100220023C6E9002302AF3A468030F8
:10E9580046F02CFB804618BB3B7B03F0100315B137
:10E96800C3F300122A7014B10BB93B682360BEB11F
:10E978007B89398903F01F025200480A0192C3F3C8
:10E9880045120092DB0A01F01F0200F2BC70C1F3CD
:10E99800431146F0B6FE044BA0FB0330C6E9003035
:10E9A80040464AB0BDE8F08100CA9A3B01483DF0B4
:10E9B800BEBC00BF843C002038B5094D04462B6816
:10E9C80083420CD0074B19783DF0DCF92C60011E0E
:10E9D80018BF0121BDE83840034801F053BB38BDDA
:10E9E800803C0020400C0020843C002070B50B4C7B
:10E9F800257895B901260A490A48267001F01CFBBA
:10EA08002A46314607483DF0BCFC4FF08072064B61
:10EA180018681A60FFF7D0FF257070BD38490020CC
:10EA2800F0730708843C0020803C0020014B1870DC
:10EA3800704700BF400C0020014B1878704700BF9A
:10EA4800400C0020014B1878704700BF394900205E
:10EA5800014B1870704700BF394900202DE9F34178
:10EA680016F008FF3E4B074620F47F0020F47F4055
:10EA780098423C4D0BD117F47F4FC7F3072406D0BB
:10EA880016F0F2FE2C70204602B0BDE8F08100239B
:10EA98002B703CF0E6FF072803D8A223C340DB070E
:10EAA80035D4314816F0E0FEFFF7A0FF4FF07E5353
:10EAB8002E4801A901933DF0E0FBDDED017AF5EE6A
:10EAC800C07AF1EE10FA24DB9FED297AF4EEC77ACA
:10EAD800F1EE10FA1DD89FED277A67EE877AFCEEE3
:10EAE800E77A17EE905A3DF0CBF90024064688469F
:10EAF80020462146A84271F100030DD30020FFF7FC
:10EB08005BFFFFF753FF4CBB384616F0ADFE002401
:10EB1800B9E74FF47A75E6E7ACB9FA220023F2F7C1
:10EB28009BF97D2A73F100030DD32046FFF744FFBC
:10EB380000F044FF044658B13DF0A2F94FF47A754D
:10EB48000646884604E00C48FFF736FF002CEFD055
:10EB58003DF096F9801B61EB0801CBE7112492E7A1
:10EB6800AF0000AD39490020AF1100AD3A340808B4
:10EB78000000804F00007A4400303000024B43EA26
:10EB8800002016F071BE00BFAF0000AD0D4D08B5F6
:10EB98002B780446012B0FD901280DD90A4838F0E3
:10EBA800E0F82146094838F0DCF82978084838F0B8
:10EBB800D8F838F0DAFEFCE72046FFF7DFFF44F02C
:10EBC80061FC00BF39490020543408086A34080839
:10EBD8007634080810B50446002838D01C4800F0E0
:10EBE80031FF631E112B12D8DFE803F02D1111112C
:10EBF8001111112B1129111127212523091F15483E
:10EC080000F020FFBDE81040134800F01BBF023C95
:10EC18001248E4B200F016FF0A2C16D8104B53F82D
:10EC2800240000F00FFF0F48EAE70F48E8E70F4815
:10EC3800E6E70F48E4E70F48E2E70F48E0E70F4848
:10EC4800DEE70F48DCE70F48DAE70F48E9E710BDD1
:10EC5800F09208087693080803930808E2990808D0
:10EC680050750708139308082D980808949A0808FF
:10EC78006594080877940808649508083895080882
:10EC88003B9A0808329608082394080808B5FFF745
:10EC980003FD044B03F178029A62BDE8084016F0C0
:10ECA80005BE00BF684000200022014B1A60704773
:10ECB800983C00200122034B1A700022024B1A6074
:10ECC800704700BF3A490020983C00200022014BC1
:10ECD8001A7070473A490020024A136803431360C8
:10ECE800704700BF9C3C0020024A136823EA0003D7
:10ECF800136070479C3C0020014B1878704700BF98
:10ED08003A49002038B50B4B1B7893B10A4B1B6866
:10ED18007BB90A4C25683DF0C2F82060236813B916
:10ED280023680133236025B9BDE838400120FFF787
:10ED3800ADBF38BD3A4900209C3C0020983C0020DB
:10ED480010B50C4C206890B10B4B1B6883B93DF093
:10ED5800A6F8236883422368A0EB030040F2EE2361
:10ED680088BF00F1FF30984294BF0020012010BDF9
:10ED78000020FCE7983C00209C3C0020024B1868CF
:10ED8800003818BF01207047983C002010B5054C8A
:10ED980023782BB93DF023F844F09FFB012323701F
:10EDA80010BD00BF3B49002073B505460C46C1B1F4
:10EDB8000E4B1B78C3B90A4601AB01460C4804F058
:10EDC800E1FD06460B4B1B7853B905F0F3F940B14A
:10EDD800214628463DF00BF82146284616F03CFF10
:10EDE8003446204602B070BD0E46EBE73C49002091
:10EDF800B40800203D490020024B1A7818701046CC
:10EE0800704700BF3D490020024B1A781870104621
:10EE1800704700BF3C490020034B1B7813B90348D7
:10EE28003DF014B8704700BF3E4900208D340808F3
:10EE380010B10122024B1A70024800F0EBBA00BF71
:10EE48003F490020A03C0020F8B5234B1E7826B18E
:10EE5800BDE8F8400120FFF7EBBF204B20481E70AB
:10EE68003FF0C7FB1E483FF0AAFB78B33CF0C7FF52
:10EE780080F00105EDB21A483FF0B3FB80F00104C1
:10EE8800E4B21DB10120FFF7B7FF064604B3012025
:10EE9800FFF7BAFF074613483CF0D8FF12483CF08A
:10EEA800D5FFFEF72BFD11483CF0D0FF10483CF091
:10EEB800CDFF10483CF0CAFF15B13046FFF79CFF64
:10EEC80044B13846BDE8F840FFF79EBF0125D2E7B8
:10EED8002746E0E7F8BD00BF3E4900203F49002033
:10EEE800E807002094340808993408089E34080874
:10EEF800A234080891340808044B1B7823B9044B42
:10EF08001B780BB1FFF7A0BF704700BF3E49002038
:10EF18003F4900200122014B1A7070473E490020EA
:10EF28000022024B02481A7000F074BA3E490020D1
:10EF3800A03C0020034B044A04481A6000225A608F
:10EF48003FF051BBA03C002001EF0108E80700207A
:10EF580008B547F0FBFC3CF0DCFF01F0CFFFFFF702
:10EF6800A1FB47F0F5FC3CF0D4FF002044F092FAF6
:10EF7800034BC3E90001BDE8084047F0E8BC00BF07
:10EF88005034002008B5FFF79FFBBDE80840002279
:10EF9800014902483DF0CAB859EF0108B43C0020C5
:10EFA80010B5074C04F098F923680BB916F0A0FCCB
:10EFB800236801332360BDE8104004F0A7B900BFFF
:10EFC800B03C002008B504F087F9074B1A6812B165
:10EFD8001A68013A1A601B680BB916F097FCBDE86D
:10EFE800084004F093B900BFB03C00202DE9F04F71
:10EFF8009E4BAFB01D6804460291002D40F02D8154
:10F008000223ADF810500593ADF81250FFF78AFBB4
:10F01800804618B900264FF0000837E0FFF78AFB52
:10F0280007460028F6D08022914992483DF005F91C
:10F03800DFF860928E4E2B46002818BF4E462A46AF
:10F04800314638460095FFF76FFC48B12B462A46F3
:10F05800494638460095FFF767FC0028DAD14E4646
:10F06800854B06A8069301220023314603F0E0FEF3
:10F0780006A83EF034FE0028CDD106A80DF11202F4
:10F0880004A93EF047FE06A83EF0E8FDBDF81030A2
:10F0980033B97A4A137A527AADF81030ADF81220A3
:10F0A800B4FBF3F3782B98BF012305A9744898BFE4
:10F0B80005933DF0D7F8BDF81020DDF814C0BDF871
:10F0C80012300CFB02F794FBF7F794FBFCF40CFBF3
:10F0D80003F10298DFF8C0A190FBF1F1BAF810B083
:10F0E80068480BF1010BA0F828C0A0B2A0EB0B04F4
:10F0F800B4FBF2F4012FB8BF0127BAF812A0624D91
:10F10800AAEB030AA5F80EA04FF0010AA4B22C83BB
:10F1180012FB04F4A4B22C82041BAC8195F8504075
:10F128001FFA87FE44F0020485F85040574C022924
:10F13800B8BF0221AA83A28312FB0EF292B2801AF0
:10F148002282029AA5F81AA092FBFCF24FF0000A5C
:10F1580017FB01F9013989B2EB836B82E38313FB57
:10F1680001F39BB2DFF834B16382D31AE38194F8D8
:10F178005030A081DBF8000043F002031FFA89F940
:10F18800A5F822A0A4F818E06183A4F822A084F8C6
:10F19800503038B13EF062FDDBF8000016F0AAFCF2
:10F1A800CBF800A0B8F1000F1ED00021A02016F067
:10F1B80081FC8046CBF80000B0B12F4B4A46036073
:10F1C8003146002303F034FE40463EF088FD0346F6
:10F1D800DBF80000002B43D13EF086FDDBF800A0F1
:10F1E8008046BAF10E0F03D1244B9A46D3F8048017
:10F1F80040463DF0E2FA1D4E02903068BDF810B06E
:10F2080018B116F077FC00223260B9F1FF0F8CBFFD
:10F2180002220122002102FB09F0039216F04AFCA7
:10F228003060D0B1029B039AB3FBFBF3686202FB28
:10F2380007009BB2414660621448EB82AB82E382CE
:10F24800A3823DF048F941460F483DF044F9524643
:10F258000D4B0E490E483FF0C2FA2FB0BDE8F08FB3
:10F2680016F048FC0023CBF80030BDE7C83C00206E
:10F2780040490020CB340808B47E07080CA90708C9
:10F28800E3340808E4060020FC08002050090020A8
:10F29800B4080020B1340808D4090020C43C002078
:10F2A80010B5074C206850B116F024FC0023054A1D
:10F2B80023605362044A5362044AC2E9033310BD0F
:10F2C800C83C002050090020FC080020B408002099
:10F2D800024B1868003818BF01207047C83C00204E
:10F2E80010B5044C23781BB9FFF75AFE012323708D
:10F2F80010BD00BFC049002010B5054C16F042F9FA
:10F3080023780BB1FFF75EFE0023237010BD00BF0A
:10F31800C049002010B50F4B04460360838843F0B2
:10F328000503838044F0A2F801230E220A4984F8D9
:10F338008430231DC4E90823C4E90D2323616161D6
:10F34800064B0749A060C4F88040E260A162E3630D
:10F3580010BD00BF24B107081DBF0508A1C00508DE
:10F368007BC00508034B1868034B002808BF1846E4
:10F37800704700BFCC3C002071852149014B1860C3
:10F38800704700BFCC3C00202DE9F843DFF88080AF
:10F3980000AF05460E463CF00EFDD8F8003043B3EA
:10F3A8001A483CF094FFC0F500720446D8F80000F3
:10F3B80043689919914223D90734D21A294624F06F
:10F3C800070442F0E8F9E946ADEB040D69460F4839
:10F3D800D8F8004000F040FB0146204642F09BFA76
:10F3E8000A21D8F8000042F047FA0023C8F8003094
:10F3F800CD4631462846FFF7D7FCBD46BDE8F88321
:10F408003246294642F0C7F9F3E700BF6993080876
:10F41800143C002010B5044603F05EFFE3681BB9F6
:10F428000C4A1168A14203D1BDE8104003F06EBF39
:10F43800A360094B1968E160196809B119688C6003
:10F44800116801B914601C6003F060FF16F02EFA11
:10F4580010BD00BFD83C0020D43C00202DE9F0416D
:10F46800144E47F076FA33680BB3134D03F034FFAC
:10F478002C681CB1BDE8F04103F048BF01230F4AD6
:10F488002B603368346014601BB92B68013B2B6018
:10F49800F0E79F68C3E90244D3E9006803F036FF48
:10F4A8000EB14046B04703F017FF3B46ECE7BDE816
:10F4B800F08100BFD83C0020D03C0020D43C002084
:10F4C8002DE9F7430025A846144E019503F004FFE3
:10F4D800346801AF54B9019B3360114B1D60114B67
:10F4E8001C6003B0BDE8F04303F010BFD4F80890E7
:10F4F8002046C4F808800BF0D7F818B10023E36061
:10F508004C46E7E760680BF0CFF80028F6D12B46A9
:10F518003C60254604F10807F1E700BFD83C00200D
:10F52800D43C0020D03C002010B5044B1C6804B922
:10F5380010BD606841F096F9A468F8E7D83C00204F
:10F548006FF013030B41DB0710B502460C4615D5C7
:10F558000B490C483FF01FFC022C03D0052C0BD0A4
:10F56800094900E0094907483FF015FCBDE810408B
:10F57800074904483FF0EABB0649F4E710BD00BF5D
:10F58800F79A0808E88607084E980808F5970808C3
:10F59800273A0808019808082DE9F04FA1B004AFF0
:10F5A80082460E469146FFF7C5F828B90125284638
:10F5B8007437BD46BDE8F08F0022002307F1100420
:10F5C800CDE900239549012202943CF05DFB002817
:10F5D800ECD13B7C0BB9042560E020463CF0BFFD34
:10F5E8005B28804629D040B30AF1FF3B1BF8015F36
:10F5F8005DBB404614F05EF918B120463CF0AFFD03
:10F608008046B8F13D0F22D120463CF0A8FD2228C3
:10F618000CBF0123002389F8003040F0D080204639
:10F628003CF088FD22282FD01DD858B30A2829D0AD
:10F63800C1B230463CF0ABFDF1E720463CF09DFB03
:10F64800014620463CF090FBC3E7454506D0B8F19B
:10F658000A0FBED020463CF091FDBAE720463CF0A8
:10F6680069FD8046C2E75C28E2D120463CF062FD95
:10F678007628DDD8612819D80A2803D0552851D012
:10F688000028D5D1052508E020463CF068FD0A2869
:10F6980003D0232806D00028F4D1EDB220463CF050
:10F6A8002DFB84E720463CF069FDF6E7A0F16203F4
:10F6B800142BBDD801A252F823F000BFC3F70108EC
:10F6C80039F6010839F6010839F6010829F7010861
:10F6D80039F6010839F6010839F6010839F6010842
:10F6E80039F6010839F6010839F601081DF701084D
:10F6F80039F6010839F6010839F6010819F7010841
:10F7080039F6010821F70108A7F7010825F70108CC
:10F718000D208DE70A208BE7092089E70B2087E772
:10F728000C2085E74FF0080B0BF1080323F00703C3
:10F73800E846ADEB030D0DF1100AD1460AEB0B03B9
:10F7480020467B603CF0F6FC7B6809F8010B994584
:10F75800F6D1002307F10C010AF80B3010225046AD
:10F7680032F0C0FFFB6801464B4524D1B0F5881F35
:10F778001ED27F2816D9B0F5006F15D3B0F5803F9B
:10F788002CBF04230323327B22B1726813443268EE
:10F798009A420BD9304642F076F8C5463FE74FF01B
:10F7A800040BC1E70123EEE70223ECE77360F4E7FB
:10F7B8000225C54671E7C54664E7082038E70A28E8
:10F7C8003FF460AF00283FF45DAF00250D281BD043
:10F7D8000ADC092818D00A2811D080B1C1B23046F5
:10F7E8003CF0D5FC002514E020280DD02328F5D1C5
:10F7F800736820465B1B73603CF0C0FC02E07368D2
:10F808005B1B7360002548E7C1B230463CF0BFFC83
:10F81800013520463CF08EFCD8E700BFCC33080801
:10F8280030B587B00D4610220DF1070302A93CF050
:10F83800B9FC044648B99DF8073083B9094902A8BC
:10F84800F1F764FB20B901232B70204607B030BDC7
:10F85800054902A8F1F75AFB08B92C70F5E7052409
:10F86800F3E700BFFC340808013508082DE9F0412A
:10F878008EB002AC0F46302221460DF103033CF056
:10F8880091FC054628B99DF80380B8F1000F04D013
:10F89800052528460EB0BDE8F0812046F1F748FB63
:10F8A8002618A6420CD99DF808302B2B01D02D2BF9
:10F8B80006D12D3BD3F1000848EB03080DF10904EC
:10F8C800311B022923DD2378692B15D163786E2B30
:10F8D8001DD1A378662B1AD14FF0FF43E01C01938A
:10F8E800B042D5D1DDED017AB8F1000F01D0F1EECB
:10F8F800677AC7ED007ACCE76E2B08D16378612B65
:10F9080005D1A3786E2B02D1054BE01CE7E7204612
:10F9180001AA10F07FFE0028BAD08442E0D1B7E7F0
:10F928000000C07F70B5054688B004A80C462021A9
:10F9380041F043FF28460DF1060204A9FFF72CFE0B
:10F94800064630B99DF8063033B104A805F0CEFF5D
:10F958002060304608B070BD28460DF10701FFF75A
:10F968005FFF38B99DF80730002B0CBF1E233E23DC
:10F978002360EEE7284602A93CF039FC18B9029842
:10F9880042F006FCE4E7284603A9FFF76FFF88B9B1
:10F99800DDED037AF4EE677AF1EE10FA7DBF17EE2B
:10F9A800903A23F0030343F00203034B78BFA3F11B
:10F9B800FF43DDE70526CCE70200400010B586B01E
:10F9C8000B4901A800F038FB012101A83CF0FFFC1D
:10F9D80001203EF071FF01A83CF0B6FC044601A8E6
:10F9E8003CF0A5FC84F00100C0B206B010BD00BF19
:10F9F800C0720708A1F18003602B70B5064619D8BC
:10FA0800194602230D480E4C10F8012B914205DAD5
:10FA180003FB0144E518A54206D870BD891A12FBFC
:10FA280003F201331444EFE7304614F8011BFFF7E3
:10FA3800E1FFF0E7BDE8704041F025BF74440808D5
:10FA48007E4408080246024902483FF07FB900BFD9
:10FA580007350808E48A07082DE9FF47054680248A
:10FA68000A4615F8011B6846013141F0C1FE009EA7
:10FA78003C4FDFF8F880DFF8F890013E019B9E428A
:10FA880005D8684641F0E9FE04B0BDE8F087C3B187
:10FA9800029A1A4412F8013C202B35D0A3F16102D6
:10FAA800192A33D9A3F14102192A31D9A3F1300215
:10FAB800092A2FD9252B2FD013F0800F14BF062326
:10FAC800042317F803C00CEB4C020CEB8203002252
:10FAD80018F8031003EB080A8E46134628785B00D3
:10FAE8002040003818BF0120640843EA000304BF1F
:10FAF8008024013501328B42D2B20FD31AF80200AA
:10FB080000EB41018644E9E70023DAE70123D8E75F
:10FB18000223D6E70323D4E70523D2E7124A4B444E
:10FB280032F81C207244521A995C012916D10B2212
:10FB380000202B7840002340003B18BF01236408B5
:10FB480004BF80240135013A40EA0300F1D141F0B5
:10FB58008DFC0146684641F0DEFE8FE76846FFF7F8
:10FB680049FF8BE7DE47080858FF0708B74708082A
:10FB78005B46080808B5024837F0F3F8002008BDCE
:10FB88000A35080838B5FEF7D5FD044620B90D48F2
:10FB980037F0E7F8022038BD3CF011F820B90A48E0
:10FBA80037F0DFF80420F6E7084D2B782BB920460C
:10FBB8003CF049F808B90648F2E7012300202B7009
:10FBC800E9E700BF1D3508082F350808C34900209C
:10FBD80042350808F8B514460E461F46FEF7AAFD3A
:10FBE80005460420FFF778F83B462246314628466A
:10FBF80045F073FDD5F8CC30A34207D134B14FF4AA
:10FC08000072314605F5807054F023FFD5F8BC30FA
:10FC18000020A3429EBF0122014B1A70F8BD00BF0D
:10FC2800C249002038B50C461546FEF783FD022C64
:10FC380003D0052C07D0012C15D12A46214617F0F0
:10FC480039FE002038BD2A4600210A4C17F032FE42
:10FC58000420FFF749F82378002BF2D0FFF752F879
:10FC680000232370EDE70448214637F07AF86FF057
:10FC78008500E7E7C24900205235080870B50546F7
:10FC88000C4637F06EFFD8B1237853B9144A28468A
:10FC98001370F4F785FD20B10121124A124837F09C
:10FCA800AFFC2678012E0BD100220D4B28461A7086
:10FCB800F4F7D8FD20B10D4A31460B4837F0A0FCC7
:10FCC8002378052B06D16368054A003B18BF01233A
:10FCD800137070BD042B02BF0022014B1A70F8E7A5
:10FCE800C14900206F3508084C5507088F350808AA
:10FCF80013B5964837F035F8954837F032F89549F6
:10FD0800954837F08FFF034638B1944A012194484B
:10FD180002B0BDE8104037F07CBC92498E4837F0FD
:10FD280081FF034608B1904AF0E790498A4837F0C6
:10FD380079FF034608B18E4AE8E704F03BFA98B920
:10FD48000E2004F0B7FA04F03BFAD8B90E2004F0FC
:10FD5800BFFA8848F3F7D8FB014608B3864802B0D3
:10FD6800BDE8104036F0FDBF0121802015F0A2FE4D
:10FD780003460028E4D080228049814804F004FA30
:10FD88007F48DEE70121802015F094FE0346002815
:10FD9800DCD080227B497C4804F0F6F97A48D6E723
:10FDA8006D4837F09EFE0128044650D1774836F05A
:10FDB800D8FF2146764A6848F5F77AFE38B1754A81
:10FDC8000121674802B0BDE8104037F019BC7248FD
:10FDD80036F0C7FF04F0EEF948B1704923462246D1
:10FDE8005D48F5F785FF014608B16D48B7E704F0AF
:10FDF800E7F940B101236B491A465748F5F778FFF0
:10FE080001460028F1D1012367491A465248F5F7FF
:10FE18006FFF014608B16548A1E7654836F0A1FFC4
:10FE280004F094FA60B1634836F09BFF01236249FD
:10FE38001A464948F5F75CFF014608B15F488EE766
:10FE480001210223EF224448009137F051FE5C481B
:10FE580036F087FF00215B4A3F48F5F729FE044644
:10FE680008B1594AACE704F0A5F978B1574836F01B
:10FE780078FF0123224649493748F5F739FF28B169
:10FE8800534802B0BDE8104036F06BBF04F098F953
:10FE980050B14E4836F065FF0123002241492E48F3
:10FEA800F5F726FF0028EBD1012300223E492A4816
:10FEB800F5F71EFF044608B10146ACE704F046FA20
:10FEC80060B1444836F04DFF3B49012322462248A1
:10FED800F5F70EFF014608B13F4840E70124022329
:10FEE800EF2200211C48009437F002FE3B4836F010
:10FEF80038FF0021184837F01FFE394836F031FF27
:10FF08003849154838F05AF908B1374A58E7374898
:10FF180036F027FF04F046FB354836F022FF0E483E
:10FF2800F4F7FEFB034608B1324AEFE6324836F0F2
:10FF380018FF094837F015FE30B90748F4F730FCC8
:10FF4800034608B12D4AE1E602B010BDB0350808F5
:10FF5800C2350808CC0700206C120020DE350808DE
:10FF68004C550708B40700200C3608089C070020E9
:10FF78003E3608082C0700206B3608088852070808
:10FF8800B83400206C520708583400208E36080810
:10FF980044070020AF360808D63608081D2308088D
:10FFA800FC360808FD2208088C2308081F370808B3
:10FFB8004437080869370808FE2408088B370808FA
:10FFC800B137080858070020D2370808F937080859
:10FFD8001F3808083F3808086138080887380808B3
:10FFE8009D38080885FC0108B3380808D738080880
:08FFF800E9380808F438080894
:020000040802F0
:100000001D3908082E39080808B5064B1B7803F07F
:10001000FF002BB1044837F0A3FD80F00100C0B20F
:1000200008BD00BFC14900206C12002008B504F0D3
:10003000C5F80028014808BF002008BDB8340020DA
:1000400038B50D4600F10C0200F108010446A888FD
:10005000FBF728FB00280ADBA06865603AF0EEFF9A
:1000600038B9094836F081FE20463CF064F9012099
:1000700038BD4FF48032217BA0683CF04BF900285A
:10008000F2D16073F4E700BF7939080838B5044647
:100090000D468068227B012303FA02F1036982681E
:1000A0001B680B40003B18BF0123AB4214BFD36851
:1000B00013699847014610B1024836F056FEA57301
:1000C00038BD00BF9039080838B50129094A0446EF
:1000D0000D4618BF4FF40032017B80683CF01AF9DE
:1000E000014620B1044836F040FE012038BDE573DA
:1000F000FCE700BF06000200A839080890F950305C
:10010000214A002B836AB4BF418A018A002B08BFB1
:10011000134610B5B0F90C4082890C44997BA4B207
:10012000C1B193F9051011FB02F15A88114409B2CB
:10013000A0F8461093F905205B8812FB04F21344E3
:100140001BB29942D2BFA0F84A30A0F84A10A0F8DA
:10015000463010BD93F9041011FB02F11A881144C6
:1001600009B2A0F8441093F904201B8812FB04F292
:1001700013441BB29942D2BFA0F84830A0F84810EF
:10018000A0F84430E5E700BF000B002090F95030A4
:10019000214A002B836AB4BF018A418A002B08BF21
:1001A000134610B5B0F90E40C2890C44997BA4B235
:1001B000C1B193F9041011FB02F11A88114409B27C
:1001C000A0F8441093F904201B8812FB04F2134496
:1001D0001BB29942D2BFA0F84830A0F84810A0F84E
:1001E000443010BD93F9051011FB02F15A881144F7
:1001F00009B2A0F8461093F905205B8812FB04F2BF
:1002000013441BB29942D2BFA0F84A30A0F84A105A
:10021000A0F84630E5E700BF000B00202DE9F04FC5
:10022000964685B0A0F814E01EFB03FE1FFA8EFE72
:10023000BEF5807F0446A0F816E04FF0040C34BFF2
:1002400001200220BCFBF0FCBDF83CA0BDF84060E2
:10025000BDF84C2006FB0AF50292BDF85020AC45D3
:100260000E9FBDF84490BDF84880BDF854B0019190
:10027000039240D30020BEF1FF0F606209D804F161
:10028000230E85420ED0013084450EF801BFF8D10F
:1002900008E004F1220E854204D0013084452EF896
:1002A00002BFF8D10120029B1AFB09F1A381039B35
:1002B0006683E381019B16FB08F6C4E901374FF61C
:1002C000FF732387A387B4F85030218223F47E7311
:1002D00043EAC003A4F8503000232149A362214B14
:1002E000A4F818A08B426682A4F81C90A4F81E8083
:1002F0001BD137F06DFBBEF1FF0F0CD96D00284606
:100300003EF0EBFF844605442CF802BBAC45FBD124
:1003100060620020C7E728463EF0DFFF84460544C0
:100320000CF801BBAC45FBD1F2E70F498B42E0D0A2
:100330000E498B42DDD00E498B42DAD00D498B42FB
:10034000D7D0BA0709D13968994206D12146384633
:1003500005B0BDE8F04F03F09FBD05B0BDE8F08FDC
:10036000688C070878820708F4980708B48607089D
:100370008C8C0708F88C070808B5034693F85020C2
:10038000084642F00202996083F850200E490F4A55
:100390008A4201D137F01CFB0D498A42FAD00D493F
:1003A0008A42F7D00C498A42F4D00C498A42F1D0F3
:1003B000810707D10168914204D11946BDE8084080
:1003C00003F06ABD08BD00BF688C07087882070883
:1003D000F4980708B48607088C8C0708F88C07087F
:1003E00070B5C68A9E4202D80C4811F061F890F8A8
:1003F000504024070DD500F12405048BFF2E02FB8D
:1004000004148CBF25F814302B55BDE870403CF027
:100410008CB8456A002DF0D170BD00BFE994080882
:100420002DE9F04FA9B0109390F850300546180709
:100430009046039140F1ED8005F12403099395F86E
:100440005130990740F0EA8005F1440739464046AB
:100450001EAA47F014FB002800F0E080404647F059
:1004600091FBAA6A95F85030917BC3F38016B1EBEB
:10047000D31FC3F3401402BF334626461C461379EC
:10048000B6EBD31F00F0D080B8F90430B8F90010F3
:100490005B1A013B9BB208934FF0FF3306935379ED
:1004A000B4EBD31F40F0C48003B21EA940460793AB
:1004B00047F07CFBAB6A95F850C09A7B59790F9056
:1004C000187921AB86EAD010CDE9007382EADC12FC
:1004D0001EAB84EAD11147F075FBB5F84420BDF896
:1004E00084309B1A99B21BB20A93BDF888301491DC
:1004F0009B1AB5F84610BDF886201BB2521A179306
:1005000093B212B21892BDF88A20521AA96A12B296
:1005100019920A79B6EBD21F15BFBDF87C00B8F866
:100520000000B8F80420BDF87820121A92B212B276
:100530000E924A79B4EBD21F15BFBDF87E00B8F811
:100540000200B8F80620BDF87A20121A92B212B250
:1005500095F850000D928A7BB2EBD01F01BFDDE908
:100560000D02CDE90D20DDE90602CDE906208A79EC
:100570000592AA8B0B922A8B0C92199AADF89630A1
:1005800093424DDA189A0E999A1A0A440699E88B02
:1005900012FB01F208996C8B0A4492B21592059AEB
:1005A000B3FBF2F3B3FBF0F16A8C00FB11330A44A6
:1005B000B2FBF4F604FB162294B21A940C9C169328
:1005C00014FB02F292B20A9B1B92059A93FBF2F77C
:1005D00002FB17390B9B002297FBF3F603FB167700
:1005E0002B8CCDE912221E4496FBF4F34FF0FF3220
:1005F00004FB1366149B1FFA89F93FB2B6B2179930
:10060000ADF894308B4220DBBDF8963001339BB2BD
:10061000B3E76B6A0993002B7FF411AF00230F93AC
:100620000F9829B0BDE8F08F00230893012335E728
:10063000B8F90220B8F906309B1A089A013B13FB5F
:1006400000239BB2089340422EE70A99994213D0A7
:10065000059909F101091FFA89F949450CD10B994E
:1006600001373FB2B94205D10C990136B6B2B14259
:1006700057D000274FF000090A995C1A0D9B1C44C3
:10068000079B14FB03F4159B1C4424B2002CA346C7
:10069000B8BF04F11F0B614201F01F0104F01F03FA
:1006A00058BF4B42012101FA03F31193109B4FEA0B
:1006B0006B1B53F82B301199194240F04781E98A9E
:1006C0001B9BFF29334409999BB28CBF11F813A0DF
:1006D00011F803A092458DF898A00ED0AB8A0B9923
:1006E000BAFBF3F203FB12A313FB01F31BB2129349
:1006F000EB8B13FB02F31BB21393129B169AD919BF
:10070000139B94489A1800231C932493924B89B20C
:1007100092B28342ADF89A10ADF89C2005D137F023
:1007200057F900263746B146A6E78C4B8A489842CF
:10073000F5D08B4B9842F2D08A4B9842EFD08A4B3F
:100740009842ECD06B6813F0030C049349D11B68FA
:10075000834246D1049812B209B23CF036F8249094
:1007600001237C4A8DF87430804B9342D7D07B4A6A
:100770009342D4D07A4A9342D1D07A4A9342CED08F
:10078000794A9342CBD0A86882070AD102689A427C
:1007900007D11A9B0399CDE9006324AA1CAB03F08F
:1007A000E7FAA8680E283DD1249B1C939DF874306D
:1007B000002B00F0CD80109B119A53F82B3013437F
:1007C000109A42F82B30039B1B78102B6BD11C9B8B
:1007D000329A22F81430BDF89430524601339BB25D
:1007E0000DE7634B5B48834299D0DFF870E17345B6
:1007F00095D0DFF86CE1734591D0DFF868E173457F
:100800008DD0DFF864E1734589D0BCF1000FA7D12A
:10081000049800689842A3D1049812B209B23BF040
:1008200035FF9CE7534B4B4A93423FF478AF4B4A1A
:1008300093423FF474AF4A4A93423FF470AF494A3F
:1008400093423FF46CAF484A93423FF468AF10F0D4
:10085000030208D10168994205D103991CAB24AA6F
:1008600047F02EFAA2E7444B3A498B423FF457AF88
:100870003A498B423FF453AF39498B423FF44FAF73
:1008800038498B423FF44BAF37498B423FF447AF77
:10089000002A8BD102689A4288D103991CAB24AA02
:1008A0003CF02BFA82E7202B04D11C9B329A42F8B1
:1008B000243090E7182B0BD1329B04EB4404BDF895
:1008C00070109DF872203298234401539A7082E789
:1008D000082B03D11C9B329A13557CE7072B3FF65C
:1008E0007AAF4FF0080BBBFBF3FB039B9B7A8BB9F2
:1008F000404647F047F994FBF0F18BB2B3FBFBF2B3
:1009000000FB114112FB00100BFB123310FB0BF02C
:10091000184404B2039B03991A7894FBFBF30BFB76
:10092000134414FB02F4C97AE4B239B10BF1FF3B72
:100930001BFB02FBABEB040B5FFA8BF432991C9AA6
:10094000C95CA2400A433299CA5444E7924642E73E
:100950000F9340E7688C070840780708F498070869
:10096000B48607088C8C0708F88C0708788207087B
:1009700094770708A4750708207907082DE9F8433C
:10098000B0F93830B0F93C200446934211D090F8C9
:10099000511088070DD0A38794F85030314ADFF802
:1009A000E09023F007034A4584F850300ED137F029
:1009B0000FF894F85010490701D49342ECD104F198
:1009C000380104F1440047F03CF8E5E7DFF8B48073
:1009D0004245ECD0244FBA42E9D0244EB242E6D090
:1009E000234DAA42E3D0A06810F0030119D1036897
:1009F000934216D147F0A8F91E4B4B45D7D043453B
:100A0000D5D0BB42D3D0B342D1D0AB42CFD06068B7
:100A1000820719D102689A4216D1BDE8F8433BF02B
:100A20001BBF154B4B45C2D04345C0D0BB42BED0C7
:100A3000B342BCD0AB42BAD00029DDD102689A42A1
:100A4000DAD13CF0A8F9D7E70C4B4B45AFD0434582
:100A5000ADD0BB42ABD0B342A9D0AB42A7D0BDE82A
:100A6000F88300BFA4750708B48607088C8C0708B4
:100A7000F88C07084078070820790708947707085A
:100A8000688C0708F49807082DE9F84F90F8512072
:100A9000824697070C46B0F93860B0F93C500DD04B
:100AA00042F00402AE4280F8512003D12546284688
:100AB000BDE8F88F016400F13805F8E790F85020A0
:100AC00050071FD5AE421DD00AF12C050AF1380798
:100AD0000AF144062A463146384647F020F82846AF
:100AE00047F05AF8BAF81020BAF812104A43B0EB9F
:100AF000420F89BF3546CAF83440CAF84040CAF8A8
:100B00004C70D4E7724ADFF8DCB15A4501D136F0B7
:100B10005FFF704B9A42FAD0DFF8CC914A45F6D08D
:100B2000DFF8C8814245F2D06B4FBA42EFD0DAF815
:100B30000400810715D10168914212D121463BF092
:100B40007CFE84420DD0BAF81620012A1ED10AF18B
:100B50002C0146F076FF9AF8502042F001028AF804
:100B600050209AF85020920715D501229AF850008B
:100B700062F3410087078AF85000C1B201D4AE4247
:100B80003BD1CAF84C400AF1440590E79AF850204E
:100B900042F00202E3E7514A5A45B8D04D4B9A421F
:100BA000B5D04A45B3D04245B1D0BA42AFD0DAF859
:100BB0000800830717D04A495945A8D0454B9942A8
:100BC000A5D04945A3D04145A1D0B9429FD0DAF87C
:100BD000080010F003020ED107688F42C6D13CF026
:100BE000D8F80246C2E701689142E4D147F0AAF87A
:100BF0000028BAD1DFE70022B8E7CD077FF556AF6E
:100C0000DAF82860BAF90CC0B37BBAF90E8013B9D0
:100C10004246E04694468806BAF92C20BAF930706C
:100C200005D5BAF81000821AC01B12B207B24D06E1
:100C3000BAF92E00BAF932E007D5BAF81250281ADC
:100C4000A5EB0E0500B20FFA85FEB3EBD11F05D15F
:100C50007146BE460F46014610460A4696F90410F4
:100C6000404411FB00F130886244014409B2AAF803
:100C70002C1096F905500EEB080015FB02F5728852
:100C8000674415442DB2AAF82E5096F9042012FBA1
:100C900000F23088024412B2AAF8302096F905001A
:100CA000768810FB07F0304400B28542CABFAAF82C
:100CB0003250AAF83200AAF82E009142C4BFAAF816
:100CC0003010AAF82C20CAF834400AF12C05EEE6C0
:100CD00040780708F4980708F88C0708A4750708F7
:100CE00020790708688C0708B48607088C8C0708E9
:100CF0002DE9F04700228A46A6B00446816102AB86
:100D00001146504602923FF07CFF029808B111F064
:100D100081FB01231A220093504602AB03A93FF046
:100D20007FFE034602980028F1D11A2B05D102223A
:100D30006E4903A853F0BFFE18B140F2DB3012F049
:100D4000CBFADDF81A50282D03D025F010036C2BB8
:100D500018D10123A5F10C060093324602AB504690
:100D60000DF126013FF05CFE034602980028CED12B
:100D70009E42E2D1DDF82A3053B1032B08D05C4803
:100D800010F096FB0C2DF5D029465A4810F0C8FB00
:100D9000DE1E7342734184F82030BDF82830DDF840
:100DA000162084F82130DDF81E305349A380DDF889
:100DB00022302281E38024203EF0EDF90022064615
:100DC00011463BF06FFD94F82130E661102B2DD1D8
:100DD000372D02D894F8203003B3DDF84230E360B9
:100DE000DDF846302361DDF84A30636194F8212054
:100DF000A388072A71D90820B0FBF2F0D108002897
:100E00006BD111FB03F2910793B203D023F00303DC
:100E100004339BB2638126B0BDE8F0874FF478734A
:100E20004FF4F840C4E903031F23DEE7082BDDD8A5
:100E3000272D02D9DDF83A600EB901269E402F49D0
:100E400010203EF0A8F91FFA86F90022494607460D
:100E500046F000FF012E34D04FEA89091FFA89F9C4
:100E600048463EF03AFA0E3580460022504602AB24
:100E7000A9B23FF0C6FE029800287FF448AF0123D4
:100E80004A460093414602AB50463FF0C9FD034637
:100E9000029800287FF43BAF994501D018486FE7CE
:100EA00005460146013558F82120ADB2384646F0D6
:100EB000F5FEB5422946F5D340463EF021FAE761FA
:100EC00094E700223846114646F0E8FE6FF07F4274
:100ED0003146384646F0E2FEF1E75343DA061CBFDE
:100EE00023F01F032033C3F3CF0393E7C53908086A
:100EF000F9950808A696080820790708A475070838
:100F00002B94080808B5FDF789FB10B9FDF71CFF05
:100F100070B108BD0D4A934203D1BDE808403CF0D2
:100F2000E7BC0B4A9342F4D1BDE8084001F0CEB9CA
:100F300008480368002BECD0074A9342E9D0074ADF
:100F40009342E7D1BDE8084045F09FBFDC7C07082D
:100F5000B47A0708183500208C8C0708E0BE070813
:100F60004FF0FF3370B5204E204C336023682BB90F
:100F70003368E3B9BDE87040FEF796B91C4DAB424B
:100F8000F6D01C4A934204D1204645F097FF2560D5
:100F9000EEE7194A934203D1204601F0C7F9F6E77C
:100FA000164A9342F3D1204601F02CFDEFE7144C92
:100FB0002368002BDED00E4DAB42DBD0114A9342AA
:100FC00004D120463CF069F92560D3E70E4A9342EC
:100FD00003D1204601F094FEF6E70C4A9342F3D188
:100FE000204602F0EBFBEFE7E40700201835002075
:100FF0008C8C0708E0BE0708B47A0708DC7C070879
:10100000DC3C0020547C0708587E07083481070820
:10101000F8B5334C334E23680BB1B3420DD1266083
:1010200031480368002B59D0B34257D02F4A93421E
:1010300046D1BDE8F84019F03DBF2D4A934216D184
:101040006568A54203D304F1AC039D42E8D9284664
:1010500009F02EFB0028E3D0264B782229461846BB
:1010600053F0FBFC6060284645F0B7FFD8E7224A02
:1010700093421ED16568A54203D304F1AC039D429F
:10108000CED9284609F014FB0028C9D0194A2B46AE
:10109000944605F1280E174618685968083303C7A7
:1010A00073453A46F7D12846C4F804C046F075F9AE
:1010B000B6E7124A9342B3D120463DF0E3F9AFE7D9
:1010C0000F4A934203D1BDE8F84001F05BB90D4AE5
:1010D000934203D1BDE8F84001F0A6BCF8BD00BFC3
:1010E000DC3C00208C8C070818350020E0BE070887
:1010F000547C0708E43C0020587E07083481070828
:10110000B47A0708DC7C070808B5144803681BB9E3
:10111000134803684BB908BD124A9342F8D0124AEB
:101120009342F5D13DF038FAF2E70E4A9342F2D0FD
:101130000E4A934203D1BDE8084045F0CEBE0C4AAA
:10114000934203D1BDE808403CF0EBBB094A93420F
:10115000E1D1BDE808403CF036B800BFDC3C0020DF
:10116000183500208C8C070834810708E0BE07087A
:10117000DC7C0708B47A070810B5084B084C1B68DC
:10118000A34200D043B9BC220021064853F08BFC97
:10119000044840F8044D10BD0020FCE7183500203D
:1011A0008C8C07081C35002008B5FFF7E5FF10B947
:1011B000014810F08DF908BDAA94080810B5084B35
:1011C000084C1B680BB1A34208D1A8220021064895
:1011D00053F069FC044840F8044D10BD0020FCE7C2
:1011E000DC3C00208C8C0708E03C002008B5FFF7B1
:1011F000E5FF10B9014810F06BF908BDB09408087C
:10120000094B1B685A1C0DD0002B0BDCC02253432A
:10121000064A9818D358064A934203D0002B08BFB9
:101220000E2070470E207047E4070020183500207C
:101230008C8C07080E2807B506D14FF0FF330D4AF6
:10124000136003B05DF804FB0B4B98421A6803D19E
:101250000A4B9A4200D05AB906F0CAF8C388E6226F
:10126000009340F2171140F25D13054810F06CF93D
:101270000023E4E7E4070020183500208C8C0708E1
:10128000969C0808074A1368013304D1064B0749A6
:101290001B688B4200D17047002BFCD000231360E9
:1012A000704700BFE4070020183500208C8C070829
:1012B0002DE9F041044603FB01F5984600231F3554
:1012C00006986D090E461746A180E280A58184F834
:1012D000233038B9A8B2504380003DF0FEFF01230F
:1012E00084F823309DF81C30B8F1080FA06084F812
:1012F000223084F80E8008D9B8F1100F05D0B8F16B
:10130000200F02D00E4811F045F808220020B2FB51
:10131000F8F201239A420FD80123E07303FA00F098
:1013200003FA08F3013B238400230138206126835C
:1013300063616783BDE8F0810130C0B25B00E9E71B
:1013400006980808F0B590F82260054687B016B1F7
:101350000D4810F0BDF807C905F114078DE8070026
:10136000684646F0CBFB6A463946684646F0D7FBEE
:101370006B683A46684603A9CDE90436039646F001
:101380007EFB07B0F0BD00BFDF950808F8B590F808
:10139000224014B11E4810F09BF8002928DB8488F5
:1013A000A14225DA002A23DBC488A24220DA8489FC
:1013B00085686243847B05EB8205072C19D80822D7
:1013C000B2FBF4F2068CC77B006941FA07F70140D3
:1013D000521A013A12FB04F215F807C0D2B206FA0B
:1013E00002F11E402CEA0101964041EA0603EB554A
:1013F000F8BDE408012C01D16B54F9E7022C02D1AD
:1014000025F81130F4E7042C08BF45F82130EFE748
:10141000DF950808F0B51F4690F8223006460C46C6
:10142000154685B013B10D4810F052F8ADF80620FE
:101430004A1CADF80410ADF8082001A96A1CADF8EB
:101440000A200393FFF77EFF3B462A46214630469B
:1014500005B0BDE8F040FFF799BF00BFDF95080871
:10146000F0B590F8225004460E4685B015B11348E9
:1014700010F02EF8436801A9CDE902350195FFF778
:1014800061FF2022A17B2846B2FBF1F2C1F12007C7
:10149000954207D10023A289E1884A439A4208D89D
:1014A00005B0F0BD238C01353340BB4018437F1A93
:1014B000EEE7A26842F823000133ECE7DF95080865
:1014C0004EF64D4180EA503000FB00F30A4A9FED92
:1014D0000B7A01FB03220A4B00FB023323F000438B
:1014E00007EE903AFAEEE07A67EE877AFCEEE77A5A
:1014F00017EE900A704700BF1F07310100007F43BD
:101500000DDD085208B54369B3F1807F02D002486F
:101510000FF0DEFF416108BD909608081FB5084630
:1015200011461A4602AB01930D4B0093022341F082
:101530006FF80C4910203DF02EFE40F25E33044659
:1015400047F6FF720121029811F0CAFD9DF80C20A8
:1015500081B2204646F07EFB204604B010BD00BF9D
:1015600094750708A47507082DE9F04786B004466E
:101570000192104652B3444BDFF83C914B4501D1E8
:1015800036F026FADFF834814345F9D03F4FBB42AD
:10159000F6D03F4EB342F3D03E4DAB42F0D011F007
:1015A000030002D10A689A4210D00A460023A168BB
:1015B000394806F095F982460198042809D1514628
:1015C000204646F079FB400040F0010006B0BDE83F
:1015D000F087324B4B45D3D04345D1D0BB42CFD01F
:1015E000B342CDD0AB42CBD010F0030202D10168A0
:1015F00099420ED02A4B4B45C2D04345C0D0BB4286
:10160000BED0B342BCD0AB42BAD062B902689A42F3
:1016100009D124480022037A012100EB83031D69CC
:1016200001ABA8470190012203A906F08FFAE8B1A7
:10163000059B23F02002422A04D0012B02D01A4835
:101640000FF036FFDDE90332033A012A0CD85A784D
:10165000197812029B7842EA01421A432046514609
:1016600046F01CFB0E20B1E71048E9E7019802A9FB
:1016700005F0ECFF30B1029AB2F1807FEED30C4856
:101680000FF05AFF0B48FBE7609A0708B48607087B
:101690008C8C0708F88C0708A4750708449807087D
:1016A000B893070888890708D18F0808F58F0808BC
:1016B000BC8F0808E58F0808688C0708F4980708AD
:1016C00030B587B0084611461A4603AB01930D4B5F
:1016D0000093032340F09CFF4FF4A76347F6FF728B
:1016E0000121039811F0FCFC074905462C203DF030
:1016F00052FDDDE904230446294646F028FB204636
:1017000007B030BD347607085476070810B507498E
:101710003FF013FC044620B94FF4A17104480FF0C8
:10172000FFFE0AF089FE204610BD00BF5476070870
:101730006C970808F8B50E4615460746FFF7E6FF12
:10174000044646F0F8FBB0EB660F05D12946384653
:101750003BF0F3FB0E20F8BD204646F0ECFB324692
:1017600001460023044806F0BBF82A4601462046FD
:1017700046F0BAFBEEE700BF5476070810B50C46FA
:10178000FFF7C4FF214646F0C8FB002802DA0348F1
:101790000FF08EFE400040F0010010BDF3890808F4
:1017A0001FB50C4603AB01930D4B04310093013878
:1017B000012311F0EDFB2068FFF7A8FF044646F077
:1017C000BAFB039A01465200002342F00102054889
:1017D00006F086F80146204646F094FB04B010BDA2
:1017E0004C7607085476070810B504460846FFF7FC
:1017F0008DFF46F0A0FB042C03D0052C07D0002061
:1018000010BD80B200280CBF1E203E20F8E7034B1D
:1018100003EA400040F00100F2E700BFFEFF0100D4
:1018200070B515460E46FFF771FF1B4B1B4A044669
:10183000934201D136F0CCF8194A9342FAD0194AB2
:101840009342F7D0184A9342F4D0184A9342F1D009
:10185000B20705D132689A4202D1154810F09AFDBC
:10186000204646F068FB002301463246114806F048
:1018700037F8042D014604D12046BDE8704046F0FB
:101880005DBB25B9204646F03DFB0E2070BD2A46C3
:1018900020461AF0B5FFF8E7609A0708688C070839
:1018A000F4980708B48607088C8C0708F88C07089A
:1018B0008A9508085476070838B51C46084611462C
:1018C0004FF0021211F03CFB2468114B2340062B11
:1018D00005D0A3070AD122680E4B9A4206D12146B1
:1018E00044F686720C4840F000FD0446204603F0A2
:1018F00089F810B909480FF01FFE094924203DF06E
:101900004AFC05462146FFF7F3F9284638BD00BFDB
:101910000F0080FFB4860708A8860708948E080881
:1019200094770708F0B50C460646174654F8045B52
:101930008BB028463BF051FB06AB0193134B3A4664
:1019400021460093701E042311F022FB0023CDE9F1
:101950000433069B2846ADF80C30079BADF80E30DB
:10196000089B591C0CBFB5F904301BB2ADF8103000
:10197000099B03A95A1C0CBFB5F906301BB2ADF880
:101980001230FFF7DFFC0E200BB0F0BD2078070807
:101990000E2AF7B506460D46174602D13D480FF010
:1019A0008FFD3BF01AFB3C4B3C4A934201D136F091
:1019B0000FF83B4A9342FAD03A4A9342F7D03A4A58
:1019C0009342F4D0394A9342F1D0AA0705D12A684C
:1019D0009A4202D1364810F0DDFCEB0720D5B288E0
:1019E000F3886C105343B3EB650F05D800225C21DC
:1019F000013B30480FF088FD94FBF2F002FB1044ED
:101A0000A4B280B2042F24B205B22AD12A462146BC
:101A100030463AF0DAFE400040F0010003B0F0BD7D
:101A20000221284601AA05F047FF019B18683DF0F6
:101A3000ECFB041EB38801DB9C4204DB00224FF464
:101A4000C161013BD5E7019B58683DF0DEFB0028F2
:101A5000F38801DB9842D3DB002240F20E61013BA8
:101A6000C7E738463DF0D1FB074630463AF0ABFEBB
:101A70004FF0FF32C0F12000C240A22300213846BF
:101A800011F02EFB2A46034621463046FFF7C2FCE2
:101A90000E20C3E70C9A0808609A0708688C0708AC
:101AA000F4980708B48607088C8C0708F88C070898
:101AB0008A950808BB9C0808F8B51C4608461146DC
:101AC0004FF0061211F03CFA20683DF09EFB40F208
:101AD000FC5347F6FF72002111F002FB06466068D6
:101AE0003DF093FB40F2224347F6FF72002111F0D4
:101AF000F7FA0746A0683DF088FB40F2EF534FF439
:101B00008032012111F0ECFA0124013830FA04F39B
:101B10000BD1084924203DF045FB054623463A46B3
:101B200031463AF034FE2846F8BD072C94BF6400D5
:101B30000834EBE74078070830B585B00846114611
:101B40001A4602AB01930D4B0093022340F060FD57
:101B50000B4924203DF01FFB0399044640F23E420E
:101B600008489DF808503EF0A1FE2946C2B2204622
:101B70003AF098FE204605B030BD00BF1079070846
:101B800020790708C4C907082DE9F04F04464FF033
:101B9000000887B0CDE90312059300F15009059BB9
:101BA000984502D307B0BDE8F08F049B03EB08060D
:101BB00094F8BD30757896F901B0002B35D0B57822
:101BC00006F1030A48461AF0B9FB98B301230093C3
:101BD0000021334694F8BE20206D276EB84700954B
:101BE0005346012194F8BE20206D276EB847484621
:101BF00045F0E4FDBBF1000F23DB00203CF060FE6C
